:100000000C94172B0D94020F0D94D70E0D94AC0E7B
:100010000D94810E0D94560E0D942B0E0D94000E22
:100020000C9413CF0C94482B0C94482B0C94482B15
:100030000C94482B0C9471B50C94482B0C94482BC1
:100040000C94482B0C9496C70C94482B0C94482B7A
:100050000C94482B0C94482B0C94FDC50D942D0F3B
:100060000C94482B0C9459CE0C94482B0C94482B90
:100070000C94482B0C94482B0C94482B0C94482B34
:100080000C94482B0C94482B0C94482B0C94482B24
:100090000C94482B0C94482B0C94482B0C94482B14
:1000A0000C94482B0C94482B0C94482B0C94482B04
:1000B0000C94482B0C94482B0C94482B0C94482BF4
:1000C0000C94482B0C94482B0C94482B0C94482BE4
:1000D0000C94482B0C94482B0C94482B0C94482BD4
:1000E0000C94482BF24FF74FFC4F0650105089509C
:1000F0001A5022502A5034503E50485057506150A8
:1001000089506B5075507F50297829783078307835
:10011000307837783778377844783E783E783E784C
:100120008DCE93CEA4CEAFCEB7CECCCEBBCECCCEE2
:10013000BFCEC3CECCCEC9CEF200F0000201D600B5
:100140000A01E2000001FE00F400D4000801D8001A
:10015000FC00EE00E200E400E800DC00084AD73BC7
:100160003BCE016E84BCBFFDC12F3D6C74319ABD86
:1001700056833DDA3D00C77F11BED9E4BB4C3E91AA
:100180006BAAAABE000000803F05A84CCDB2D44E99
:10019000B93836A9020C50B9918688083CA6AAAA9B
:1001A0002ABE000000803F000D94EB050D94CC05A5
:1001B0000D94F5050D94E2140D940B060D945F0C4F
:1001C0000D94BA050D9410060D9403060D948A053E
:1001D0000D9407060D9479050D947C050D94FD058D
:1001E0000D94D9050D94D6050D94E7050D949C1337
:1001F0000D946A0A0D94BC050D94F9050D94E10562
:100200000D94DD050D94C8050D9478050D945005E9
:100210000D94EF050D94D205434F4D4D554E494376
:100220004154494F4E0044525952554E0045525286
:100230004F525300494E464F004543484F002074EB
:100240006F6F206C6F6E6720657874727573696F5D
:100250006E2070726576656E7465640A0020636F47
:100260006C6420657874727573696F6E2070726546
:1002700076656E7465640A0047322F4733206261E9
:100280006420706172616D65746572730A00536CED
:100290006565702E2E2E00205A3A200020593A20F3
:1002A0000042656420583A20004C756C7A426F74A5
:1002B0002054415A20362072656164792E005265BF
:1002C00073756D696E67207072696E7400436C6936
:1002D000636B20746F20726573756D652E2E2E0012
:1002E0004E6F206D6F76652E00456E642066696CDA
:1002F00065206C6973740A00426567696E206669DF
:100300006C65206C6973740A004D313235005344BA
:10031000207072696E74696E67206279746520005E
:100320004E6F74205344207072696E74696E670A50
:100330000046696C652064656C657465643A0044C8
:10034000656C6574696F6E206661696C65642C20EC
:1003500046696C653A20006F70656E206661696C55
:1003600065642C2046696C653A2000256973002578
:10037000696D20256973002569682025696D202530
:10038000697300256964202569682025696D202529
:10039000697300256979202569642025696820250D
:1003A000696D20256973005072696E742074696DDF
:1003B000653A2000000125301D0C1824311C0B1754
:1003C000232F1B0A1E16040308060202222B1A41C1
:1003D00042033809FF3628294527444350726F7479
:1003E00065637465642050696E0A0045787472759F
:1003F000646572202573004C756C7A426F742054CA
:10040000415A20362072656164792E003902340227
:100410002D02260218026F66660044454255473A8F
:10042000006F6B00436F6F6C696E6720646F6E6561
:100430002E0048656174696E6720646F6E652E00DA
:1004400020573A00457874727564657220257300F0
:100450004C756C7A426F742054415A203620726574
:100460006164792E0042656420646F6E652E002001
:10047000573A004265642068656174696E672E00B2
:1004800042656420636F6F6C696E672E002F2F20AA
:10049000007A5F70726F62653A20007A5F6D6178F2
:1004A0003A20007A5F6D696E3A2000795F6D61785D
:1004B0003A2000795F6D696E3A2000785F6D61784F
:1004C0003A2000785F6D696E3A20005265706F7255
:1004D00074696E6720656E6473746F7020737461E5
:1004E0007475730A00426564204C6576656C696EAC
:1004F0006720004661696C656420746F20656E61D9
:10050000626C6520426564204C6576656C696E6737
:100510000A00426564204C6576656C20436F7272F8
:10052000656374696F6E204D61747269783A004E2C
:100530006F2063617365206C696768740A004163AA
:10054000746976652045787472756465723A200026
:10055000556E6B6E6F776E20636F6D6D616E643A72
:1005600020220020204E6F7A7A6C653A200020000D
:1005700066696C616D656E7420756E6C6F61640088
:100580005761697420666F72005052494E54205072
:1005900041555345440020204E6F7A7A6C653A20CD
:1005A000006368616E6765006F6620746865206629
:1005B000696C616D656E74005761697420666F7255
:1005C000207374617274005052494E54205041554A
:1005D0005345440020204E6F7A7A6C653A20002003
:1005E000004261636B004D696E696D756D205465E5
:1005F0006D70206973203132302E00486561746956
:100600006E67206661696C65640025753A25303235
:100610007500253032753A25303275002575642015
:10062000253032753A253032750000060900FE008B
:100630000000000001090008FE000005080806008F
:100640000040F0C88888987810050808060000C0A7
:10065000F88888888888F80505050600012030F8A4
:1006600030200508080600002070F820202020E037
:100670000509090600FF2070A8A8B8888870200521
:1006800009090600FFE080C0B0A828302828050925
:10069000090600FFF8A88888888888A8F8050A0A4B
:1006A0000600FE205050505088A8A888700303030D
:1006B00006000340A04000060900FE070192032146
:1006C00020FFFF08FF07FF000000060000010707EA
:1006D00006020080808080800080030202060105FF
:1006E000A0A00507070600005050F850F85050052C
:1006F00007070600002078A07028F02005070706ED
:100700000000C0C8102040981805070706000060C8
:1007100090A040A89068020303060104C040800333
:10072000070706010020408080804020030707065D
:1007300001008040202020408005050506000120A2
:10074000A870A8200505050600012020F820200239
:1007500003030602FFC04080050101060003F80202
:100760000202060200C0C0050505060001081020AF
:100770004080050707060000708888888888700315
:10078000070706010040C040404040E0050707065B
:100790000000708808708080F8050707060000F8E0
:1007A0001020100808F005070706000010305090D0
:1007B000F81010050707060000F880F00808887098
:1007C000050707060000708080F08888700507071D
:1007D000060000F80810202020200507070600006A
:1007E0007088887088887005070706000070888800
:1007F00078080870020505060200C0C000C0C002EB
:1008000006060602FFC0C000C040800407070600BD
:100810000010204080402010050303060002F8006D
:10082000F8040707060100804020102040800507DB
:100830000706000070880810200020050707060042
:100840000070880868A8A87005070706000070886F
:1008500088F8888888050707060000F08888F088EF
:1008600088F0050707060000708880808088700582
:100870000707060000F08888888888F005070706C3
:100880000000F88080F08080F8050707060000F877
:100890008080F0808080050707060000708880B89F
:1008A000888870050707060000888888F888888887
:1008B000010707060200808080808080800507078E
:1008C00006000038101010109060050707060000A1
:1008D0008890A0C0A090880507070600008080804F
:1008E000808080F805070706000088D8A8888888D7
:1008F000880507070600008888C8A8988888050723
:100900000706000070888888888870050707060039
:1009100000F08888F0808080050707060000708856
:100920008888A89068050707060000F08888F0A06E
:100930009088050707060000788080700808F00599
:100940000707060000F820202020202005070706C2
:100950000000888888888888700507070600008856
:1009600088888888502005070706000088888888BE
:1009700088A85005070706000088885020508888FE
:1009800005070706000088888850202020050707F3
:10099000060000F80810204080F803070706010051
:1009A000E08080808080E005050506000180402011
:1009B0001008030707060100E02020202020E005A2
:1009C0000303060004205088050101060000F80218
:1009D0000202060205804005050506000070087841
:1009E00088780507070600008080B0C88888F00571
:1009F0000505060000708080887005070706000066
:100A0000080868988888780505050600007088F849
:100A100080700507070600003048E0404040400570
:100A200006060600FF70888878087005070706002C
:100A3000008080B0C888888801070706020080000F
:100A400080808080800308080601FF20002020208D
:100A500020A040040707060000808090A0C0A0905E
:100A6000030707060100C04040404040E00505057F
:100A7000060000D0A8A8A8A8050505060000B0C873
:100A80008888880505050600007088888870050636
:100A9000060600FFF08888F080800506060600FF45
:100AA000788888780808050505060000B0C88080A9
:100AB0008005050506000070807008F00407070631
:100AC00000004040E0404040300505050600008839
:100AD00088889868050505060000888888502005E4
:100AE00005050600008888A8A85005050506000031
:100AF00088502050880506060600FF8888887808F8
:100B000070050505060000F8102040F803070706E9
:100B1000010020404080404020010707060200807D
:100B2000808080808080030707060100804040208D
:100B300040408005020206000268900000000600A6
:100B40000000000006000000000006000000000099
:100B50000600000000000600000000000600000083
:100B60000000060000000000060000000000060073
:100B70000000000006000000000006000000000069
:100B80000600000000000600000000000600000053
:100B90000000060000000000060000000000060043
:100BA0000000000006000000000006000000000039
:100BB0000600000000000600000000000600000023
:100BC0000000060000000000060000000000060013
:100BD0000000000006000000000006000000000009
:100BE00006000000000006000000000006000000F3
:100BF00000000600000000000600000000000600E3
:100C000000000000060000010707060200800080C7
:100C1000808080800507070600002070A8A0A870CB
:100C200020050707060000304040E04050A80505B9
:100C300005060000887050708805070706000088C8
:100C40005020F820F820010707060200808080006D
:100C50008080800508080600003048205050209011
:100C600060030101060107A0050707060000F888D8
:100C7000B8B8B888F80507070600017008788878C2
:100C800000F80505050600012850A05028050303BB
:100C9000060001F808080202020602064080050765
:100CA00007060000F888A88898A8F8050101060042
:100CB00006F8040404060003609090600507070628
:100CC00000002020F8202000F8040505060003603D
:100CD000902040F0030505060003E020E020E0023C
:100CE000020206020640800508080600FF88888880
:100CF0008898E8808005070706000078989878189B
:100D00001818020202060202C0C00202020602FF16
:100D1000408003050506000340C04040E00507078A
:100D2000060001708888887000F805050506000136
:100D3000A0502850A00507070600008890A858B8C2
:100D400008080507070600008890B848982038056D
:100D50000808060000C040C048D838080805070742
:100D6000060000200020408088700508080600006A
:100D70004020007088F888880508080600001020C8
:100D8000007088F888880508080600002050007068
:100D900088F888880508080600006890007088F8C0
:100DA00088880508080600005000708888F8888840
:100DB0000508080600002050207088F8888805077C
:100DC000070600003860A0B8E0A0B80508080600D3
:100DD000FF70888080887020600508080600004049
:100DE0002000F880F080F8050808060000081000D0
:100DF000F880F080F8050808060000205000F88010
:100E0000F080F80507070600005000F880F080F831
:100E1000030808060100804000E0404040E003086D
:100E200008060100204000E0404040E003080806BA
:100E3000010040A000E0404040E003070706010039
:100E4000A000E0404040E005070706000070484869
:100E5000E848487005080806000068900088C8A89F
:100E600098880508080600004020708888888870E7
:100E7000050808060000102070888888887005081A
:100E80000806000020500070888888700508080651
:100E900000006890007088888870050808060000C7
:100EA0005000708888888870050505060001885004
:100EB0002050880508080600FF1070A8A8A8A87090
:100EC000400508080600004020888888888870054A
:100ED000080806000010208888888888700508089F
:100EE00006000020500088888888700508080600E1
:100EF000005000888888888870050808060000105F
:100F0000208850202020200509090600FFC04070DD
:100F10004848704040E00408080601FF609090A037
:100F20009090E080050808060000402000700878D6
:100F30008878050808060000102000700878887876
:100F40000508080600002050007008788878050819
:100F50000806000068900070087888780507070682
:100F60000000500070087888780508080600002006
:100F700050207008788878050606060000D028788A
:100F8000A0A8500506060600FF7080887020600546
:100F900008080600004020007088F88070050808E6
:100FA0000600001020007088F88070050808060010
:100FB000002050007088F880700507070600005078
:100FC000007088F880700308080601008040004027
:100FD000C04040E003080806010020400040C04037
:100FE00040E003080806010040A00040C04040E087
:100FF000030707060100A00040C04040E0050707C6
:10100000060000A040A010788870050808060000BF
:10101000689000B0C888888805080806000040204D
:10102000007088888870050808060000102000708D
:10103000888888700508080600002050007088889D
:10104000887005080806000068900070888888701D
:1010500005070706000050007088888870050505A0
:101060000600012000F800200507070600FF1070A9
:10107000A8A8A8704005080806000040200088883D
:10108000889868050808060000102000888888985D
:1010900068050808060000205000888888986805C0
:1010A0000707060000500088888898680509090627
:1010B00000FF102000888888F808700407070601E0
:1010C000FFC04060506040E00508080600FF500087
:1010D0008888887808705A00590058000920000054
:1010E00000000000000000000000007FFFE00000A2
:1010F000000000000000000000007000E0000000A0
:1011000000000000000000000061F8600000000026
:10111000000000000000000041F820000000000076
:101120000000000000000040F0200000000000006F
:1011300000000000000040602000000000000000EF
:1011400000000000005801A07F80000000000000A7
:10115000004104005C63A0FFC0000000000000002C
:101160002082005EF7A0FFC0000000000000002009
:1011700082005EF7A0FFC0000000000000004104F4
:10118000005C63A07F800000000000000082080077
:101190005801A07F80000000000000010410004002
:1011A0006020FFC00000000000000104100040F0BB
:1011B00020FFC00000000000000082080041F8206D
:1011C000FFC00000000000000041040061F8603F23
:1011D00000000000000000000000007000E01E00A1
:1011E00000000000000001FFFF807FFFE00C000016
:1011F000000000000001FFFF800000000000000070
:1012000000000000000000007FFFE0000000000080
:10121000000000000000007000E00000000000007E
:10122000000000000000630C6000000000000000EF
:101230000000000000470E20000000000000000039
:10124000000000004F0F2000000000000000000020
:101250000000005F0FA00000000000000000000080
:1012600000005E07A07F8000000000000000410435
:1012700000406020FFC0000000000000002082004D
:1012800040F020FFC000000000000000208200406D
:10129000F020FFC00000000000000041040040609A
:1012A000207F80000000000000008208005E07A090
:1012B0007F80000000000000010410005F0FA0FF0D
:1012C000C0000000000000010410004F0F20FFC00C
:1012D00000000000000000820800470E20FFC00050
:1012E000000000000000410400630C603F000000AB
:1012F00000000000000000007000E01E0000000080
:1013000000000001FFFF807FFFE00C0000000000F4
:10131000000001FFFF8000000000002200250028DF
:10132000002B002E003100340002010000050108EE
:10133000010B0100000A0B02090C0D0E0807030443
:10134000010000000000000000000000000000009C
:10135000000000000000000000000000000000127B
:10136000111000000000000000000000000000005C
:1013700000000000000000000043290A0061626CC8
:10138000656420286D696E2074656D702000436F60
:101390006C64206578747275646573206172652071
:1013A0000045313A200045303A20005A3A20005991
:1013B0003A2000583A20004D53312C4D53322050E2
:1013C000696E730A002042002050006F6B00526566
:1013D00073656E643A20001000C90210012C0140B0
:1013E00001220170011801B0010E01F00104015049
:1013F00002FA00B002F0003003E600D003DC0090F7
:1014000004D2007005C800A006BE000008B400B0F9
:1014100009AA00D00BA000600E960060118C00009D
:1014200015820020197800C01D6E00A0226400B053
:10143000275A00902C500000314600E0343C001048
:10144000383200903A2800603C1E00A03D14008015
:101450003E0A00203F00004361703A454D45524727
:10146000454E43595F5041525345523A310A004369
:1014700061703A434153455F4C494748545F42527B
:10148000494748544E4553533A300A004361703A35
:10149000544F47474C455F4C49474854533A300AEC
:1014A000004361703A534F4654574152455F504F85
:1014B0005745523A300A004361703A4C4556454C04
:1014C000494E475F444154413A310A004361703A02
:1014D0005A5F50524F42453A310A004361703A41D7
:1014E00055544F4C4556454C3A310A004361703AC9
:1014F0005052494E545F4A4F423A310A004361709C
:101500003A50524F47524553533A300A00436170A4
:101510003A4155544F5245504F52545F54454D50E7
:101520003A310A004361703A454550524F4D3A31C5
:101530000A004649524D574152455F4E414D453A8A
:101540004D61726C696E20204649524D574152459B
:101550005F56455253494F4E3A312E312E352E3675
:10156000342045585452554445525F545950453AD9
:101570004D4F41527374727564657220534F5552CA
:1015800043455F434F44455F55524C3A687474700D
:10159000733A2F2F636F64652E616C6570686F629C
:1015A0006A656374732E636F6D2F64696666757305
:1015B000696F6E2F4D41524C494E2050524F544F3F
:1015C000434F4C5F56455253494F4E3A312E3020CF
:1015D0004D414348494E455F545950453A4C756C0E
:1015E0007A426F742054415A20362045585452553F
:1015F0004445525F434F554E543A31205555494466
:101600003A38343566303033632D616562642D3489
:101610006535332D613662392D376430393834669B
:1016200064653630390A004D31343520533C696EDB
:101630006465783E206F7574206F662072616E67F6
:10164000652028302D31290A0020706F7369746974
:101650006F6E206F7574206F662072616E67652EE5
:101660000A003F50726F626520001000AD03300128
:101670006A0150022B0170030A019004F500B005C5
:10168000E500D006D800F007CE001009C500300AEA
:10169000BE00500BB700700CB100900DAB00B00E47
:1016A000A600D00FA200F0109D0010129900301378
:1016B00095005014920070158E0090168B00B01794
:1016C0008700D0188400F0198100101B7E00301CA8
:1016D0007B00501D7900701E7600901F7300B020B3
:1016E0007000D0216E00F0226B00102469003025BC
:1016F0006600502663007027610090285E00B029C4
:101700005C00D02A5900F02B5600102D5400302ECA
:101710005100502F4E0070304B0090314800B032D5
:101720004500D0334200F0343E0010363B003037E5
:1017300037005038330070392E00903A2900B03B02
:101740002300D03C1B00F03D1100103F0100F03F92
:10175000000020204D383531205A005A2D50726F2C
:101760006265204F666673657420286D6D293A0A9C
:101770000020440020490020204D33303420500008
:1017800020440020490020204D33303120500050AB
:1017900049442073657474696E67733A0A00204681
:1017A0000020420020480020204D313435205300D5
:1017B0004D6174657269616C206865617475702033
:1017C000706172616D65746572733A0A0020204D14
:1017D0003432302053004175746F20426564204CD0
:1017E0006576656C696E673A0A00205A00205900D8
:1017F00020204D323036205800486F6D65206F66CE
:10180000667365743A0A00204500205A002059008A
:1018100020580020420020540020204D3230352036
:101820005300416476616E6365643A20533C6D6990
:101830006E5F66656564726174653E20543C6D69D7
:101840006E5F74726176656C5F6665656472617403
:10185000653E20423C6D696E5F7365676D656E74B1
:101860005F74696D655F6D733E20583C6D61785F94
:1018700078795F6A65726B3E205A3C6D61785F7A59
:101880005F6A65726B3E20453C6D61785F655F6A9B
:1018900065726B3E0A0020540020520020204D3219
:1018A0003034205000416363656C65726174696F08
:1018B0006E2028756E6974732F7332293A20503C5C
:1018C0007072696E745F616363656C3E20523C7236
:1018D0006574726163745F616363656C3E20543C40
:1018E00074726176656C5F616363656C3E0A0020AB
:1018F0004500205A0020590020204D323031205818
:10190000004D6178696D756D20416363656C65722A
:101910006174696F6E2028756E6974732F73322934
:101920003A0A00204500205A0020590020204D325C
:1019300030332058004D6178696D756D206665659E
:101940006472617465732028756E6974732F7329CE
:101950003A0A00204500205A0020590020204D3925
:101960003220580053746570732070657220756E54
:1019700069743A0A0020204D3230302044300A0089
:1019800020204D3230302044002044697361626C65
:1019900065640A0046696C616D656E7420736574D8
:1019A00074696E67733A0020204D3134392043202A
:1019B0003B20556E69747320696E2043656C7369B2
:1019C00075730A002020473231202020203B20550B
:1019D0006E69747320696E206D6D0A003A20007A7A
:1019E0005F6D696E3A20202D32207A5F6D61783A02
:1019F000202035005A204F66667365742000506CB5
:101A000065617365207265736574005052494E5468
:101A100045522048414C544544005072696E7465EB
:101A2000722068616C7465642E206B696C6C282967
:101A30002063616C6C6564210A006265640A002C95
:101A40002073797374656D2073746F707065642191
:101A5000204865617465725F49443A2000544845E6
:101A6000524D414C2052554E415741592042454418
:101A700000546865726D616C2052756E6177617992
:101A800000544845524D414C2052554E4157415902
:101A900020453100544845524D414C2052554E414D
:101AA0005741592045300048656174696E6720666A
:101AB00061696C6564204245440048656174696EE3
:101AC00067206661696C65640048656174696E676A
:101AD000206661696C65640048656174696E6720A1
:101AE0006661696C65642045300057726974696E7F
:101AF0006720746F2066696C653A20006F70656EB0
:101B0000206661696C65642C2046696C653A20002A
:101B10006F70656E206661696C65642C2046696C27
:101B2000653A200046696C652073656C6563746571
:101B3000640A002053697A653A200046696C652082
:101B40006F70656E65643A20006F70656E20666127
:101B5000696C65642C2046696C653A2000206669D2
:101B60006C653A20004E6F7720002220706F730062
:101B70002220706172656E743A2200535542524FB2
:101B80005554494E452043414C4C20746172676561
:101B9000743A22004B494C4C45442E200074727913
:101BA000696E6720746F2063616C6C207375622DA1
:101BB00067636F64652066696C6573207769746814
:101BC00020746F6F206D616E79206C6576656C7323
:101BD0002E204D4158206C6576656C2069733A0063
:101BE0004572726F722077726974696E6720746FC4
:101BF00020454550524F4D210A00486F6D65202504
:101C00007325732573206669727374002066697288
:101C100073740A005A0059005800486F6D6520001F
:101C200000060900FE06018902FE20FFFE07FE06EF
:101C3000FE00000006000701060606020080808004
:101C4000800080030303060103A0A0A00507070688
:101C500000FF5050F850F850500509090600FE20CA
:101C600070A8A07028A870200608080600FF40A8E9
:101C70004810204854080507070600FF6090906050
:101C8000989068010303060203808080020707061C
:101C900002FF408080808080400207070602FF80AC
:101CA0004040404040800505050600008850F8503F
:101CB000880505050600002020F8202002040406FF
:101CC00002FEC0404080050101060002F802020247
:101CD000060200C0C0040606060100101020408065
:101CE000800406060601006090909090600306064E
:101CF00006010040C0404040E004060606010060C6
:101D000090102040F0040606060100F0206010103C
:101D1000E005060606000010305090F81004060694
:101D2000060100F080E01010E004060606010060E5
:101D300080E0909060040606060100F0101020403C
:101D4000400406060601006090609090600406065C
:101D5000060100609090701060020505060200C048
:101D6000C000C0C00207070602FEC0C000C040405D
:101D7000800505050600001860806018050303064D
:101D80000001F800F8050505060000C0300830C065
:101D90000407070601006090106040004005060639
:101DA0000600007090A8B0807005060606000020AE
:101DB0005088F88888050606060000F088F08888B4
:101DC000F00406060601006090808090600406061C
:101DD000060100E090909090E0040606060100F0F5
:101DE00080E08080F0040606060100F080E080803C
:101DF00080040606060100609080B090600406062C
:101E00000601009090F0909090030606060100E015
:101E100040404040E00506060600003810101090D3
:101E20006004060606010090A0C0A090900406067B
:101E30000601008080808080F0050606060000888C
:101E4000D8A8A8888804060606010090D0B0909013
:101E500090050606060000708888888870040606CB
:101E6000060100E09090E080800407070601FF6013
:101E70009090D0B06010040606060100E09090E05B
:101E800090900406060601006090402090600506D0
:101E900006060000F8202020202004060606010087
:101EA000909090909060040606060100909090F04B
:101EB00060600506060600008888A8A8D888050680
:101EC00006060000885020205088050606060000FF
:101ED000888850202020040606060100F0102040CB
:101EE00080F0030606060100E080808080E00406A2
:101EF000060601008080402010100306060601003F
:101F0000E020202020E00503030600032050880580
:101F100001010600FEF802020206020480400404E9
:101F2000040601007090907004060606010080808F
:101F3000E09090E0040404060100708080700406C4
:101F40000606010010107090907004040406010051
:101F500060B0C070040606060100205040E040401A
:101F60000406060601FE60909070106004060606E6
:101F700001008080E090909003060606010040007A
:101F8000C04040E00308080601FE20006020202039
:101F9000A0400406060601008080A0C0A0900306B1
:101FA00006060100C040404040E005040406000071
:101FB000D0A8A888040404060100E09090900404CE
:101FC00004060100609090600406060601FEE090A1
:101FD00090E080800406060601FE7090907010105C
:101FE000040404060100A0D080800404040601005B
:101FF00070C030E00406060601004040E04050207A
:10200000040404060100909090700404040601008A
:102010009090606005040406000088A8A85004049D
:1020200004060100906060900406060601FE909090
:1020300090709060040404060100F02040F0030753
:1020400007060100204040804040200107070602AB
:10205000FF80808080808080030707060100804029
:10206000402040408004020206010350A0FFFFFF11
:10207000FFFFFFFFFFFFFFFFFFFFFFFFFFFFFFFF70
:10208000FFFFFFFFFFFFFFFFFFFFFFFFFFFF00005E
:10209000000600070106060602008000808080809E
:1020A0000406060601FF2070A0A0702005070706A1
:1020B00000FF304840F04040F8050505060000A844
:1020C000508850A80506060600008850F820F82021
:1020D0000107070602FF80808000808080040707D8
:1020E0000601FF708060906010E0030101060105A9
:1020F000A0060707060000788494A494847803055A
:102100000506010160A06000E00505050600002845
:1021100050A05028040303060100F0101004010130
:10212000060102F00607070600007884B4A4A48420
:1021300078040101060105F0040303060102609022
:10214000600507070600FF2020F8202000F803059F
:102150000506010140A02040E0030505060101C07D
:10216000204020C002020206020440800405050649
:1021700001FF9090B0D08005060606000078E8E8E0
:10218000682828010101060202800202020602FEFE
:10219000408003050506010140C04040E0030505FD
:1021A00006010140A04000E0050505060000A05022
:1021B0002850A00508080600FF40C0405070307845
:1021C000100508080600FF40C04050680810380598
:1021D00008080600FFC0204030F0307810040707E0
:1021E00006010020002060809060050707060000BF
:1021F0004020205070888805070706000010202026
:10220000507088880507070600002050205070880D
:1022100088050707060000285020507088880507A9
:102220000706000050002050708888050707060048
:10223000002050205070888805060606000078A00F
:10224000F0A0A0B80408080601FE609080809060AD
:1022500020400407070601004020F080E080F004E1
:1022600007070601002040F080E080F00407070621
:1022700001002050F080E080F004070706010050C4
:1022800000F080E080F00307070601008040E04096
:102290004040E00307070601002040E0404040E0E6
:1022A00003070706010040A0E0404040E0030707A5
:1022B000060100A000E0404040E0050606060000E0
:1022C0007048E848487004070706010050A090D005
:1022D000B090900407070601004020609090906045
:1022E00004070706010020406090909060040707F3
:1022F00006010020506090909060040707060100DE
:1023000050A06090909060040707060100500060A4
:1023100090909060050505060000885020508804C4
:1023200008080601FF1070B0B0D0D0E080040707A5
:10233000060100402090909090600407070601007D
:102340002040909090906004070706010020509074
:1023500090909060040707060100500090909090C4
:102360006005070706000010208850202020040682
:102370000606010080E09090E08004060606010059
:102380006090A0A090A00407070601004020007004
:102390009090700407070601002040007090907034
:1023A0000407070601002050007090907004070792
:1023B00006010050A000709090700406060601000F
:1023C00050007090907004070706010020502070A4
:1023D00090907005040406000070A8B0780406060A
:1023E0000601FE708080702040040707060100404F
:1023F000200060B0C07004070706010020400060A4
:10240000B0C07004070706010020500060B0C07023
:10241000040606060100500060B0C07003070706FE
:102420000100804000C04040E00307070601002093
:102430004000C04040E003070706010040A000C084
:102440004040E0030606060100A000C04040E00452
:1024500007070601003060107090906004070706BF
:10246000010050A000E09090900407070601004092
:102470002000609090600407070601002040006083
:102480009090600407070601002050006090906063
:1024900004070706010050A0006090906004060643
:1024A00006010050006090906005050506000020C0
:1024B00000F8002004040406010070B0D0E0040716
:1024C0000706010040200090909070040707060165
:1024D00000204000909090700407070601002050F3
:1024E00000909090700406060601005000909090B5
:1024F000700409090601FE204000909090709060E1
:102500000408080601FE8080E09090E080800408C6
:10251000080601FE500090909070906052657769B7
:1025200070696E670050726F62696E6720666169DC
:102530006C65640050726F62696E67206661696CD9
:1025400065640050524F4245204641494C20434C5F
:1025500045414E204E4F5A5A4C450A005265776904
:1025600070696E670A005265776970696E6700501E
:10257000726F62696E67206661696C656400507293
:102580006F62696E67206661696C65640050524FC6
:102590004245204641494C20434C45414E204E4F38
:1025A0005A5A4C450A005265776970696E670A008D
:1025B00050726F62696E67206661696C65640A00BB
:1025C00050726F62696E67206661696C6564002095
:1025D0005A3A200020593A200042656420583A2097
:1025E000000A0A426564204C6576656C20436F7270
:1025F00072656374696F6E204D61747269783A0018
:10260000202B000A436F7272656374656420426513
:1026100064204865696768742076732E204265647B
:1026200020546F706F6C6F67793A0A00202B000A94
:102630004265642048656967687420546F706F67ED
:1026400072617068793A0A2020202B2D2D2D2042AE
:1026500041434B202D2D2B0A2020207C20202020A0
:10266000202020202020207C0A204C207C2020209C
:1026700020282B29202020207C20520A2045207C45
:1026800020202020202020202020207C20490A20DB
:1026900046207C20282D29204E20282B29207C20F4
:1026A000470A2054207C2020202020202020202089
:1026B000207C20480A2020207C20202020282D2932
:1026C000202020207C20540A2020207C2020202034
:1026D000202020202020207C0A2020204F2D2D206B
:1026E00046524F4E54202D2D2B0A2028302C3029B5
:1026F0000A004D65616E206F662073616D706C65B8
:102700006420706F696E74733A200020643A200070
:1027100020623A200045716E20636F6566666963CA
:1027200069656E74733A20613A200052756E6E6965
:102730006E6720696E204452592D52554E206D6FA0
:1027400064650A00473239204175746F2042656420
:10275000204C6576656C696E670A002842296163C2
:102760006B00284629726F6E7400285229696768C9
:102770007400284C29656674003F4E756D62657261
:10278000206F662070726F626520706F696E74735F
:1027900020697320696D706C61757369626C652066
:1027A0002832206D696E696D756D292E0A003F28EB
:1027B00056296572626F7365206C6576656C206959
:1027C0007320696D706C61757369626C6520283067
:1027D0002D34292E0A0053442063617264206F6BEC
:1027E0000A006F70656E526F6F74206661696C6568
:1027F000640A00766F6C756D652E696E697420666B
:1028000061696C65640A00534420696E69742066CE
:1028100061696C0A0043616E6E6F7420656E746549
:1028200072207375626469723A2000022E2E004D88
:1028300061696E004D6F766520302E316D6D004DF3
:102840006F766520316D6D004D6F76652031306D8E
:102850006D004D6F766520617869730045787472FC
:1028600075646572004D6F7665205A004D6F766510
:102870002059004D6F7665205800746F2072657383
:10288000756D65005761697420666F72207072699A
:102890006E74005052494E542050415553454400E7
:1028A00045787472756465206D6F7265005265734A
:1028B000756D65207072696E7400524553554D45B3
:1028C000204F5054494F4E533A0020204E6F7A7A91
:1028D0006C653A20002000506C656173652077615B
:1028E00069742E2E2E0048656174696E67206E6FC4
:1028F0007A7A6C65005052494E54205041555345E8
:10290000440020204E6F7A7A6C653A2000200068DF
:10291000656174206E6F7A7A6C652E0050726573F3
:102920007320627574746F6E20746F005052494E3C
:1029300054205041555345440020204E6F7A7A6C04
:10294000653A2000200066696C616D656E742065D3
:10295000787472756465005761697420666F7200DF
:102960005052494E54205041555345440020204E6A
:102970006F7A7A6C653A2000200066696C616D653B
:102980006E74206C6F6164005761697420666F72A9
:10299000005052494E542050415553454400202088
:1029A0004E6F7A7A6C653A2000746F20636F6E7494
:1029B000696E75652E2E2E00616E642070726573CF
:1029C0007320627574746F6E00496E736572742043
:1029D00066696C616D656E74005052494E542050AA
:1029E000415553454400656E7175657565696E673F
:1029F0002022007C3C3E5E2B3D3F2F5B5D3B2C2A22
:102A0000225C0043616E6E6F74206F70656E207380
:102A10007562646972200001050800FF0601210249
:102A20003520FFFF07FF06FF090050221656808061
:102A300080800080153353A0A0A00257575050F853
:102A400050F850500257572070A07028702013354E
:102A50005580A040A02002475740A0A040A0A05011
:102A6000251353808080122656408080808040123B
:102A700026568040404040800245559060F060906E
:102A80000255552020F82020113353604080044126
:102A900051F011335340E040024656101020408060
:102AA0008012365640A0A0A0A04012365640C0402A
:102AB0004040E00246566090106080F0024656F0BA
:102AC00020601090600246562060A0F02020024650
:102AD00056F080E01090600246566080E090906072
:102AE000024656F01020204040024656609060900A
:102AF0009060024656609090701060122555C0C0DC
:102B000000C0C0113656606000604080123656200A
:102B10004080804020034353F000F012365680403E
:102B20002020408012365640A020400040015858D6
:102B3000304898A8A8904030024656609090F09097
:102B400090024656E090E09090E0024656609080F9
:102B5000809060024656E090909090E0024656F0D9
:102B600080E08080F0024656F080E080808002465F
:102B700056609080B090600246569090F090909091
:102B8000123656E040404040E00246567020202079
:102B9000A04002465690A0C0A0A090024656808059
:102BA000808080F002465690F0F090909002465659
:102BB00090D0F0B0B0900246566090909090600235
:102BC0004656E09090E08080014757609090D0B0EA
:102BD0006010024656E09090E09090024656609059
:102BE00040209060123656E0404040404002465639
:102BF0009090909090600246569090909060600205
:102C00004656909090F0F0900246569090606090FA
:102C100090025656888850202020024656F01020F8
:102C20004080F0123656E080808080E00246568078
:102C30008040201010123656E020202020E016326E
:102C40005240A0014151F01622528040024454707B
:102C50009090700246568080E09090E0123454606C
:102C6000808060024656101070909070024454604C
:102C7000B0C060024656205040E0404001455560DB
:102C8000907010600246568080E090909012365608
:102C90004000C04040E01137572000202020A040D5
:102CA000024656808090E09090123656C0404040D8
:102CB00040E0025454D0A8A8A8024454E090909058
:102CC00002445460909060014555E090E08080019E
:102CD00045557090701010024454A0D0808012347A
:102CE0005460C020C00246564040E040502002449C
:102CF0005490909070123454A0A0A0400254548874
:102D0000A8A850024454906060900145559090707E
:102D10009060024454F02040F0024757304020C0F9
:102D2000204030221656808080808080024757C025
:102D30002040304020C006425250A0FFFFFFFFFF5E
:102D4000FFFFFFFFFFFFFFFFFFFFFFFFFFFFFFFF93
:102D5000FFFFFFFFFFFFFFFFFFFFFFFF0900502204
:102D600016568000808080800146562070A0A0709A
:102D7000200246562050E04050A002555588705021
:102D800070880256568850F820F820221757808005
:102D900080008080800247577080E0907010E017BC
:102DA0003151A002565670A8C8C8A8701435556095
:102DB000A06000E003435350A050123353E02020A2
:102DC000143151E002565670E8D8E8D870173151E6
:102DD000E015335340A04012355540E04000E01468
:102DE000355540A02040E0143555C020C020C01605
:102DF00022524080014555909090E08002565678CE
:102E0000E8E86828282411518011225240801435A6
:102E10005540C04040E014355540A04000E0034319
:102E200053A050A0024757808080A060F020024746
:102E3000578080A0D010207002475780408060A04B
:102E4000F02012365640004080A0400247574020F4
:102E50006090F0909002475720406090F090900270
:102E6000475760906090F0909002475750A0609054
:102E7000F0909002475790006090F0909002475772
:102E800060906090F0909002465670A0A0F0A0B0C4
:102E9000014757609080809060400247574020F083
:102EA00080E080F00247572040F080E080F0024749
:102EB000576090F080E080F00247579000F080E08B
:102EC00080F01237578040E0404040E012375720F2
:102ED00040E0404040E012375740A0E0404040E032
:102EE000123757A000E0404040E00256567048E8D4
:102EF00048487002475750A090D0B0909002475772
:102F000040206090909060024757204060909090E1
:102F1000600247576090609090906002475750A0C1
:102F2000609090906002475790006090909060127F
:102F30003353A040A002465670B0B0D0D0E0024754
:102F4000574020909090906002475720409090907A
:102F50009060024757609090909090600247579021
:102F600000909090906002575710208850202020A9
:102F700002465680E09090E0800246566090A0A005
:102F800090A0024757402000709090700247572051
:102F900040007090907002475720500070909070E1
:102FA00002475750A0007090907002465650007033
:102FB00090907002475760906070909070025454E7
:102FC000F068B07811355560808060400247574006
:102FD000200060B0C06002475720400060B0C06071
:102FE00002475760900060B0C060024656500060D3
:102FF000B0C060123757804000C04040E0123757E1
:10300000204000C04040E012375740A000C0404080
:10301000E0123656A000C04040E0024757A040A052
:103020001070906002475750A000E09090900247C7
:103030005740200060909060024757204000609009
:103040009060024757609000609090600247575030
:10305000A0006090906002465690006090906012D0
:1030600035554000E0004002445470B0D0E00247C3
:103070005740200090909070024757204000909059
:103080009070024757609000909090700246569062
:10309000009090907001485820400090907090608F
:1030A0000147578080E090E0808001475790009072
:1030B0009070906001050700FE0500FB01F220FF03
:1030C000FE05FE05FE02004002152580808000807E
:1030D000053242A0A002556550F850F850014656FE
:1030E0002070C030E0200255659010204048025505
:1030F00065608068906805122280800225354080D6
:103100008080400225358040404080043343A04009
:10311000A003334340E0400122324080043141E0CB
:10312000021121800255650810204080024555603B
:1031300090909060022535C040404040024555E0E7
:10314000106080F0024555E0106010E00245552007
:1031500060A0F020024555F080E010E00245556087
:1031600080E09060024555F01020404002455560D7
:10317000906090600245556090701060031323804A
:103180000080021424800080800235452040804069
:1031900020033343E000E0023545804020408002B8
:1031A0004555E0106000400255657088B8A870026F
:1031B0004555609090F090024555E090E090E00217
:1031C00035456080808060024555E0909090E00237
:1031D0003545E080E080E0023545E080E080800217
:1031E00045557080B090700245559090F0909002D7
:1031F0003545E0404040E0024555301010906002F7
:10320000455590A0C0A09002354580808080E002A6
:10321000556588D8A8888802455590D0B09090020E
:1032200045556090909060024555E09090E0800197
:103230004656609090906010024555E09090E09066
:1032400002455570806010E0023545E04040404046
:1032500002455590909090600245559090A0A040F6
:1032600002556588A8A8A850024555909060909096
:103270000245559090701060023545E0204080E096
:10328000022535C0808080C002556580402010082E
:10329000022535C0404040C005324240A0024151A5
:1032A000F0052232804002445470909070024555DF
:1032B00080E09090E00234446080806002455510C8
:1032C0007090907002445460B0C060023545204058
:1032D000E040400046567090907010600245558066
:1032E000E090909002152580008080800027374074
:1032F0000040404040800245558090A0E09002157B
:10330000258080808080025464F0A8A8A8024454DC
:10331000E090909002445460909060004656E09097
:1033200090E08080004656709090701010023444F7
:10333000A0C0808002445470C030E002354540E0B7
:10334000404020024454909090700244549090A0C9
:1033500040025464A8A85050023444A04040A00049
:103360004656909090701060024454F02040F00255
:103370003545604080406002152580808080800255
:103380003545C0402040C005425250A0FFFFFFFF1E
:10339000FFFFFFFFFFFFFFFFFFFFFFFFFFFFFFFF3D
:1033A000FFFFFFFFFFFFFFFFFFFFFFFFFF020040E8
:1033B000FFFFFFFFFFFFFFFFFFFFFFFFFFFFFFFF1D
:1033C000FFFFFFFFFFFFFFFFFFFFFFFFFFFFFFFF0D
:1033D000FFFFFFFFFFFFFFFFFFFFFFFFFFFFFFFFFD
:1033E000FFFFFFFFFFFFFFFFFFFFFFFFFFFFFFFFED
:1033F000FFFFFFFFFFFFFFFFFFFFFFFFFFFFFFFFDD
:10340000FFFFFFFFFFFFFFFFFFFFFFFFFFFFFF01CA
:10341000060D00FE09016602D620FFFE0BFE0AFE25
:103420000D00602219698080808080808000801873
:103430003363A0A0A00357675050F850F8505002D3
:1034400059692078A0A0702828F02002596948A85E
:103450005010204050A89002586840A0A040A0986A
:103460009068281363808080113B6B2040408080EF
:10347000808080404020113B6B80404020202020F5
:103480002040408006556520A870A820045565207E
:1034900020F82020113363604080065161F8113319
:1034A0006340E040025969080810102040408080C5
:1034B00002596920508888888888502002596920DC
:1034C00060A02020202020F8025969708888081008
:1034D000204080F8025969F80810207008088870A8
:1034E000025969101030505090F81010025969F8C4
:1034F0008080B0C80808887002596970888080F0A0
:1035000088888870025969F80810102020404040CF
:103510000259697088888870888888700259697033
:10352000888888780808887011386840E040000072
:1035300040E04011386840E040000060408002599F
:1035400069081020408040201008045464F80000EE
:10355000F802596980402010081020408002596903
:103560007088880810202000200259697088889887
:10357000A8A8B080780259692050888888F888887F
:1035800088025969F048484870484848F00259692B
:10359000708880808080808870025969F04848482F
:1035A00048484848F0025969F8808080F08080805F
:1035B000F8025969F8808080F08080808002596923
:1035C0007088808080988888700259698888888887
:1035D000F888888888123969E0404040404040407F
:1035E000E0025969381010101010109060025969EB
:1035F000888890A0C0A090888802596980808080C7
:1036000080808080F80259698888D8A8A88888882E
:103610008802596988C8C8A8A898988888025969F2
:10362000708888888888888870025969F0888888B6
:10363000F080808080015A6A70888888888888A88D
:103640007008025969F0888888F0A090888802592B
:1036500069708880807008088870025969F8202095
:10366000202020202020025969888888888888881E
:1036700088700259698888888850505020200259E3
:103680006988888888A8A8A8A8500259698888509D
:103690005020505088880259698888505020202036
:1036A0002020025969F808101020404080F8113B92
:1036B0006BE0808080808080808080E0025969801B
:1036C0008040402010100808113B6BE02020202093
:1036D0002020202020E0085363205088015161F809
:1036E0002A226280400256667008788898680259DB
:1036F00069808080F088888888F0025666708880AB
:103700008088700259690808087888888888780253
:1037100056667088F880887002596930484040F0D9
:103720004040404000586870888888780888700257
:103730005969808080B0C8888888881238684000BD
:10374000C040404040E0004A6A10003010101010A5
:1037500090906002596980808090A0C0A0908812EB
:103760003969C040404040404040E0025666D0A821
:10377000A8A8A888025666B0C888888888025666B5
:10378000708888888870005868F0888888F0808001
:10379000800058687888888878080808025666B0DB
:1037A000C8808080800256667088601088700258D9
:1037B000684040F04040404830025666888888881B
:1037C0009868025666888888505020025666888815
:1037D000A8A8A85002566688502020508800586833
:1037E0008888889868088870025666F8102040809B
:1037F000F8015B6B1820202020C0202020201822F8
:103800001969808080808080808080015B6BC0200F
:103810002020201820202020C008536348A890FFB3
:10382000FFFFFFFFFFFFFFFFFFFFFFFFFFFFFFFFA8
:10383000FFFFFFFFFFFFFFFFFFFFFFFFFFFFFFFF98
:103840000D00602219698000808080808080800364
:1038500058682070A8A0A0A870200259693048407C
:1038600040E0404048B0035666887050507088026F
:10387000596988885050F820F820202219698080E2
:1038800080800080808080124A6A60908060909082
:10389000601090601A3262A0A00359697088A8D89D
:1038A000C8D8A88870045767700878887800F8032B
:1038B00056662850A0A05028045363F80808163113
:1038C00061E00359697088E8D8D8E8D888700A514F
:1038D00061F8174464609090600357672020F820D7
:1038E0002000F807356540A02040E007356540A07E
:1038F0004020C02A226240800058688888888898C2
:10390000E8808002596978E8E8E8E86828282826ED
:103910002161C0202262408007356540C04040E000
:10392000045767708888887000F8035666A050288E
:103930002850A0025A6A40C04040E00818283808C1
:10394000025A6A40C04040E01028081038025A6A03
:1039500040A04020A04818283808025969200020BB
:10396000204080888870025A6A4020002050888851
:10397000F88888025A6A10200020508888F88888C1
:10398000025A6A30480020508888F88888025A6AAB
:1039900028500020508888F88888025A6A505000C1
:1039A00020508888F88888025A6A20502020508841
:1039B00088F8888802596958A0A0A0B0E0A0A0B8F3
:1039C000005B6B7088808080808088702040025A05
:1039D0006A402000F88080F08080F8025A6A102047
:1039E00000F88080F08080F8025A6A304800F88041
:1039F00080F08080F8025A6A505000F88080F08091
:103A000080F8123A6A804000E04040404040E012B6
:103A10003A6A204000E04040404040E0124A6A607C
:103A20009000E04040404040E0123A6AA0A000E030
:103A30004040404040E0025969F0484848E8484862
:103A400048F0025A6A2850008888C8A898888802D6
:103A50005A6A40200070888888888870025A6A10E4
:103A6000200070888888888870025A6A3048007000
:103A7000888888888870025A6A28500070888888E8
:103A8000888870025A6A50500070888888888870C8
:103A90000355658850205088015B6B08709898A882
:103AA000A8A8C8C87080025A6A4020008888888800
:103AB000888870025A6A10200088888888888870F0
:103AC000025A6A30480088888888888870025A6A52
:103AD00050500088888888888870025A6A102000B0
:103AE0008888502020202002596980F0888888F03A
:103AF000808080025969609090A0A0908888B00270
:103B00005969402000700878889868025969102027
:103B10000070087888986802596930480070087801
:103B20008898680259692850007008788898680257
:103B30005969505000700878889868025A6A30486D
:103B40003000700878889868025666702870A0A8BF
:103B50005000586870888080887020400259694001
:103B600020007088F88088700259691020007088E1
:103B7000F88088700259693048007088F880887031
:103B80000259695050007088F88088701239698035
:103B90004000C040404040E0123969204000C04031
:103BA000404040E0124969609000C040404040E021
:103BB000123969A0A000C040404040E0025A6A505B
:103BC000206010708888888870025969285000B079
:103BD000C888888888025969402000708888888849
:103BE00070025969102000708888888870025969AD
:103BF00030480070888888887002596928500070A1
:103C00008888888870025969505000708888888830
:103C100070035767202000F80020200158680870C2
:103C200098A8A8C8708002596940200088888888B0
:103C30009868025969102000888888889868025915
:103C4000693048008888888898680259695050000F
:103C5000888888889868005B6B102000888888981E
:103C600068088870005A6A8080B0C88888C8B080A8
:103C700080005B6B505000888888986808887000C6
:103C80000000000000000000000000000000000034
:103C90000000000000000000000000000000000024
:103CA00000000C000000000000000C0000000000FC
:103CB00000001200000000000000230000000000CF
:103CC000000021000000000000004C800000000007
:103CD00000005E8000000000000092400000000034
:103CE0000000A140000000000001212000000000B1
:103CF00000027F90000000000002001000000000A1
:103D00000007FFF8000000000004000800000000A9
:103D10000008000400000000000800060000000089
:103D2000001000020000000000301E010000000032
:103D300000207F81000000000041FFE080000000C3
:103D40000043FCF08000000000873B78400000004A
:103D5000018EDBFC60000000010FEBCC20000000B6
:103D6000021FEDB610000000021FDEB610000000BA
:103D70000439CD7F080000000436E0FF0800000091
:103D8000087EC0BB84000000187F005D8600000034
:103D9000107FC0ED82000000203CC07301000000D5
:103DA000203B337F01000000701BE77E0380000092
:103DB000C81DEEDE04C00000880FDEDC04400001F8
:103DC000240FDF3C092000012607DBF81920000240
:103DD0007203E7F0139000025101FFE0229000040B
:103DE00089007F802448000904801E004824000BBD
:103DF000FE400000DFF40010004000008002001FC1
:103E0000FFFFFFFFFFFE00000000000000000000B9
:103E10000000000000000000000000000000001092
:103E200022103C3C0E1F001022100422110400102E
:103E300022100822110400102210083C1104001066
:103E40002210102211040010221020221104001E42
:103E50001C1E3C3C0E04000000000000000000009E
:103E60000000000000000000000000000000000052
:103E70000000000000000000000000000000000042
:103E80000000000000000000000000000000000032
:103E90000000000000000000000000000000000022
:103EA0000000000000000000000000000000000012
:103EB000000000000000000000000000000A003BBD
:103EC00020454550524F4D20496E6465783A200098
:103ED0005570646174696E67207A6F666673657485
:103EE00020696E20454550524F4D3A20000600068D
:103EF0000006000600060006000600060006003F59
:103F0000C01F800F00060006000F001F803FC00684
:103F10000006000600060006000600060006000671
:103F20000007F8000C0C0010020020010060018066
:103F30004000804003E04001C0400080400000405D
:103F400000006000002000001000000C0C0007F8CA
:103F50000001FE0003030004008008004018006018
:103F60001000207C002038002010002000002000DD
:103F7000002000006000004000008003030001FEFC
:103F800000FFFFFF7F80FFC0FFC0FFC07F807F80FA
:103F9000FFC0FFC0FFC03F001E000C005A204F664C
:103FA00066736574004D6F76652058004D6F7665B9
:103FB0002059004D6F7665205A00457874727564FB
:103FC0006572000200002100240027002A002D0055
:103FD0003000330001010000040107010A01010261
:103FE000102020080810204010204080020102010B
:103FF00008040201010204081020408080402010C3
:10400000080402018004020180402010080402011B
:104010000804020101020408102040800102040883
:10402000102040800505050507050808080802025C
:1040300002020A0A08080404040401010101010142
:1040400001010303030303030303040707070C0C25
:104050000C0C0C0C0C0C02020202060606060606EC
:1040600006060B0B0B0B0B0B0B0B1FFFFFFFFFFFD2
:10407000FF600000000001FF400000000000FF8022
:1040800000000000007F83CF00000C303F87FF80DE
:10409000000C301F867980000C000F8C30C7838C99
:1040A00030E78C30CFC7CC31F38C30DCECEC33B95B
:1040B0008C30D86C6C33198C30D06C0C33198C303C
:1040C000D86C0C33198C30DC6C0E3B198C30CF7CE7
:1040D000079F198C30C77C038F1940000000000037
:1040E00002600000000000061FFFFFFFFFFFF82036
:1040F00020506C616E6E65724275666665724279BB
:104100007465733A20002046726565204D656D6FB9
:1041100072793A2000436F6D70696C65643A20448F
:10412000656320313520323031370A00207C204150
:104130007574686F723A2028416C657068204F6210
:104140006A6563747320496E632E2C204C756C7AFB
:10415000426F7420476974205265706F7369746F81
:104160007279290A004465632031352032303137B5
:1041700031353A32323A323400204C617374205572
:104180007064617465643A2000312E312E350A0066
:104190004D61726C696E0020536F66747761726551
:1041A0002052657365740A00205761746368646FF8
:1041B000672052657365740A002042726F776E2023
:1041C0006F75742052657365740A002045787465B4
:1041D000726E616C2052657365740A00506F77656A
:1041E0007255700A0073746172740A006572726F9E
:1041F000722077726974696E6720746F2066696CCB
:10420000650A004572726F723A00456E6473746F8E
:1042100070732025632025632025632025630020FB
:10422000503A00205A3A0020593A0020583A006586
:104230006E6473746F7073206869743A20006563EC
:10424000686F3A00446F6E6520736176696E67200F
:1042500066696C652E0A004D323900004D3234001B
:104260005072696E7420706175736564004D3132EF
:1042700035004D363030204230004D3234004D3262
:1042800033202573006175746F25692E67004578AA
:10429000747275646572004D6F7665205A004D6FBB
:1042A00076652059004D6F76652058004D6F766514
:1042B0006D656E74004D6F7665206178697300449A
:1042C000697361626C6520737465707065727300E8
:1042D0004D383400426564204C6576656C696E67C4
:1042E000004732382058590A4D3130392053313780
:1042F000350A473238205A0A4D313039205231348C
:10430000350A4731320A4732390A4D3130342053A9
:1043100030004175746F20686F6D6500473238005A
:104320004D61696E00290A002062797465733B2033
:10433000637263200053657474696E6773205374ED
:104340006F72656420280020496E76616C69642074
:1043500065787472756465722000205A3A0020599D
:104360003A0020436F756E7420583A0020453A0099
:10437000205A3A0020593A00583A00205A00205951
:1043800000580020204D61783A2000205A00205922
:1043900000580020204D696E3A20004F6E20004FDB
:1043A000666600536F667420656E6473746F707315
:1043B0003A200053657474696E67205472617665A3
:1043C0006C20416363656C65726174696F6E3A203D
:1043D0000053657474696E6720526574726163740A
:1043E00020416363656C65726174696F6E3A200089
:1043F00053657474696E67205072696E74204163EE
:1044000063656C65726174696F6E3A200053657400
:1044100074696E67205072696E7420616E642054F6
:10442000726176656C20416363656C657261746965
:104430006F6E3A200020643A0020693A0020703AFA
:104440000020643A0020693A0020703A004B494C41
:104450004C45442E200024F4D43050C38E20C2A2F8
:104460004017828B7011127A910D816CD90AA86164
:10447000E108C7586607615143061E4B5D05C145FB
:10448000A7041A411104093D9803713931034036DC
:10449000DB0265339102D4305402802E1D02632C5E
:1044A000EE01752AC501B028A001102781018F25D2
:1044B00064012B244B01E0223401AC211F018D202B
:1044C0000D01801FFC00841EED00971DDF00B81C4D
:1044D000D200E61BC600201BBC00641AB200B21951
:1044E000A8000A19A0006A189900D1179100401776
:1044F0008B00B516840031167E00B31579003A158D
:104500007300C7146F0058146A00EE136600881316
:10451000630025135E00C7125B006C125700151272
:104520005400C111510070114F0021114B00D610E1
:1045300049008D1047004610440002104200C00F91
:104540004000800F3E00420F3C00060F3B00CB0EA8
:104550003800930E37005C0E3500270E3400F30D43
:104560003200C10D3100900D3000600D2E00320D73
:104570002D00050D2C00D90C2B00AE0C2900850C4C
:1045800029005C0C2700350C27000E0C2600E80BD8
:104590002400C40B2400A00B23007D0B23005A0B26
:1045A0002100390B2100180B2000F80A1F00D90A3E
:1045B0001E00BB0A1E009D0A1D00800A1D00630A22
:1045C0001C00470A1B002C0A1B00110A1A00F709DD
:1045D0001A00DD091900C4091900AB091900920974
:1045E00017007B091800630917004C0916003609EB
:1045F0001600200916000A091500F5081500E00844
:104600001400CC081400B8081400A4081400900882
:1046100013007D0812006B081300580812004608AA
:1046200012003408110023081100120811000108BB
:104630001100F0071000E0071000D0071000C007BD
:104640001000B0070F00A107100091070E008307AC
:104650000F0074070F0065070E0057070E0049078B
:104660000E003B070D002E070E0020070D0013075C
:104670000D0006070D00F9060C00ED060D00E00622
:104680000C00D4060C00C8060C00BC060C00B006DA
:104690000C00A4060B0099060C008D060B00820688
:1046A0000B0077060B006C060B0061060A0057062C
:1046B0000B004C060A0042060A0038060A002E06C5
:1046C0000A0024060A001A060A0010060900070656
:1046D0000A00FD050900F4050900EB050900E205E3
:1046E0000900D9050900D0050900C7050900BE0564
:1046F0000900B5050800AD050800A50509009C05E1
:104700000800940508008C050800840508007C0555
:104710000800740508006C050700650508005D05C4
:104720000700560508004E0507004705070040052D
:10473000080038050700310507002A050700230592
:1047400007001C050600160507000F0507000805F1
:10475000060002050700FB040600F5040700EE044E
:104760000600E8040600E2040700DB040600D504A6
:104770000600CF040600C9040600C3040600BD04F9
:104780000600B7040600B1040500AC040600A60448
:104790000600A00405009B04060095040500900493
:1047A00006008A04050085040500800406007A04DA
:1047B000050075040500700405006B04050066041F
:1047C0000500610405005C0405005704050052045F
:1047D00005004D04050048040500430405003E049F
:1047E00004003A04050035040500300404002C04DC
:1047F000050027040400230405001E0404001A0415
:10480000040016040500110404000D04040009044A
:1048100005000404040000040400FC030400F80381
:104820000400F4030400F0030400EC030400E803B4
:104830000400E4030400E0030400DC030400D803E4
:104840000400D4030400D0030400CC030400C80314
:104850000300C503030024F404D9201BC40C5C0E20
:104860009804C4095F0265077101F405F900FB04AF
:10487000B30048048700C1036900580355000303CF
:104880004500BE023A008402310053022A00290288
:10489000250004022000E4011C00C8011900AF013A
:1048A00017009801140084011300710110006101C8
:1048B000100051010E0043010D0036010B002B01C9
:1048C0000B0020010B00150109000C010900030178
:1048D0000800FB000800F3000800EB000700E400FC
:1048E0000600DE000600D8000600D2000600CC005C
:1048F0000500C7000500C2000500BD000400B900A6
:104900000400B5000400B1000400AD000400A900DB
:104910000400A5000300A20003009F0004009B0008
:10492000030098000300950002009300030090002C
:1049300003008D0002008B00030088000200860047
:10494000020084000300810002007F0002007D005D
:1049500002007B000200790002007700010076006F
:1049600002007400020072000100710002006F007A
:1049700002006D0001006C0002006A000100690085
:10498000020067000100660001006500010064008C
:1049900002006200010061000100600001005F0090
:1049A00002005D0001005C0001005B0001005A0094
:1049B0000100590001005800010057000100560095
:1049C0000100550001005400010053000000530095
:1049D00001005200010051000100500001004F0091
:1049E00001004E0000004E0001004D0001004C008F
:1049F00001004B0000004B0001004A00010049008B
:104A00000100480000004800010047000100460086
:104A10000000460001004500000045000100440080
:104A2000010043000000430001004200000042007A
:104A300001004100000041000100400001003F0072
:104A400000003F0001003E0000003E0001003D006C
:104A500000003D0001003C0000003C0000003C0064
:104A600001003B0000003B0001003A0000003A005A
:104A70000100390000003900010038000000380052
:104A80000000380001003700000037000100360048
:104A9000000036000000360001003500000035003F
:104AA0000000350001003400000034000000340034
:104AB0000100330000003300000033000100320029
:104AC000000032000000320001003100000031001F
:104AD0000000310001003000000030000000300014
:104AE00001002F0000002F0000002F0000002F0009
:104AF00001002E0000002E0000002E0001002D00FD
:104B000000002D0000002D0000002D0001002C00F1
:104B100000002C0000002C0000002C0001002B00E5
:104B200000002B0000002B0000002B0001002A00D9
:104B300000002A0000002A0000002A0001002900CD
:104B400000002900000029000000290000002900C1
:104B500001002800000028000000280000002800B4
:104B600000002800010027000000270000002700A7
:104B7000000027000000270001002600000026009A
:104B8000000026000000260000002600010025008D
:104B90000000250000002500000025000000250081
:104BA0000000250001002400000024000000240073
:104BB0000000240000002400010023000000230066
:104BC0000000230000002300000023000000230059
:104BD000000023000100220000002200000022004B
:104BE000000022000000220000002200010021003D
:104BF0000000210000002100000021000000210031
:104C00000000210000002100010020000000200021
:104C10000000200000002000000020000000200014
:104C2000000020000000200001001F0000001F0005
:104C300000001F0000001F0000001F0000001F00F8
:104C400000001F0001001E0000001E0000001E00EA
:104C500000001E0000004D383420582059205A20F2
:104C600045004572723A204D494E54454D50204200
:104C70004544004D494E54454D5020747269676754
:104C800065726564004572723A204D494E54454D37
:104C900050204531004572723A204D494E54454DE1
:104CA00050204530004572723A204D415854454DD0
:104CB0005020424544004D415854454D5020747297
:104CC00069676765726564004572723A204D4158A4
:104CD00054454D50204531004572723A204D41589F
:104CE00054454D502045300020746F6F206C6F6E1E
:104CF0006720657874727573696F6E20707265765F
:104D0000656E7465640A0020636F6C642065787456
:104D1000727573696F6E2070726576656E74656406
:104D20000A00436172642072656D6F7665640043AA
:104D300061726420696E736572746564004D36300B
:104D40003020486F74656E6420746F6F20636F6CE1
:104D50006420746F206368616E67652066696C61AA
:104D60006D656E740A004B64200023646566696E8D
:104D700065202044454641554C545F004B69200056
:104D800023646566696E65202044454641554C5450
:104D90005F004B70200023646566696E65202044C7
:104DA000454641554C545F00504944204175746F4D
:104DB00074756E652066696E69736865642120503C
:104DC000757420746865206C617374204B702C209E
:104DD0004B6920616E64204B6420636F6E73746155
:104DE0006E74732066726F6D2062656C6F772069D8
:104DF0006E746F20436F6E66696775726174696F58
:104E00006E2E680A00504944204175746F74756EA7
:104E100065206661696C6564212074696D656F75D4
:104E2000740A00504944204175746F74756E652092
:104E30006661696C6564212054656D70657261748A
:104E400075726520746F6F20686967680A00204B6F
:104E5000643A2000204B693A2000204B703A200031
:104E60000A20436C617373696320504944200A002F
:104E70002054753A2000204B753A2000206D61784F
:104E80003A2000206D696E3A200020643A2000200C
:104E9000626961733A2000526573746F72652066AF
:104EA00061696C73616665004D3530320A4D35308D
:104EB00030004C6F61642073657474696E677300B1
:104EC00053746F72652073657474696E6773004103
:104ED0006476616E6365642053657474696E67738C
:104EE000004D61696E005072696E742061626F726C
:104EF0007465640041626F7574204669726D7761F4
:104F00007265004E6F2053442063617264005072DA
:104F1000696E742066726F6D2053440053746F7015
:104F2000207072696E7400526573756D65207072C1
:104F3000696E74005061757365207072696E7400DB
:104F40004368616E67652066696C616D656E7400AB
:104F5000436F6E66696775726174696F6E00546540
:104F60006D7065726174757265004D6F76656D6503
:104F70006E740054756E6500496E666F20736372BF
:104F800065656E00202F002042403A0020403A0024
:104F90004E6F204C696E65204E756D62657220778C
:104FA00069746820636865636B73756D2C204C6150
:104FB0007374204C696E653A200053544F5050452D
:104FC000442E20005072696E7465722073746F7085
:104FD0007065642064756520746F206572726F72ED
:104FE000732E2046697820746865206572726F722E
:104FF00020616E6420757365204D39393920746FD6
:1050000020726573746172742E202854656D70650A
:105010007261747572652069732072657365742E90
:10502000205365742069742061667465722072650E
:105030007374617274696E67290A004E6F20436849
:1050400065636B73756D2077697468206C696E6534
:10505000206E756D6265722C204C617374204C69F2
:105060006E653A2000636865636B73756D206D69CA
:10507000736D617463682C204C617374204C696E8D
:10508000653A20004C696E65204E756D6265722030
:105090006973206E6F74204C617374204C696E6567
:1050A000204E756D6265722B312C204C617374201B
:1050B0004C696E653A20004D313130004D3331007E
:1050C0004D383420582059205A204500534420722E
:1050D000656164206572726F720A00446F6E6520AC
:1050E0007072696E74696E672066696C650A004B40
:1050F000494C4C45442E20004B494C4C2063617573
:10510000736564206279204B494C4C20627574743D
:105110006F6E2F70696E0A004B494C4C45442E202F
:10512000004B494C4C2063617573656420627920A3
:10513000746F6F206D75636820696E616374697642
:10514000652074696D65202D2063757272656E74BB
:1051500020636F6D6D616E643A20004C756C7A420D
:105160006F742054415A2036204F66662E004F66D9
:1051700066004F6E2000456E6473746F702061622C
:105180006F72740053746570732F6D6D004A657291
:105190006B00416363656C65726174696F6E005684
:1051A000656C6F63697479005A204F666673657425
:1051B00000416476616E6365642053657474696E42
:1051C0006773005654726176206D696E0056547292
:1051D0006176206D696E005654726176206D696E3D
:1051E00000566D696E00566D696E00566D696E00F1
:1051F000566D6178204500566D6178204500566DEA
:105200006178204500566D6178205A00566D6178AE
:10521000205A00566D6178205A00566D61782059E9
:1052200000566D6178205900566D617820590056FE
:105230006D6178205800566D6178205800566D6178
:10524000782058004D6F74696F6E004573746570F7
:10525000732F6D6D004573746570732F6D6D005AFB
:1052600073746570732F6D6D005A73746570732F4E
:105270006D6D005973746570732F6D6D0059737483
:105280006570732F6D6D005873746570732F6D6D3D
:10529000005873746570732F6D6D004D6F74696F76
:1052A0006E0056652D6A65726B0056652D6A6572D3
:1052B0006B0056652D6A65726B00567A2D6A6572B1
:1052C0006B00567A2D6A65726B0056792D6A65728D
:1052D0006B0056792D6A65726B0056792D6A65727E
:1052E0006B0056782D6A65726B0056782D6A657270
:1052F0006B0056782D6A65726B004D6F74696F6E26
:10530000004F666673657473206170706C696564C4
:10531000004572723A20546F6F206661722100540A
:105320006F6F206661722066726F6D2072656665B0
:1053300072656E636520706F696E740A00486172F1
:1053400064636F6465642044656661756C742053A2
:10535000657474696E6773204C6F616465640A00DC
:10536000282300002823000064000000102700000C
:105370000000964300009643000040400000C841F2
:105380000000C9420000C9420000C84400804F44E8
:10539000202863616C63756C6174656429210A005F
:1053A00020213D2000454550524F4D20435243207F
:1053B0006D69736D61746368202D202873746F723A
:1053C0006564292000290A002062797465733B20F6
:1053D00063726320002073746F7265642073657458
:1053E00074696E677320726574726965766564208E
:1053F0002800204D61726C696E3D563430290A00D8
:1054000028454550524F4D3D00454550524F4D2087
:1054100076657273696F6E206D69736D6174636810
:105420002000000020002300260029002C002F006F
:105430003200000100000301060109010000A0C1C3
:105440000000A0C1000000000000914300809743CD
:10545000000087435A204F666673657400466C6F80
:105460007700466C6F770046616E207370656564E7
:1054700020310046616E2073706565642031004202
:10548000656400426564004E6F7A7A6C65004E6F09
:105490007A7A6C6500537065656400537065656465
:1054A000004D61696E00416D6178204500416D617C
:1054B00078204500416D6178205A00416D61782067
:1054C0005A00416D6178205900416D617820590082
:1054D000416D6178205800416D6178205800412D60
:1054E00074726176656C00412D74726176656C0032
:1054F000412D7265747261637400412D726574721E
:1055000061637400416363656C00416363656C00B3
:105510004D6F74696F6E000000A0C100809743005A
:105520000000005761726E696E673A20486F6D69BE
:105530006E672042756D702044697669736F7220C2
:105540003C20310A000202040000A0400000A040FC
:105550000000004000009B430080A14300008743FF
:1055600000004842000048420000404000000000A7
:10557000FF01FF5A2070726F6265206F75742E20D4
:105580006265640A005A2070726F6265206F7574DC
:105590002E2062656400486F6D6520585920666949
:1055A0007273740A00486F6D6520585920666972DD
:1055B000737400436F6F6C646F776E0046616E208A
:1055C000737065656420310046616E207370656597
:1055D0006420310042656400426564004E6F7A7A4F
:1055E0006C65004E6F7A7A6C65004D61696E004E95
:1055F000414E494E495459494E46CDCCCC3D0AD72F
:10560000233C17B7D13877CC2B329595E6241FB1C0
:105610004F0A000020410000C84200401C4620BC48
:10562000BE4CCA1B0E5AAEC59D74DA00F4CE1124CE
:105630001FBECFEFD1E2DEBFCDBF00E00CBF14E054
:10564000A0E0B2E0E8E1F3E402E00BBF02C00790A3
:105650000D92A831B107D9F725E1A8E1B4E001C066
:105660001D92A531B207E1F716E5CCE2D6E500E0E0
:1056700006C022970109FE010BBF0F940C21CA320C
:10568000D10780E00807A9F70E943AB00D947B216A
:105690000C9400002F923F924F925F926F927F92F4
:1056A0008F929F92AF92BF92CF92DF92EF92FF9232
:1056B0000F931F93CF93DF93CDB7DEB7C958D109AE
:1056C0000FB6F894DEBF0FBECDBF00912E0920E6C5
:1056D000029F800111240255184F8091800680FF9F
:1056E0001AC0EEE3F2E484917F013FEFE31AF30A7C
:1056F000811102C0780104C00E944159F701F3CF23
:10570000D7018D917D01882319F00E944159F8CF6E
:105710008AE00E94415910926A06109269068FE34E
:1057200080937F0610927E0610927D0610923204BE
:10573000109233041092340410923504F8018081E1
:105740000F5F1F4F8032D1F38E34B1F4818190ED21
:10575000980F9A3020F08D3211F08B3269F4329626
:10576000DF0131962C9120532A30D0F3CD01FC017A
:10577000019620812032D9F3F0937706E0937606E4
:105780007F01BFEFEB1AFB0A10816AE270E0C701EC
:105790000F944C21009739F0DC0111978C918032E5
:1057A000E1F311961C921D3429F0143519F01734C9
:1057B00009F0CAC0F7014E2F9F2F81918032D9F393
:1057C00080538A3008F0C0C010937F0620917D0678
:1057D00030917E06E42FF92F6AE0AF014F5F5F4FF3
:1057E000629FC001639F900D1124208130E02053FF
:1057F0003109820F931F218120532A3030F090937A
:105800007E0680937D069A0103C09C01FA01E5CFD4
:10581000D9012F5F3F4F4C914032D1F31D34D1F469
:105820008E31910591F03CF48731910571F08C3106
:10583000910581F40AC08537910564F08737910599
:1058400024F0803AE3E09E0729F4B0936A06A0931F
:1058500069067AC010926A0610926906D0907606A0
:1058600041E050E0FD0131962C91222309F46CC0F7
:105870002132A1F41D3491F48032910579F4F09332
:105880006A06E093690663E270E0CF010F944C2151
:10589000009709F459C0DC011C9256C00FEB020FAF
:1058A0000A31A0F59F01F90160812F5F3F4F6032FF
:1058B000D1F320ED260F2A3040F023ED260F2230C1
:1058C00020F06B3211F00C9455419F01602F70E075
:1058D000DB01B595A795B595A795B595A795AE5C50
:1058E000BB4F07707A01002E01C0EE0C0A94EAF754
:1058F000FC90FE28FC922115310511F02D1901C0F4
:1059000020E0DB01A85EBB4F2C930AC02091690602
:1059100030916A06232B21F4B0936A06A09369069E
:10592000208121542A3110F4DF019CCFDF01319610
:105930006C9160536A30D0F39D01F9012F5F3F4FA6
:1059400060816032D1F3F0CF80917F068D3411F405
:105950000C948735843511F40C94F840873411F099
:105960000C94384180917D0690917E068A31910594
:1059700009F47CC7A4F48430910544F48230910585
:105980000CF01FC197FF2BC00C945241843091053D
:1059900009F4E5C60C9709F427C70C9452418E31DF
:1059A000910511F40C94D5343CF48C31910509F433
:1059B000E6C70CF462C7E8C78B35910511F40C9467
:1059C0007E358C35910511F40C9483358A3591051B
:1059D00011F00C94524110927C060C94524180912B
:1059E0005702882311F40C9452410F94290887E33D
:1059F00094E00F94CA060F94280A8091800683FDD4
:105A00008FC0C0904304D0904404E0904504F090CF
:105A10004604209188073091890740918A07509168
:105A20008B07C701B6010F94E419882309F478C0E5
:105A300080913604811138C060910A0270910B0286
:105A4000882777FD8095982F0F94EA199B01AC0168
:105A50006091600670916106809162069091630684
:105A60000F94E41987FF20C0C0928807D09289075D
:105A7000E0928A07F0928B07EEE3F2E484918F01C3
:105A80000F5F1F4F882321F00E944159F801F6CF84
:105A9000EDE5F2E084918F010F5F1F4F882321F025
:105AA0000E944159F801F6CFC0904304D0904404BD
:105AB000E0904504F09046042091880730918907D2
:105AC00040918A0750918B07C701B6010F94161EAB
:105AD00020E030E048E453E40F943D20181604F52C
:105AE000C0928807D0928907E0928A07F0928B07CC
:105AF000EEE3F2E484918F010F5F1F4F882321F0C2
:105B00000E944159F801F6CFEEE3F2E084918F0153
:105B10000F5F1F4F882321F00E944159F801F6CFF3
:105B200020913704309138044091390450913A045F
:105B300060917C0770917D0780917E0790917F072F
:105B40000F94E41981111DC020913B0430913C0455
:105B500040913D0450913E0460918007709181070F
:105B600080918207909183070F94E419811109C0F5
:105B700060910C0270910D0280910E0290910F02C3
:105B80001AC06091A6027091A702882777FD8095C0
:105B9000982F0F94EA1920910C0230910D02409138
:105BA0000E0250910F020F94491A2AE037ED43E29A
:105BB0005CE30F94491A0E94FCDE0F9429070C94B1
:105BC000524120915702222311F40C94524111E0CA
:105BD000029709F010E00F94290882E50F9413084A
:105BE000882309F45CC10F9444066B017C0140904A
:105BF0007C0750907D0760907E0770907F07209112
:105C00008007309181074091820750918307639606
:105C10002CAF3DAF4EAF5FAF63978091370490914B
:105C20003804A0913904B0913A0467968CAF9DAFC7
:105C3000AEAFBFAF679720913B0430913C044091D9
:105C40003D0450913E046F962CAF3DAF4EAF5FAF19
:105C50006F9720E030E0A901C701B6010F94E41965
:105C6000882309F462C5A301920167966CAD7DADEE
:105C70008EAD9FAD67970F94E419811111C06396A3
:105C80002CAD3DAD4EAD5FAD63976F966CAD7DAD08
:105C90008EAD9FAD6F970F94E419882309F445C525
:105CA00020E030E0A901C701B6010F94E419881F74
:105CB0008827881F181759F080E090E0A0E8BFEB14
:105CC000AB968CAF9DAFAEAFBFAFAB970AC020E035
:105CD00030E040E85FE3AB962CAF3DAF4EAF5FAF37
:105CE000AB97A301920167966CAD7DAD8EAD9FAD74
:105CF00067970F94161EA3966CAF7DAF8EAF9FAFC4
:105D0000A39763962CAD3DAD4EAD5FAD63976F9697
:105D10006CAD7DAD8EAD9FAD6F970F94161EA7969F
:105D20006CAF7DAF8EAF9FAFA797A3962CAD3DAD67
:105D30004EAD5FADA397CA01B9010F94491A4B014B
:105D40005C01A7962CAD3DAD4EAD5FADA797CA01E6
:105D5000B9010F94491A9B01AC01C501B4010F941C
:105D6000171E0F9482206B966CAF7DAF8EAF9FAFE6
:105D70006B9720E030E040E05FE30F94491A4B015D
:105D80005C01A7019601C701B6010F94491A6B0186
:105D90007C01A5019401C501B4010F94491A9B012E
:105DA000AC01C701B6010F94161E0F9482209B010F
:105DB000AC01AB966CAD7DAD8EAD9FADAB970F9446
:105DC000491A4B015C0167962CAD3DAD4EAD5FAD00
:105DD0006797C301B2010F94171E20E030E040E046
:105DE0005FE30F94491A6B017C01A7966CAD7DAD02
:105DF0008EAD9FADA79790586B962CAD3DAD4EAD37
:105E00005FAD6B970F94F31E9B01AC01C501B4010C
:105E10000F94491A9B01AC01C701B6010F94171EDC
:105E2000A30192010F94161E6B017C016F962CAD9D
:105E30003DAD4EAD5FAD6F9763966CAD7DAD8EADF4
:105E40009FAD63970F94171E20E030E040E05FE3C2
:105E50000F94491A2B013C016B962CAD3DAD4EAD14
:105E60005FAD6B97A3966CAD7DAD8EAD9FADA397E7
:105E70000F94F31E9B01AC01C501B4010F94491AA4
:105E80009B01AC01C301B2010F94171E63962CADA8
:105E90003DAD4EAD5FAD63970F94161E14C089E4FF
:105EA0000F941308882329F00F9444066B017C019A
:105EB00003C0C12CD12C76018AE40F9413088823E7
:105EC000F9F00F9444066F966CAF7DAF8EAF9FAF25
:105ED0006F9720E030E0A901C701B6010F94E419E3
:105EE00081111EC020E030E0A9016F966CAD7DAD40
:105EF0008EAD9FAD6F970F94E419811111C015C439
:105F000020E030E0A901C701B6010F94E41988230D
:105F100009F40BC46F961CAE1DAE1EAE1FAE6F977C
:105F2000D701C601B05863968CAF9DAFAEAFBFAF7F
:105F300063976F962CAD3DAD4EAD5FAD6F975058EA
:105F400067962CAF3DAF4EAF5FAF67979C01AD0139
:105F5000BC01CD010F94491A4B015C0167962CAD31
:105F60003DAD4EAD5FAD6797CA01B9010F94491AB7
:105F70009B01AC01C501B4010F94171E0F94822040
:105F8000EB966CAF7DAF8EAF9FAFEB9780917C07A8
:105F900090917D07A0917E07B0917F07A3968CAF6B
:105FA0009DAFAEAFBFAFA397A7019601BC01CD01D6
:105FB0000F94171EAB966CAF7DAF8EAF9FAFAB97B4
:105FC000209180073091810740918207509183078B
:105FD000A7962CAF3DAF4EAF5FAFA7976F962CAD96
:105FE0003DAD4EAD5FAD6F97A7966CAD7DAD8EADFF
:105FF0009FADA7970F94171EAF966CAF7DAF8EAF76
:106000009FAFAF978091370490913804A0913904E5
:10601000B0913A04E3968CAF9DAFAEAFBFAFE397BC
:10602000AB962CAD3DAD4EAD5FADAB97BC01CD0198
:106030000F94161E6B017C0120913B0430913C04AF
:1060400040913D0450913E04E7962CAF3DAF4EAFDA
:106050005FAFE797AF962CAD3DAD4EAD5FADAF975F
:10606000E7966CAD7DAD8EAD9FADE7970F94161E94
:106070004B015C018091840790918507A091860770
:10608000B0918707C158DF4F88839983AA83BB8368
:10609000CF57D0409C01AD0160913F047091400406
:1060A00080914104909142040F94161E6B966CAF40
:1060B0007DAF8EAF9FAF6B97209188073091890796
:1060C00040918A0750918B07CD57DF4F2883398342
:1060D0004A835B83C358D040609143047091440469
:1060E00080914504909146040F94161EEF966CAF74
:1060F0007DAF8EAF9FAFEF97A701960163966CAD12
:106100007DAD8EAD9FAD63970F94491A2B013C0175
:10611000A501940167966CAD7DAD8EAD9FAD67977F
:106120000F94491A9B01AC01C301B2010F94171ED1
:106130002B013C01A501940163966CAD7DAD8EAD44
:106140009FAD63970F94491A4B015C01A70196011B
:1061500067966CAD7DAD8EAD9FAD67970F94491A74
:106160009B01AC01C501B4010F94161EA30192015D
:106170000F948A1E6B017C0120E030E0A9010F948E
:10618000E41987FF0AC02BED3FE049EC50E4C7015A
:10619000B6010F94171E6B017C01112351F02BEDFA
:1061A0003FE049EC50E4C701B6010F94161E6B01A5
:1061B0007C0120E030E0A901C701B6010F94E41989
:1061C000811128C0E3962CAD3DAD4EAD5FADE39798
:1061D000A3966CAD7DAD8EAD9FADA3970F94E419E2
:1061E000811118C0E7962CAD3DAD4EAD5FADE79780
:1061F000A7966CAD7DAD8EAD9FADA7970F94E419BA
:10620000811108C08BEDC82E8FE0D82E89ECE82EC6
:1062100080E4F82EEB962CAD3DAD4EAD5FADEB9727
:10622000C701B6010F94491A9B01AC010F94491A9A
:106230004B015C016B962CAD3DAD4EAD5FAD6B97E8
:10624000CA01B9010F94491A9B01AC01C501B401FF
:106250000F94171E0F9482204B015C012FE632E150
:1062600043E85AE30F94E41987FD5BC2C501B4010A
:106270000F948C1F0F94601F1B016115710519F499
:1062800022242394312CB10180E090E00F94E8198E
:106290004B015C019B01AC01C701B6010F94F31ED9
:1062A000A3966CAF7DAF8EAF9FAFA397A50194016E
:1062B0006B966CAD7DAD8EAD9FAD6B970F94F31E5D
:1062C000EB966CAF7DAF8EAF9FAFEB97A5019401BE
:1062D000EF966CAD7DAD8EAD9FADEF970F94F31E35
:1062E000EF966CAF7DAF8EAF9FAFEF97A3962CADBF
:1062F0003DAD4EAD5FADA397CA01B9010F94491AE8
:1063000020E030E040E05FE30F94491A9B01AC01CC
:1063100060E070E080E89FE30F94161EE3966CAF98
:106320007DAF8EAF9FAFE397C158DF4F88819981D2
:10633000AA81BB81CF57D04089879A87AB87BC871A
:10634000CD57DF4F288139814A815B81C358D040C6
:106350002D873E874F87588B6091A6027091A702C8
:10636000882777FD8095982F0F94EA1920910C02C9
:1063700030910D0240910E0250910F020F94491A74
:106380002AE037ED43E25CE30F94491AE7966CAFDD
:106390007DAF8EAF9FAFE7970F941C0ADC01CB0156
:1063A00088539F4FAF4FBF4F6B968CAF9DAFAEAF33
:1063B000BFAF6B9760964FAC609761965FAC61978B
:1063C00062966FAC629763967FAC6397A1E0B0E092
:1063D000A596BFAFAEAFA59719E1B12EA5962EAD8C
:1063E0003FADA5972215330508F057C10E942A6CCE
:1063F0000F941C0A6B962CAD3DAD4EAD5FAD6B9707
:10640000621B730B840B950B97FD11C00F941C0A34
:10641000DC01CB0188539F4FAF4FBF4F6B968CAFC2
:106420009DAFAEAFBFAF6B9780E00E9455F1BA94BD
:1064300009F44FC0E3962CAD3DAD4EAD5FADE39793
:1064400067966CAD7DAD8EAD9FAD67970F94491A81
:106450006B017C01A3962CAD3DAD4EAD5FADA39716
:10646000B201C3010F94491AA70196010F94171E98
:10647000162FA72E982E892EE3962CAD3DAD4EAD4E
:106480005FADE397B201C3010F94491A6B017C0120
:10649000A3962CAD3DAD4EAD5FADA39767966CADA9
:1064A0007DAD8EAD9FAD67970F94491A9B01AC01EE
:1064B000C701B6010F94161E2B013C01812F9A2DA6
:1064C000A92DB82D67968CAF9DAFAEAFBFAF6797C4
:1064D0005FC0A596AEADBFADA597BD0180E090E0D1
:1064E0000F94E819A3962CAD3DAD4EAD5FADA397CB
:1064F0000F94491A4B015C010F94F01E6B017C0153
:10650000C501B4010F9478204B015C01A7019601ED
:1065100063966CAD7DAD8EAD9FAD63970F94491AB8
:106520002B013C01A50194016F966CAD7DAD8EAD44
:106530009FAD6F970F94491A9B01AC01C301B20143
:106540000F94171E2B013C01A501940163966CADBD
:106550007DAD8EAD9FAD63970F94491A4B015C01E1
:10656000A70196016F966CAD7DAD8EAD9FAD6F9717
:106570000F94491A9B01AC01C501B4010F94161E7A
:1065800067966CAF7DAF8EAF9FAF6797B9E1BB2EBB
:106590009201A301AB966CAD7DAD8EAD9FADAB9777
:1065A0000F94171E69837A838B839C8367962CAD27
:1065B0003DAD4EAD5FAD6797AF966CAD7DAD8EAD29
:1065C0009FADAF970F94171E6D837E838F8398873F
:1065D000EB962CAD3DAD4EAD5FADEB9769857A8501
:1065E0008B859C850F94171E69877A878B879C877C
:1065F000EF962CAD3DAD4EAD5FADEF976D857E85D1
:106600008F8598890F94171E6D877E878F87988B4B
:10661000CE0101960F94CA06C090750689819A81B1
:10662000AB81BC8188A399A3AAA3BBA38D819E81C2
:10663000AF81B8858CA39DA3AEA3BFA389859A859E
:10664000AB85BC8588A799A7AAA7BBA7AE01485D63
:106650005F4FBE016C5D7F4FCE0180960E94D5A238
:10666000E796ECACFDAC0EAD1FADE7979E01235F46
:106670003F4FAE01485D5F4FBE016C5D7F4FCE0165
:1066800080960E943ECFA596EEADFFADA5973196C0
:10669000A596FFAFEEAFA597A1CEC09075068091ED
:1066A000370490913804A0913904B0913A0488A33A
:1066B00099A3AAA3BBA380913B0490913C04A09111
:1066C0003D04B0913E048CA39DA3AEA3BFA38091D3
:1066D0003F0490914004A0914104B091420488A7E6
:1066E00099A7AAA7BBA7AE01485D5F4FBE016C5D2D
:1066F0007F4FCE0180960E94D5A2E796ECACFDAC10
:106700000EAD1FADE79723E434E0AE01485D5F4F67
:10671000BE016C5D7F4FCE0180960E943ECF0F94EC
:1067200029070F94280A0C945241E3E0F2E4849183
:106730008F010F5F1F4F882321F00E944159F801FC
:10674000F6CFE8E7F2E084918F010F5F1F4F8823B7
:1067500011F40C9452410E944159F801F4CF80E5A4
:106760000F941308882329F00E94A25A4B015C0160
:1067700003C0812C912C540183E50F9413088823C6
:1067800061F00F94440620E030E04AE754E40F94AF
:10679000491A0F94601F4B015C010E947EFB80919F
:1067A0001002811105C060E08EE892E00E942CA4E6
:1067B0000F94280AC0905304D0905404E0905504DC
:1067C000F0905604C80CD91CEA1CFB1C0F941C0A40
:1067D0006C197D098E099F0997FD02C00C945241E6
:1067E00080E00E9455F1F2CF0E94AE7681110C94A8
:1067F000524180E50F941308882319F00F94340652
:1068000001C060E06FAF83E50F941308882319F08F
:106810000F94340601C06CE06BAF84E50F9413084D
:10682000882319F00F94340601C063E068A382E561
:106830000F941308882319F00F94440604C060E0F5
:1068400070E080ED90E469837A838B839C839E0162
:10685000205E3F4FAE014F5F5F4FBE01655C7F4FD3
:10686000CE01CF960E94A8E80C94524181E080931B
:106870005702109274060C9452410E94AE76811118
:106880000C94524180E50F941308882321F00F9453
:106890003406462F01C040E060918407709185075F
:1068A000809186079091870700E010E020E231ECAC
:1068B00009831A832B833C8300E010E822E933E448
:1068C0000D831E832F83388700E010E020EA31E437
:1068D00009871A872B873C8700E010E020EC3FE710
:1068E0000D871E872F87388B413071F1423021F59B
:1068F00018A219A21AA21BA220E030E040EA51E43B
:106900000F94171E7B018C0120E030E047E853E430
:106910000F943D20181624F4E12CF12C07E813E421
:10692000A701B8014BAF5CAF6DAF7EAFBE01605E3B
:106930007F4FCE01CB9611C020E030E040EA51E419
:106940000F94E41987FF0BC018A219A21AA21BA268
:10695000BE01605E7F4FCE0109960E94A1E818A299
:1069600019A21AA21BA2AE01405E5F4FBE016B5F6F
:106970007F4FCE0101960E949DE80C94524180E029
:106980000F9401110C94524181E080936F07249879
:106990002C9A0898109A0E948D7C10926F07249A66
:1069A0002C98089A10980C94524120E030E0A901EC
:1069B00060917C0770917D0780917E0790917F07A1
:1069C0000F94171E182F88E5C957DF4F6883C758E3
:1069D000D040C857DF4F7883C858D040C757DF4FE3
:1069E0009883C958D0400F941308C957DF4F688166
:1069F000C758D040C857DF4F7881C858D040C757D4
:106A0000DF4F9881C958D040882321F00F94440665
:106A10009B0102C09B01812FA901BC0148A359A37E
:106A20006AA37BA320E030E0A90160918007709108
:106A3000810780918207909183070F94171E5B0155
:106A40008C0189E50F941308882321F00F944406E4
:106A50005B018C01A501B80149835A836B837C8358
:106A600040904B0450904C0460904D0470904E0444
:106A700020914704309148044091490450914A04C0
:106A800068A179A18AA19BA10F94161E6B017C01BC
:106A90002CE032E040EA51EC0F943D2087FF02C029
:106AA0000C94524121E230E041E953E4C701B601C0
:106AB0000F94E419181614F40C945241A301920196
:106AC000B501C8010F94161E6B017C012CE032E069
:106AD00040EA51EC0F943D2087FF02C00C945241D4
:106AE00021E230E847E953E4C701B6010F94E41905
:106AF000181614F40C9452410C94664181E0809372
:106B00007C060C9452410E949AEB0C945241809165
:106B10007D0690917E068937910511F40C947D3E97
:106B20000CF0D5C08D34910509F4A1C50CF053C00B
:106B30008931910509F4E1C21CF58431910509F40C
:106B40005AC27CF48131910509F44AC22CF40297AF
:106B500008F4C3C10C945241429709F474C70C94D1
:106B600052418631910509F48DC20CF487C28731F8
:106B7000910509F48DC2489709F4A0C20C945241C2
:106B80008F31910509F47EC47CF48B31910509F4B1
:106B9000D0C20CF4C0C28C31910509F406C34E97E3
:106BA00009F407C30C9452418A32910509F40AC5CD
:106BB0002CF4809709F41EC40C9452418B34910537
:106BC00009F452C58C34910511F00C9452410E9485
:106BD00005780C9452418B36910509F4A2C6ACF5A8
:106BE0008535910509F460C7C4F48235910509F42F
:106BF00023C74CF48135910511F00C9452410E9449
:106C000066FB0C9452418335910509F418C784350D
:106C1000910509F418C70C9452418836910509F47E
:106C200029C54CF48C35910511F00C9452410F9408
:106C30000F030C9452418936910509F4E4C58A3654
:106C4000910509F44BC60C9452418337910509F420
:106C50002EC7D4F48E36910509F458C534F48D3618
:106C6000910509F411C60C9452418F36910509F42F
:106C70005EC58237910511F00C9452410E947EFB53
:106C80000E9493BF0C9452418637910509F412C7B4
:106C900074F48537910511F00C94524160E08091B5
:106CA000690690916A060E941CA40C945241873791
:106CB000910509F436C78837910511F00C945241BB
:106CC00081E080936E0780936D070C94524180336E
:106CD00031E0930711F40C94043F0CF078C08D3C24
:106CE000910511F40C948B3EACF58E3B910509F4A3
:106CF000E3C5ACF48C38910509F482C534F48D37C2
:106D0000910509F424C60C9452418139910509F486
:106D1000F9C78B39910509F490C50C945241893C0F
:106D2000910509F4F2C74CF4883C910511F00C94DC
:106D300052410E94FFC00C9452418B3C910509F4D2
:106D4000E7C78C3C910511F00C9452410E949EBE05
:106D50000C945241823E910509F4E6C7DCF4833D70
:106D6000910509F4DBC74CF48E3C910511F00C94AD
:106D700052410F9404050C9452418C3D910509F445
:106D8000D0C78D3D910511F00C9452410E944CC129
:106D90000C9452418D3251E0950711F40C94013F4F
:106DA0003CF48C32914011F40C94D83E0C94524136
:106DB0008E32E1E09E0711F40C94073F8F32914030
:106DC00011F00C9452410E9461DF0C945241853FB6
:106DD00021E0920711F40C94663F0CF045C0813914
:106DE00041E0940711F40C940A3FFCF48F35A1E0C4
:106DF0009A0711F40C947B404CF48E35914011F0BD
:106E00000C9452410E940D4F0C9452418336F1E094
:106E10009F0711F40C94CD408039914011F00C94EF
:106E200052410E947EFB0C945241843A31E0930718
:106E300009F4F4C754F48239914011F00C94524192
:106E400080E00E940BEB0C9452418C3AA1E09A072F
:106E500011F40C94633F843F914011F00C94524123
:106E60000E9484C10C9452418335E3E09E0711F4E3
:106E70000C94723FB4F4873F21E0920711F40C9414
:106E80006C3F14F40C94693F8C3142E0940711F488
:106E90000C946F3F8835924011F40C94753F0C941C
:106EA00052418C38A3E09A0711F40C9478404CF4CA
:106EB0008B38934011F00C9452410E942E5F0C9439
:106EC0005241803AF3E09F0709F4D0C2873E9340D5
:106ED00011F40C94E6400C94524100916906109113
:106EE0006A0680E50F941308882369F00E94A25A6D
:106EF0006B017C01BB24B39461157105810591057B
:106F000031F4B12C04C0B12CC12CD12C760183E515
:106F10000F9413088823F9F00F94440620E030E022
:106F20004AE754E40F94491A0F94601F6B017C01E7
:106F3000B11013C0611571058105910571F401153A
:106F4000110559F0D8018C91882339F061E0C8010E
:106F50000E941CA407C0BB2091F360E08DEC92E07E
:106F60000E942CA481E08093330A0E947EFB0F9440
:106F7000280AC114D104E104F104D1F08090530433
:106F800090905404A0905504B09056048C0C9D1C15
:106F9000AE1CBF1C0F941C0A681979098A099B0949
:106FA00097FF1AC08091330A81110C94BC4114C020
:106FB0008091330A882321F080E00E9455F1F8CFB8
:106FC00080915E1260E0882319F08EEB92E002C09F
:106FD00089EA92E00E942CA41092330A0C94524148
:106FE00060E080EE92E00E942CA417981698159805
:106FF00014980C945241E8EFF2E084918F010F5FF6
:107000001F4F882321F00E944159F801F6CF1092BA
:107010000A1540E050E0BA0186EB92E10E945D74EF
:107020008BE1E6EBF2E1DE01159601900D928A9577
:10703000E1F78091B4129091B5129C838B8380E22A
:1070400093E09A83898340E050E0BE016F5F7F4FF9
:107050008CEB93E00E9429AECE0101960E948591AF
:10706000E9EEF2E084918F010F5F1F4F882311F446
:107070000C9452410E944159F801F4CF0E9438907B
:107080000C94524110925E1210925F120C94524175
:10709000E0916906F0916A068081882329F08032A8
:1070A00009F410823196F8CF40E061E080916906E2
:1070B00090916A060E9448680C94524119821A8283
:1070C0001B821C8218A219A21AA21BA2809173060D
:1070D000882341F040E0BE016F5F7F4FCE01809674
:1070E0000E9415E480915F12882319F081E080935B
:1070F0005E120E948E770C94524110925E120E9492
:10710000057889E093E09093B80A8093B70A0E94CB
:1071100056BA0C94524180915F12882311F40C945A
:10712000524183E50F94130881110C94C1410C94D2
:10713000524180915F12882351F1EEE0F3E0849197
:107140008F010F5F1F4F882321F00E944159F801E2
:10715000F6CF609101157091021580910315909101
:1071600004154AE00E94914C8FE20E9441596091BF
:10717000FD147091FE148091FF14909100154AE067
:107180000E94914C8AE00E9441590C945241E0E2E5
:10719000F3E084918F010F5F1F4F882311F40C944B
:1071A00052410E944159F801F4CF0E9446BD0C940F
:1071B000524180915F12882311F40C94524180E572
:1071C00094E10E94238C80E594E10E942690109225
:1071D0005D1210925C12E0906906F0906A06809150
:1071E0005F12882311F40C9452410E942E901D824C
:1071F00018861C821B8280E293E09A83898382EB4B
:1072000092E19093D2128093D112F70180818F3254
:1072100009F06AC06FE270E0C7010F944C218C0145
:107220000F5F1F4F9E012F5F3F4F59010115110541
:1072300009F460C06FE270E0C8010F944C216C014A
:10724000009709F458C00817190708F054C04C01FA
:10725000801A910AA401B801CE0180960F946C2186
:10726000E0E2F0E0EC0FFD1FE80DF91D10828E0149
:10727000005E1F4FD8018D918D01882319F00E9467
:107280004159F8CF8AE00E9441596091D112709122
:10729000D2126115710519F06C5F7F4F02C060E07A
:1072A00070E021E0AE01405E5F4FCE0105960E9486
:1072B0002FAD811111C0BE01605E7F4F87E593E065
:1072C0000E94A29B8EE20E9441598AE00E9441598D
:1072D000C5010E948591E6C7B092D212A092D11248
:1072E00086010F5F1F4FA2CF83ED92E19093D212E0
:1072F0008093D11287016091D1127091D2126115E1
:10730000710519F06C5F7F4F02C060E070E018A259
:107310001BA222E0A801CE0180960E942FADF82E7C
:10732000882311F1CE0180960E94618CF82E88236B
:10733000D9F06CA57DA58EA59FA541E00E94D470D3
:10734000F82E882389F0E8A9B0E2EB9FF001112420
:10735000E95AFB4F309739F085EE80831BA20E94DB
:107360009670F82E01C0F12CCE0180960E9480917B
:10737000FF2011F1A1E3EA2EA3E0FA2EF701849198
:10738000882331F0FFEFEF1AFF0A0E944159F6CF30
:10739000D8018D918D01882319F00E944159F8CFB1
:1073A0008AE00E9441591092011510920215109224
:1073B00003151092041519C0FFE3EF2EF3E0FF2E22
:1073C000F7018491882331F0FFEFEF1AFF0A0E9442
:1073D0004159F6CFD8018D918D01882319F00E9473
:1073E0004159F8CF8EE20E944159CE0101960E9488
:1073F000859158C780915E1281110E947EFB009199
:10740000690610916A0680E50F94B207882321F07F
:107410000E942F5BF82E01C0F12C80915F1288230F
:1074200009F440C74F2D61E0C8010E94486883E518
:107430000F941308882381F00F943406AB01BC012C
:107440004093011550930215609303157093041532
:1074500080E594E10E945D7480915F12882319F0A9
:1074600081E080935E12F1101DC743CE80916906C2
:1074700090916A0621E020935D1240E060E00E9456
:10748000486810C70E945A77ECE3CE2ED12CE12C2D
:10749000F12CA70196010F94B91D162F072FCA01D1
:1074A000B901A70196010F94B91DD62EC72ECA01A6
:1074B000B90128E130E040E050E00F94B91DFB0134
:1074C000C9016DE671E00F94DF209B014D2D5C2D0D
:1074D000DE0111967D012115310599F00F931F935F
:1074E000CF92DF92FF93EF939F938F933F932F93CE
:1074F00083E993E09F938F93FF92AF930F947E194C
:1075000012C00097B1F00F931F93CF92DF92FF93B9
:10751000EF939F938F9383E893E09F938F93FF92D2
:10752000AF930F947E190FB6F894DEBF0FBECDBF98
:1075300030C0309779F00F931F93CF92DF92FF9373
:10754000EF9387E793E09F938F93FF92AF930F940E
:107550007E19E9CF452B69F00F931F93CF92DF92ED
:107560008FE693E09F938F93FF92AF930F947E19D2
:10757000DACF0F931F938BE693E09F938F93FF9245
:10758000AF930F947E190F900F900F900F900F9064
:107590000F9060E0C7010E941CA4EEE3F2E4849126
:1075A0008F010F5F1F4F882321F00E944159F8017E
:1075B000F6CFB70187EA93E00E94A29B8AE00E947F
:1075C000415970C683E50F941308882309F46AC6ED
:1075D0000E941B5BE82E80E50F941308811112C0F6
:1075E00081E0E11001C080E080936F07882329F0DB
:1075F00024982C9A0898109A55C6249A2C98089A80
:10760000109850C680E50F941308882331F00F942A
:10761000340677FD47C68B0102C00DE010E0802FD5
:10762000E4EBF3E09491891731F0319693E0EC3D6F
:10763000F907C1F7B7C6E3E0F2E484918F010F5F69
:107640001F4F882321F00E944159F801F6CFECED3D
:10765000F3E084918F010F5F1F4F882309F422C646
:107660000E944159F801F5CF0E948E771BC60E94F7
:10767000457718C688E690E00E94BFC0811112C607
:107680008091800683FD0EC683E50F94130888233E
:1076900009F408C60F9444060F945B1F7093F30F10
:1076A0006093F20F80E00E9411520F94440620E094
:1076B00030E040E752E40F94E41918163CF00E94C1
:1076C000457760E087EF93E00E942CA40F94440676
:1076D00020916006309161064091620650916306E8
:1076E0000F943D2018160CF0DDC58EED92E09F93AF
:1076F0008F938BEE93E09F938F931F920E949376CC
:107700000F900F900F900F900F90CCC58EE40F94B8
:107710001308882309F4C6C50F94340660935706EE
:10772000709358068093590690935A06BBC583E51B
:107730000F941308882321F00E941B5BC82E01C000
:10774000C12CC0928006EEE3F2E484918F010F5FBA
:107750001F4F882321F00E944159F801F6CFEAE13A
:10776000F4E084918F010F5F1F4F882321F00E9466
:107770004159F801F6CFCC2099F17CE0E72E74E076
:10778000F72E00E010E020E0D12CC601002E02C050
:10779000959587950A94E2F780FF17C099249394F2
:1077A000920E222319F08CE20E944159F701259193
:1077B0003491F90184915901FFEFAF1ABF0A882370
:1077C00029F00E9441599501F4CF922E0F5F1F4F6F
:1077D00022E0E20EF11C0530110571F0292DD5CF04
:1077E000E6E1F4E084918F010F5F1F4F882321F0C1
:1077F0000E944159F801F6CF8AE00E94415952C5D2
:107800000E949D924FC589E690E00E94BFC0811101
:107810000C943A45E1E2F4E084918F010F5F1F4F31
:10782000882321F00E944159F801F6CF0E94C9F047
:107830008AE00E9441590C943A4583E50F9413085D
:10784000882309F42FC50E941B5B80935F068D334C
:1078500018F08CE380935F060F941C0A6B017C0187
:1078600020915F0630E0A8EEB3E00F94071EC60E2D
:10787000D71EE81EF91EC0925B06D0925C06E0920D
:107880005D06F0925E060EC58DE690E00E94BFC0D8
:10789000811108C58091800683FD04C583E50F949E
:1078A000130860968FAF6097811199C582E50F9498
:1078B0001308811194C5F6C48091800683FDF2C43B
:1078C00083E50F9413086C968FAF6C9781112AC7CC
:1078D00082E50F941308811125C7E4C483E50F9452
:1078E0001308882339F00F9434068B016F3F71051C
:1078F00019F010F00FEF10E080E50F9413088823C3
:1079000031F00E941B5B823008F0CCC401C080E0E3
:10791000E82FF0E0EE0FFF1FE05AFE4E11830083C8
:10792000C1C480E50F941308882339F00F943406FE
:107930006230710508F0B6C402C060E070E0FB017F
:10794000EE0FFF1FE05AFE4E11821082ABC48CE492
:107950000F94B207882319F00F94440604C060E026
:1079600070E080E090EC27966CAF7DAF8EAF9FAF5C
:1079700027978AE50F941308882319F00F9444067B
:1079800003C060E070E0CB0120E030E040E251E471
:107990000F94171E23966CAF7DAF8EAF9FAF2397CA
:1079A00088E50F941308882319F00F94440603C048
:1079B00060E070E0CB0120E030E040E251E40F9461
:1079C000171E6BAF7CAF8DAF9EAF89E50F94130888
:1079D000882319F00F94440603C060E070E0CB01E7
:1079E00020E030E847E953E40F94171E20E030E030
:1079F00040E251E40F94161E68A379A38AA39BA3C7
:107A000019821A821B821C828091730681114AC4DA
:107A1000C12CE12C8E010F5F1F4F9E01205E3F4F56
:107A2000AE01455C5F4FBE01615C7F4FCE018D5B57
:107A30009F4F0E943DE536C410927B0633C481E01F
:107A400080937B062FC483E50F941308882399F055
:107A50000F94440620E030E04AE754E40F94491ABA
:107A60000F94601F609353027093540280935502E9
:107A70009093560217C488E50F94B2078111D7C7B7
:107A800089E50F94B2078111D2C78AE50F94B20736
:107A90008111CDC785E40F94B2078111C8C70E9438
:107AA0007EFB0F947B06FEC30F94FD07FBC30E9471
:107AB000F159F8C385E40F94B207882381F00E943E
:107AC0002F5B882361F0EEE3F2E484918F010F5F76
:107AD0001F4F882321F00E944159F801F6CF81E41D
:107AE0000F94B207882381F00E942F5B882361F0F6
:107AF000EDE8F4E084918F010F5F1F4F882321F0A0
:107B00000E944159F801F6CF0091690610916A066A
:107B1000D8018D918D01882309F46ECE0E944159C0
:107B2000F7CF81E080936F0724982C9A0898109AD9
:107B3000EBECF4E084918F010F5F1F4F882321F05D
:107B40000E944159F801F6CFE3ECF4E084918F01F3
:107B50000F5F1F4F882321F00E944159F801F6CF93
:107B60001E9B03C009EF12E002C004EF12E0F8010F
:107B700081918F01882319F00E944159F8CF8AE042
:107B80000E944159EBEBF4E084918F010F5F1F4F8E
:107B9000882321F00E944159F801F6CF029903C0D1
:107BA00009EF12E002C004EF12E0D8018D918D01BF
:107BB000882319F00E944159F8CF8AE00E94415968
:107BC000E3EBF4E084918F010F5F1F4F882321F0D6
:107BD0000E944159F801F6CF1D9B03C009EF12E046
:107BE00002C004EF12E0F80181918F01882319F09F
:107BF0000E944159F8CF8AE00E944159EBEAF4E033
:107C000084918F010F5F1F4F882321F00E944159FB
:107C1000F801F6CF019B03C009EF12E002C004EFA8
:107C200012E0D8018D918D01882319F00E944159ED
:107C3000F8CF8AE00E944159E3EAF4E084918F0191
:107C40000F5F1F4F882321F00E944159F801F6CFA2
:107C50001C9903C009EF12E002C004EF12E0F80122
:107C600081918F01882319F00E944159F8CF8AE051
:107C70000E944159EBE9F4E084918F010F5F1F4F9F
:107C8000882321F00E944159F801F6CF379B03C0A9
:107C900009EF12E002C004EF12E0D8018D918D01CE
:107CA000882319F00E944159F8CF8AE00E94415977
:107CB000E1E9F4E084918F010F5F1F4F882321F0E9
:107CC0000E944159F801F6CF009903C009EF12E074
:107CD00002C004EF12E0F80181918F01882319F0AE
:107CE0000E944159F8CF8AE00E94415910926F07D3
:107CF000249A2C98089A1098D5C210926E07109268
:107D00006D07D0C20E947E59CDC20E948458CAC25B
:107D10000F94E007C7C20E94B25AC4C20E9403BFB8
:107D2000C1C20F941F08BEC280E50F94B20788231A
:107D300009F4B8C20F943406F62E062F172F83E5E8
:107D40000F941308882321F00F9434066B0103C0AD
:107D5000CC24CA94DC2C96012F5F3F4F2330310591
:107D600008F0A0C217FD9EC20E947EFBFFEFCF1657
:107D7000DF0631F0CA94CD2871F000E010E00DC0AC
:107D80008F2D0F94BF0931E020E0892B09F030E0FE
:107D9000032F122F02C001E010E08F2D0F94BF09B6
:107DA0008017910709F47EC280E00E9455F1F5CF5B
:107DB00083E50F941308882319F00F94340602C04A
:107DC00064E071E079A368A380E50F941308882329
:107DD00039F00F943406693833E1730730F402C088
:107DE00068EE73E07A83698304C088E893E19A833C
:107DF0008983BE01605E7F4FCE0101960E94B96DFE
:107E000051C20E9488BD4EC20E9422BE4BC20E9437
:107E1000584F48C281E00E940BEB44C286E50F94A4
:107E2000B207882321F082E195E00E9452C083E5E9
:107E30000F94B207882321F00E942F5B182F01C0F6
:107E400010E083E50F94B207882319F0812F0E9478
:107E5000E491F0906B06111103C0EEE3F2E41AC056
:107E6000F110FBCFE3E0F2E484918F010F5F1F4F2D
:107E7000882321F00E944159F801F6CFE3EFF4E0A6
:107E800084918F010F5F1F4F882339F30E9441595E
:107E9000F801F6CF84918F010F5F1F4F882321F0E7
:107EA0000E944159F801F6CFFF2019F063E073E01A
:107EB00002C067E073E085EE94E00E94A29B8AE036
:107EC0000E944159EFC10F94F603ECC10E9427FEB6
:107ED000E9C10E94E1FCE6C10E944864E3C10E943E
:107EE0003E5BE0C10E94B75FDDC10E94AE76882391
:107EF00019F081E00F94011185E40F94B2078823F3
:107F000019F00F94440604C060E070E080E090EC4B
:107F10002F966CAF7DAF8EAF9FAF2F978AE50F94F2
:107F20001308882319F00F94440604C060E070E041
:107F300080E291E42B966CAF7DAF8EAF9FAF2B9715
:107F400088E50F941308882319F00F94440604C0A1
:107F500060E070E080E291E427966CAF7DAF8EAF79
:107F60009FAF279789E50F941308882319F00F9482
:107F7000440604C060E070E882E993E423966CAFA5
:107F80007DAF8EAF9FAF239785E50F94B20788230F
:107F900019F00F94440604C060E070E088EC92ECA5
:107FA0006BAF7CAF8DAF9EAF8CE40F94B20788238C
:107FB00019F00F94440603C060E070E0CB0168A3A1
:107FC00079A38AA39BA382E40F941308882321F04A
:107FD0000F943406F62E02C085E0F82ED0904F1292
:107FE0008091730681117EC0CC24C394EF2C8E0146
:107FF000055C1F4F9E01215C3F4FAE014D5B5F4F03
:10800000BE01695B7F4FCE01855B9F4F0E943DE5BE
:10801000882309F467C081E08093330A11E08091DE
:10802000330A882309F44AC060E08F2D0E942F6E26
:10803000809172068823F1F110936D0640E050E0C4
:10804000BA0183EB96E90E94EDA68091330A88235A
:1080500021F081E00E9455F1F8CF10926E06109247
:108060006F061092700610927106109272060E94AE
:1080700011520E9453F310936D0640E050E0BA0194
:1080800089E095E90E94EDA60F941C0A685370459B
:108090008F4F9F4F60936E0670936F0680937006AC
:1080A00090937106109272061093330A61E08F2D3F
:1080B0000E942F6E81E00E9455F1B1CF00E010E0E8
:1080C00028E432E409831A832B833C83809173066E
:1080D000882341F04F2DBE016F5F7F4FCE01809608
:1080E0000E9415E441E0D412DDC00E948E77DAC010
:1080F0000E94F25ED7C083E50F941308882309F429
:1081000049C00E941B5B813039F0823009F042C0C7
:1081100008E213E0F12C23C008E213E0F12CD801AF
:108120008D918D010F941308882339F00E941B5BF9
:108130004FEF682F8F2D0E944656F394B4E0FB1248
:10814000EECF82E40F941308882321F10E941B5B79
:108150004FEF682F1CC0F394F4E0FF1679F0F8019C
:1081600081918F010F9413088823A9F30E941B5B50
:10817000482F6FEF8F2D0E944656EDCF82E40F946B
:108180001308882339F00E941B5B482F6FEF84E0AF
:108190000E9446560E94614E85C0E3E0F2E484915D
:1081A0008F010F5F1F4F882321F00E944159F80172
:1081B000F6CFEFE2F5E084918F010F5F1F4F882328
:1081C00009F470C00E944159F801F5CF81E0809315
:1081D00057021092740683E50F94B207811103C011
:1081E0000E94F94D5FC00E942F5B81115BC0F8CFE8
:1081F000F0907D06FF2021F1EEE3F2E484918F01FF
:108200000F5F1F4F882321F00E944159F801F6CFDC
:1082100084E50E9441596F2D70E080E090E04AE0D3
:108220000E94914C80E20E9441590BE013E0D8017A
:108230008D918D01882309F4DFCA0E944159F7CF3F
:1082400010927506EEE3F2E484918F010F5F1F4FE9
:10825000882321F00E944159F801F6CF60E070E0D8
:108260008EE395E00E943F4F8AE00E9441591AC078
:10827000EEE3F2E484918F010F5F1F4F882321F01A
:108280000E944159F801F6CF609176067091770609
:1082900080E595E00E94A29B82E20E9441598AE01B
:1082A0000E9441590E94914DE5C320916906309189
:1082B0006A06232B39F49F012150310930936A0655
:1082C0002093690620E030E00C94662C80E00E9448
:1082D000E4910F944B0A83E50F94B207882309F4C5
:1082E00049C00E942F5B21E0482FBE016F5F7F4F86
:1082F000CE0180960E94B2786B017C019B01AC019B
:108300000F94C320811131C02CEA35EC47E257E3CA
:1083100068A179A18AA19BA10F94171EAB01BC0192
:1083200081EA92E00E944EBD2CEA35EC47E257E329
:1083300069817A818B819C810F94171EAB01BC01EE
:108340008CE992E00E944EBD2CEA35EC47E257E3FF
:10835000C701B6010F94171EAB01BC0187E992E07B
:108360000E944EBD8AE00E9441590F94320A0E9439
:1083700093BF98CF81E0B7CF80E00E9455F10C9475
:10838000CA370F943406AB01BC01409301155093DA
:108390000215609303157093041580E594E10E9423
:1083A0005D7480CF802F0E94AF4F6E2D802F0F9471
:1083B000E709F12CB701802F0E94CE4F063011053E
:1083C00029F4F0926311E09262116CCF083011052C
:1083D00009F068CFF0926111E092601163CF0F94C1
:1083E00044060F945B1F7093F30F6093F20F80E0CD
:1083F0000E9411520F94440620E030E040E752E41E
:108400000F94E419181644F00E94457760E080E567
:1084100094E00E942CA402C00E948E776091F20F1B
:108420007091F30F882777FD8095982F0F94EA19A4
:10843000209160063091610640916206509163067A
:108440000F943D2018160CF065C18EED92E09F93BD
:108450008F9384E494E09F938F931F920E9493766E
:108460000F900F900F900F900F9081E080938902F2
:1084700067961CAE1DAE1EAE1FAE67976B961CAE08
:108480001DAE1EAE1FAE6B9710E0A0961FAEA0975C
:108490003CE3A4963FAFA4974CE1A8964FAFA897B2
:1084A00056E4AC965FAFAC97D12CE12C60E8F62E89
:1084B0000FEB812C912C54016091F20F7091F30F0E
:1084C000882777FD8095982F0F94EA19762E672ECE
:1084D000582E492E262F372F482F592F6D2D7E2DA0
:1084E0008F2D902F0F94E4198823D9F020916006E6
:1084F000309161064091620650916306672D762D9A
:10850000852D942D0F94E419182F111F1127111F79
:1085100060968FAD6097882341F0112331F011E010
:10852000E7C07D2C6E2C5F2C402E0F941C0A6B0133
:108530007C01DC01CB016B962CAD3DAD4EAD5FAD4A
:108540006B97821B930BA40BB50BB7FD3BC0D701F8
:10855000C60188519C4FAF4FBF4F6B968CAF9DAFFC
:10856000AEAFBFAF6B970E94C9F0E0E4F4E0849136
:108570001F019FEF291A390A882321F00E944159CF
:10858000F101F5CF81149104A104B104A9F0C50152
:10859000B40168517C4F8F4F9F4F6C197D098E0934
:1085A0009F0928EE33E040E050E00F94B91DCA0166
:1085B000B9010E94024D03C08FE30E9441598AE035
:1085C0000E94415980E00E9455F10F94280AA09121
:1085D00060066C96AFAF6C97209061063090620693
:1085E000009163062A2F322D432D502F672D762DB3
:1085F000852D942D0F94161E9F7720E030E040E2E9
:1086000051E481149104A104B10429F40F94E419F4
:1086100087FD05C006C00F943D20181614F44601CE
:108620005701112309F44AC067962CAD3DAD4EADFC
:108630005FAD6797211531054105510541F0D7011F
:10864000C601821B930BA40BB50BB7FD37C06C960C
:108650002FAD6C97322D432D502FA0966FADA09764
:10866000A4967FADA497A8968FADA897AC969FAD22
:10867000AC970F94161E20E030E040EC5FE30F94BF
:10868000E41987FD4CCFD701C601805A9541AF4F01
:10869000BF4F67968CAF9DAFAEAFBFAF67976C967D
:1086A0009FAD6C97A0969FAFA097A4962FAEA4976E
:1086B000A8963FAEA897AC960FAFAC978091890271
:1086C0008823B1F081149104A104B10429F4D72CBA
:1086D000E62CF52C042DF0CEA8EECA1AA3E0DA0A97
:1086E000E108F108C818D908EA08FB08F7FCEFCF41
:1086F00080918902882309F4D5CD60E0112329F007
:1087000084E294E00E942CA4CDCD82E394E00E9408
:108710002CA4C8CD6096BFAD6097B111A6CE89EEEE
:1087200092E095CE0F9444060F945B1F6739710554
:1087300014F066E970E07093EF0F6093EE0F0E9403
:10874000C7510F94440620E030E040EA50E40F9413
:108750003D20181614F40E948E776091EE0F7091F0
:10876000EF0F882777FD8095982F0F94EA192091B5
:1087700064063091650640916606509167060F9435
:10878000E41960E087FF03C080E894E002C083E75B
:1087900094E00E942CA481E0809389028091750668
:1087A0008093680667961CAE1DAE1EAE1FAE67971F
:1087B0006B961CAE1DAE1EAE1FAE6B9760961FAEC5
:1087C0006097A0961FAEA097BCE3A496BFAFA497F6
:1087D000ECE1A896EFAFA897F6E4AC96FFAFAC97A4
:1087E000C12CD12C40E8E42E5FEBF52E812C912C8E
:1087F00054016091EE0F7091EF0F882777FD8095FF
:10880000982F0F94EA19162F072F782E692E262FEE
:10881000372F482F592FB601C7010F94E419882329
:1088200031F12091640630916506409166065091C1
:108830006706612F702F872D962D0F94E419881FDE
:108840008827881F60968FAF60976C962FAD6C97C6
:10885000222389F0882379F080918902882309F402
:1088600021CD60E085E694E00E942CA41BCD1C2D58
:108870000D2D7E2C6F2C0F941C0A6B017C01DC01EA
:10888000CB016B962CAD3DAD4EAD5FAD6B97821BB2
:10889000930BA40BB50BB7FD3BC0D701C6018851A4
:1088A0009C4FAF4FBF4F6B968CAF9DAFAEAFBFAF7E
:1088B0006B970E94C9F0EFE6F4E084912F019FEFDF
:1088C000491A590A882321F00E944159F201F5CF33
:1088D00081149104A104B104A9F0C501B401685147
:1088E0007C4F8F4F9F4F6C197D098E099F0928EE91
:1088F00033E040E050E00F94B91DCA01B9010E9475
:10890000024D03C08FE30E9441598AE00E94415901
:1089100080E00E9455F10F94280A20906406309060
:10892000650640906606509067069101A201612F8E
:10893000702F872D962D0F94161E9F7720E030E024
:1089400040EA50E481149104A104B10429F40F9485
:10895000E41987FD05C006C00F943D20181614F4D5
:10896000460157016096AFAD6097AA2309F443C052
:1089700067962CAD3DAD4EAD5FAD679721153105C6
:108980004105510541F0D701C601821B930BA40B91
:10899000B50BB7FD30C09101A201A0966FADA097B5
:1089A000A4967FADA497A8968FADA897AC969FADDF
:1089B000AC970F94161E20E030E040EC5FE30F947C
:1089C000E41987FD49CFD701C601805A9541AF4FC1
:1089D000BF4F67968CAF9DAFAEAFBFAF6797A09606
:1089E0002FAEA097A4963FAEA497A8964FAEA89797
:1089F000AC965FAEAC9780918902882309F42CCFA6
:108A000081149104A104B10429F4C12ED02EE72CC5
:108A1000F62CEFCE98EEC91A93E0D90AE108F108D6
:108A2000C818D908EA08FB08F7FE16CFEECF0E9457
:108A30007EFB88E50F94B207882319F0179A1092ED
:108A40006A0789E50F94B207882319F0169A1092E5
:108A50006B078AE50F94B207882319F0159A1092D4
:108A60006C0785E40F94B207882309F41BCC0F949C
:108A7000790618CCC757DF4F0FB6F894DEBF0FBE8C
:108A8000CDBFDF91CF911F910F91FF90EF90DF90BD
:108A9000CF90BF90AF909F908F907F906F905F909E
:108AA0004F903F902F9008950F93CF93DF93C82F4F
:108AB000D62F04E0262F41E3682F8DEA91E10F9431
:108AC000FE088823C9F02D2F41E36C2F8DEA91E138
:108AD0000E94D3B78C2F0E94B6928FEF8D0F8C0F10
:108AE0000E94B6922D2F44E36C2F8DEA91E1DF9125
:108AF000CF910F910C94D3B7DF91CF910F9108953F
:108B00007F928F929F92AF92BF92CF92DF92EF921D
:108B1000FF920F931F93CF93DF93CDB7DEB72A97C2
:108B20000FB6F894DEBF0FBECDBF10928D118091AD
:108B30008511882351F00E94E6AC40E050E0BA0174
:108B400089E29CEE0E94EDA6C9C44091A602509114
:108B5000A7028091891190918A11A0918B11B091F7
:108B60008C119A01280F391F4436510524F42536FB
:108B700031053CF41CC04436510551F02436310512
:108B8000B4F484E690E09093A7028093A60213C009
:108B90008B309105A105B1051CF02A50310907C0A1
:108BA000863F9F4FAF4FBF4F74F4265F3F4F3093C8
:108BB000A7022093A6021092891110928A11109296
:108BC0008B1110928C118091A6029091A7028A308D
:108BD00091053CF0883E23E092072CF087EE93E06D
:108BE00002C08AE090E09093A7028093A6020E94C0
:108BF00049A4782E0E947E6F8091E111853198F40E
:108C0000772049F08091601190916111892B19F0C2
:108C10000CEF11E102C00FED10E123E14FE061E044
:108C200089E00E9448928091E1118D3108F084C161
:108C3000883008F03FC080917206711002C0811127
:108C400039C06091F20F7091F30F882777FD8095FE
:108C5000982F0F94EA1920E030E040E05FE30F9492
:108C6000171E0F945B1F643671052CF46A30710572
:108C700024F04CE003C042E101C046E022E130E0D4
:108C8000241B310937FF02C02F5F3F4F35952795D1
:108C90003195219531092B5F2093E41127E0209332
:108CA000E511CB010E94739E0E94C76F8CED90E18D
:108CB0000E94BA6F8091E1118D31D0F58091E3115E
:108CC0008531B0F120E030E040E05FE36091600684
:108CD0007091610680916206909163060F94171E51
:108CE0000F945B1F9B01643671050CF0F4C22A30AF
:108CF00031050CF4EEC24CE022E130E0241B3109D6
:108D000037FF02C02F5F3F4F35952795319521954D
:108D100031092B5F2093E4112CE12093E511CB0165
:108D20000E94739E0E94C76F8CED90E10E94BA6F03
:108D30008091E111853140F58091E311813120F17D
:108D40006091F20F7091F30F882777FD8095982F2F
:108D50000F94EA19209160063091610640916206F5
:108D6000509163060F943D2018160CF0B6C2109275
:108D7000CD1102E022E041E16DE08DEA91E10E9437
:108D800053B881E08093CD118091E111883008F0D3
:108D90003FC080918406711002C0811139C060917A
:108DA000EE0F7091EF0F882777FD8095982F0F9425
:108DB000EA1920E030E040E05FE30F94171E0F94C3
:108DC0005B1F643671052CF46A30710524F04CE0A9
:108DD00003C042E101C046E022E130E0241B31093A
:108DE00037FF02C02F5F3F4F35952795319521956D
:108DF00031092F5A2093E41127E02093E511CB018C
:108E00000E94739E0E94C76F8CED90E10E94BA6F22
:108E10008091E1118D31D0F58091E3118531B0F170
:108E200020E030E040E05FE3609164067091650609
:108E300080916606909167060F94171E0F945B1F32
:108E40009B01643671050CF053C22A3031050CF4D5
:108E50004DC24CE022E130E0241B310937FF02C053
:108E60002F5F3F4F359527953195219531092F5A21
:108E70002093E4112CE12093E511CB010E94739E15
:108E80000E94C76F8CED90E10E94BA6F8091E11152
:108E9000853140F58091E311813120F16091EE0F31
:108EA0007091EF0F882777FD8095982F0F94EA191E
:108EB00020916406309165064091660650916706E0
:108EC0000F943D2018160CF015C21092CD1102E03F
:108ED00022E042E168E58DEA91E10E9453B881E029
:108EE0008093CD118091E1118C3130F58091E311A7
:108EF000843110F18091601190916111019644E6E6
:108F0000489F9001499F300D112437FF02C0215026
:108F10003F4F832F932F990F990B009769F028E605
:108F20002093E4112BE12093E5110E94739E0E948F
:108F3000C76F85E20E949D6F8091E111843328F410
:108F40008091E3118A3208F0DEC18091E11185330E
:108F500028F48091E311813308F0FAC180915E1208
:108F6000882309F44DC08091E111843308F048C092
:108F70008091E311823308F443C080915314882315
:108F800009F4EAC18091FD149091FE14A091FF14A0
:108F9000B09100150097A105B10509F4DDC1BC0130
:108FA000CD016D597F4F8F4F9F4F24E630E040E059
:108FB00050E00F94B91D60910115709102158091D8
:108FC0000315909104150F94B91D622F48E4649F16
:108FD000B0011124882777FD8095982F0F94EA1906
:108FE0002AE037ED43E25CE30F94491A0F94601FC7
:108FF000262F02E042E367E38DEA91E10E9453B835
:109000008091E111813308F05DC08091E3118932D4
:1090100008F458C00E945A776B017C018CE3882EBB
:10902000912CA12CB12CC701B601A50194010F947C
:10903000B91DCA01B901A50194010F94B91DCA0156
:10904000962E872E59018E010F5F1F4F41E8C416DF
:1090500041E5D40641E0E406F10408F47FC1B9011A
:1090600028E130E040E050E00F94B91D79018F9283
:109070009F92C50168E170E00F94DF209F938F936A
:109080003F932F932CE136E03F932F931F930F9341
:109090000F947E190FB6F894DEBF0FBECDBF9AE0D5
:1090A000E916F10408F489C198E0892F880F890F27
:1090B0008195855A8093E41180E38093E511C8017E
:1090C0000E94C76FE091A711F091A81184818111CE
:1090D000CCC060917C0770917D0780917E07909154
:1090E0007F070F945B1FCB010E940A9EBC018AE997
:1090F00096E00F94572160918007709181078091CD
:109100008207909183070F945B1FCB010E940A9EF8
:10911000BC0185E996E00F9457212CEA35EC47E233
:1091200057E360918407709185078091860790913D
:1091300087070F94171E20E030E048EC52E40F94AC
:10914000491A0F945B1F6B017C0197FD19C090E1D8
:10915000C91697E2D906E104F104E4F0C701B601AB
:1091600020E137E240E050E00F94DB1DCA01B90175
:109170002AE030E040E050E00F94DB1D605D0BC062
:10918000F094E094D094C094C11CD11CE11CF11C5B
:109190006DE201C060E26093860628EEC21623E00D
:1091A000D206E104F10494F0C701B60128EE33E0E1
:1091B00040E050E00F94DB1DCA01B9012AE030E025
:1091C00040E050E00F94DB1D605D01C060E2609301
:1091D0008706C701B60124E630E040E050E00F9476
:1091E000DB1D9AE0892E912CA12CB12CCA01B9016A
:1091F000A50194010F94DB1D605D60938806C70193
:10920000B601A50194010F94DB1D162F662381F092
:109210008EE280938906CA01B901A50194010F94D9
:10922000DB1D605D60938A06105D10938B0617C08E
:10923000CA01B901A50194010F94DB1D662339F021
:109240008EE280938906605D60938A0605C080E2A5
:1092500080938A068093890680E280938B0666E875
:1092600076E08EE896E00F9457218091E1118632E6
:10927000A8F48091E3118E3188F008E020E84EE1F7
:1092800060E08DEA91E10E9453B88091E11186324D
:1092900028F48091E3118F3108F091C08091E111A1
:1092A000823328F48091E3118C3208F0F8C0809169
:1092B000E1118F3308F012C18091E311883308F473
:1092C0000DC11092E4118EE38093E5110E941B7092
:1092D00005C146E011CD42E10FCD02E022E041E1BF
:1092E0006DE08DEA91E10E9453B84ECD46E0B2CDDB
:1092F00042E1B0CD02E022E042E168E58DEA91E191
:109300000E9453B8EFCD07E028E04AE26AE28DEA16
:1093100091E10E9453B805E022E04CE262E38DEA5D
:1093200091E10E9453B86AE08AE2BEDB6091AF111E
:109330007091B01182E38093C9118BE28093CA11BE
:1093400029EC31E142E38DEA91E10F942009FDCD52
:109350006AE486E3A9DB02CE60E038CE44E6A416D8
:10936000B104C0F48F929F92C50168E170E00F9440
:10937000DF209F938F9382E196E09F938F931F93BB
:109380000F930F947E190FB6F894DEBF0FBECDBFBA
:1093900095E08BCE8F929F923F932F938AE096E039
:1093A0009F938F931F930F930F947E190FB6F8948A
:1093B000DEBF0FBECDBF96E078CE97E076CE10929E
:1093C000CD1183E08093E41185E28093E51177204D
:1093D00029F08AED90E10E94BA6F0DC08091A3112F
:1093E000811102C08FE305C080916A078111F1CF1E
:1093F00080E20E949D6F8BE08093E41115E2109350
:10940000E5118AE996E00E94C76F8BE28093E41130
:109410001093E511772029F088ED90E10E94BA6F52
:109420000DC08091A411811102C08FE305C080910D
:109430006B078111F1CF80E20E949D6F83E38093DF
:10944000E41115E21093E51185E996E00E94C76FDB
:1094500083E58093E4111093E511772029F086EDE0
:1094600090E10E94BA6F0DC08091A511811102C0D8
:109470008FE305C080916C078111F1CF80E20E94DB
:109480009D6F8BE58093E41185E28093E5118EE872
:1094900096E00E94C76F81E08093CD11FFCE84E0FB
:1094A0000E94856F83E08093E41112E31093E5112D
:1094B00086E00E94A86F0E947E6F8CE08093E4118A
:1094C0001093E5118091A6029091A7020E94739ECD
:1094D0000E94C76F85E20E949D6FE9CE2A960FB663
:1094E000F894DEBF0FBECDBFDF91CF911F910F91DA
:1094F000FF90EF90DF90CF90BF90AF909F908F90B4
:109500007F9008951F93CF93DF9310928D118091D8
:10951000891190918A11A0918B11B0918C11813099
:109520009048A105B10540F01092891110928A115E
:1095300010928B1110928C11C0918911409182066A
:10954000141604F5842F992787FD909505972C2FE5
:10955000332727FD309528173907A4F045301CF034
:10956000CBEFC40F01C0C0E08C2F992787FD9095E9
:10957000A92FB92F8093891190938A11A0938B11F1
:10958000B0938C11C0938611D0E012E0C11109C0D4
:109590008091A8028823D9F121E041E067EC75E0D1
:1095A00020C0C13049F48091A802882381F120E0D5
:1095B00041E068EB75E015C0C23049F48091A80223
:1095C000882329F120E041E068EA75E00AC0C33051
:1095D00061F48091A8028823D1F020E041E061EAA3
:1095E00075E08D2F0E94A29412C0C43081F4809146
:1095F000A802882351F021E040E066E975E08D2F54
:109600000E94A2948D2F0E94D26F1093A802DF5F58
:10961000CF5FD53009F0BACFD0938206DF91CF91DA
:109620001F9108951F93CF93DF9310928D11809116
:10963000891190918A11A0918B11B0918C11813078
:109640009048A105B10540F01092891110928A113D
:1096500010928B1110928C11C0918911409181064A
:10966000141604F5842F992787FD909505972C2FC4
:10967000332727FD309528173907A4F045301CF013
:10968000CBEFC40F01C0C0E08C2F992787FD9095C8
:10969000A92FB92F8093891190938A11A0938B11D0
:1096A000B0938C11C0938611D0E012E0C11109C0B3
:1096B0008091A8028823D9F121E041E069E875E0B2
:1096C00020C0C13049F48091A802882381F120E0B4
:1096D00041E060E875E015C0C23049F48091A8020D
:1096E000882329F120E041E060E775E00AC0C3303B
:1096F00061F48091A8028823D1F020E041E06EE679
:1097000075E08D2F0E94A29412C0C43081F4809124
:10971000A802882351F021E040E063E675E08D2F38
:109720000E94A2948D2F0E94D26F1093A802DF5F37
:10973000CF5FD53009F0BACFD0938106DF91CF91BA
:109740001F9108950F931F93CF93DF9310928D1164
:109750008091891190918A11A0918B11B0918C11F7
:1097600081309048A105B10540F010928911109206
:109770008A1110928B1110928C11C0918911409115
:1097800083061416D4F4842F992787FD90950197AA
:109790002C2F332727FD30952817390774F0CFEF8A
:1097A000C40F8C2F90E0A0E0B0E0809389119093DB
:1097B0008A11A0938B11B0938C1110928711809114
:1097C0008611C81714F4C0938611809186119927C9
:1097D00087FD909504962C2F332727FD309582170F
:1097E000930724F48CEF8C0F8093861110918611CF
:1097F000D0E081E002E0111123C08823B9F01C16EB
:10980000ACF04091891150918A1160918B11709147
:109810008C114F5F5F4F6F4F7F4F40938911509373
:109820008A1160938B1170938C11CF5F8091A80285
:10983000882309F469C021E041E06BEF75E04EC078
:10984000113019F58823B9F0C230ACF44091891178
:1098500050918A1160918B1170918C114F5F5F4F05
:109860006F4F7F4F4093891150938A1160938B11F2
:1098700070938C11CF5F8091A802882309F444C0B3
:1098800020E040E066EE75E029C01230E9F48091F6
:109890008511811105C08091A8028823A9F109C012
:1098A000C230C9F70E944BA780918711882399F392
:1098B00033C081E0C23009F080E024E041EE55E0A1
:1098C0006D2F0E941FB920C0133061F48091A8024F
:1098D0008823D1F020E041E06FED75E08D2F0E94EC
:1098E000A29412C0143081F48091A802882351F010
:1098F00021E040E064ED75E08D2F0E94A2948D2F51
:109900000E94D26F0093A802DF5F1F5FD53011F075
:1099100080E071CFD0938306DF91CF911F910F919B
:109920000895AF92BF92CF92DF92EF92FF920F9382
:109930001F93CF93DF93CDB7DEB7A0970FB6F89400
:10994000DEBF0FBECDBF6115710581059105B1F177
:10995000B12CC42ED12CE12CF12CAA24A394AB0C55
:1099600001E010E00C0F1D1F0B0D111DB7FC1A9527
:10997000A70196010F94B91DF8016083B901CA01CE
:10998000611571058105910511F41B2D12C0BA2CCA
:10999000E4CFE1E0F0E0EC0FFD1FE10FF11D17FD5A
:1099A000FA9580818A3040F490E3890F0E944159F2
:1099B00011501F3F71F715C097E3F7CF80E3A096D2
:1099C0000FB6F894DEBF0FBECDBFDF91CF911F91D0
:1099D0000F91FF90EF90DF90CF90BF90AF900C94DD
:1099E0004159A0960FB6F894DEBF0FBECDBFDF91F0
:1099F000CF911F910F91FF90EF90DF90CF90BF908C
:109A0000AF900895CF92DF92EF92FF926B017C01AD
:109A100097FF0BC08DE20E944159F094E094D094DE
:109A2000C094C11CD11CE11CF11C4AE0C701B60165
:109A3000FF90EF90DF90CF9074CF8F929F92AF9274
:109A4000BF92CF92DF92EF92FF92CF936B017C0196
:109A5000B42E20E030E0A9010F94E41987FF07C07D
:109A60008DE20E944159F7FAF094F7F8F094C0E0C3
:109A700060E070E080E09FE3CB1541F02DEC3CEC22
:109A80004CEC5DE30F94491ACF5FF6CF9B01AC011C
:109A9000C701B6010F94171E6B017C010F94601F64
:109AA0004B015C014AE03DDFCC2389F1C501B401E3
:109AB0000F94E8199B01AC01C701B6010F94161E63
:109AC0006B017C018EE20E94415920E030E040E2CF
:109AD00051E4C701B6010F94491A6B017C010F9440
:109AE0005B1F4B01AA2497FCA094BA2CC501B401BA
:109AF00089DFC501B4010F94EA199B01AC01C701CC
:109B0000B6010F94161E6B017C01C150F1F6CF9186
:109B1000FF90EF90DF90CF90BF90AF909F908F908D
:109B20000895CF93DF930F94280AE0912E09F0E077
:109B3000E457F84F8081882309F458C0EBECF3E137
:109B40008491EF012196882321F00E944159FE0162
:109B5000F7CFC0912E0980E6C89FE0011124C255BD
:109B6000D84F88818E3419F0E8ECF3E110C080E220
:109B70000E94415989910E944159899190ED980F15
:109B80009A30C8F38D32B9F38B32A9F3EDCF8491BB
:109B9000EF012196882321F00E944159FE01F7CF61
:109BA0000F9494086FE070E0681B7109882777FDB7
:109BB0008095982F27DFE5ECF3E18491EF01219662
:109BC000882321F00E944159FE01F7CF80912F098F
:109BD00064E070E0681B7109882777FD8095982FF5
:109BE00011DF8AE0DF91CF910C944159DF91CF9141
:109BF0000895CF93DF938FB7F8949091B60A90931E
:109C0000B50A8FBFEEECF3E18491EF012196882332
:109C100021F00E944159FE01F7CF609157067091E3
:109C200058068091590690915A066F5F7F4F8F4F6B
:109C30009F4FE8DE8AE00E944159DF91CF9171CFBA
:109C4000EF92FF920F931F93CF93DF931F92CDB7A5
:109C5000DEB7082F162FE3E0F2E484917F012FEFA7
:109C6000E21AF20A882331F099830E944159F701E0
:109C70009981F3CFE02FF92F84917F019FEFE91AAB
:109C8000F90A882321F00E944159F701F5CF60912C
:109C90005706709158068091590690915A06B2DE87
:109CA0008AE00E9441591111A4DF1092C110109254
:109CB000C0100F90DF91CF911F910F91FF90EF9007
:109CC0000895CF93DF93E7EBF3E18491EF012196C1
:109CD000882321F00E944159FE01F7CFE3EBF3E125
:109CE0008491EF012196882321F00E944159FE01C1
:109CF000F7CF62B36695617070E080E090E082DE3D
:109D000062B3617070E080E090E07CDE8AE00E94E7
:109D10004159EFEAF3E18491EF012196882321F084
:109D20000E944159FE01F7CF60910601772767FD38
:109D30007095872F972F662797FD6395772788273C
:109D4000992760DE62B362FB662760F970E080E00D
:109D500090E058DE8AE00E944159EBEAF3E18491F9
:109D6000EF012196882321F00E944159FE01F7CF8F
:109D70006091060166FB662760F970E080E090E084
:109D800041DE6091060165FB662760F970E080E0C6
:109D900090E038DE8AE00E944159E6EAF3E18491DE
:109DA000EF012196882321F00E944159FE01F7CF4F
:109DB0006091060163FB662760F970E080E090E047
:109DC00021DE609106016295617070E080E090E0B4
:109DD00019DE8AE00E944159E1EAF3E18491EF0142
:109DE0002196882321F00E944159FE01F7CF60910E
:109DF00006016695617070E080E090E003DE60919E
:109E0000060162FB662760F970E080E090E0FADD11
:109E10008AE0DF91CF910C9441591F93CF93DF9348
:109E200083E50F94B207811104C0C8E2D3E010E0CB
:109E30000DC0C0E00E941B5B682F8C2FD1D7CF5F75
:109E4000C530C1F7F2CF1F5F143059F089910F94DC
:109E5000B2078823C1F30E941B5B682F812FC0D7F4
:109E6000F2CF82E40F94B207882329F00E941B5B93
:109E7000682F84E0B5D7DF91CF911F9122CF0F9348
:109E80001F93CF93DF938B01FC018491EF01219607
:109E9000882321F00E944159FE01F7CFB80188279D
:109EA00077FD8095982FDF91CF911F910F91AACDCB
:109EB000CF93DF9383E50F94B207C82F882371F007
:109EC0000F9444060F945B1F70930B0260930A0279
:109ED00021E0672B09F020E02093360480E50F9401
:109EE000B207882369F080910A0290910B02892BB6
:109EF00019F00E942F5B01C081E0809336042CC0D2
:109F0000C1112AC0EEE3F2E48491EF012196882387
:109F100021F00E944159FE01F7CF80913604882339
:109F200019F066EF72E002C06CE273E08EE893E134
:109F30000E94A29B60910A0270910B028DE793E14F
:109F40009EDFE9E7F3E18491EF012196882321F078
:109F50000E944159FE01F7CFDF91CF91089590E023
:109F6000FC01E252F04C2491FC01EC5DFF4B84912A
:109F7000882399F090E0880F991FFC01EC53F04C76
:109F8000A591B491875E9C4EFC01859194919FB7F9
:109F9000F8948C91822B8C939FBF08951F93CF933D
:109FA000DF93182FEB01DBDF209711F460E004C092
:109FB000CF3FD10539F461E0812FDF91CF911F911F
:109FC0000D94E709E12FF0E0ED5CFC4E449150E088
:109FD000FA013197E231F10508F09BC0EE58FF4FCE
:109FE0000D94062184B5806884BDC7BD97C084B533
:109FF000806284BDC8BD92C08091800080688093DB
:10A000008000D0938900C093880088C08091800030
:10A01000806280938000D0938B00C0938A007EC0C2
:10A0200080918000886080938000D0938D00C093E1
:10A030008C0074C08091B00080688093B000C093A1
:10A04000B3006CC08091B00080628093B000C09378
:10A05000B40064C080919000806880939000D09399
:10A060009900C09398005AC08091900080628093BC
:10A070009000D0939B00C0939A0050C080919000B4
:10A08000886080939000D0939D00C0939C0046C050
:10A090008091A00080688093A0008091A0008F7BB9
:10A0A0008093A000D093A900C093A80037C08091EE
:10A0B000A00080628093A000D093AB00C093AA0060
:10A0C0002DC08091A00088608093A000D093AD0047
:10A0D000C093AC0023C08091200180688093200150
:10A0E000D0932901C093280119C08091200180627A
:10A0F00080932001D0932B01C0932A010FC080913F
:10A100002001886080932001D0932D01C0932C0101
:10A1100005C0C038D1050CF04ECF48CFDF91CF91AC
:10A120001F9108951F93CF93DF93E091BB11F0919E
:10A13000BC11309719F08DEA91E11995C091AF11DA
:10A14000D091B011E091DE11F091DF1182E019950C
:10A15000E091DE11F091DF1181E0199520E030E00F
:10A1600045E1BE018DEA91E10F942009182F882363
:10A1700041F020EE31E147E1BE018DEA91E10F941B
:10A180002009E091DE11F091DF1180E01995812F17
:10A19000DF91CF911F910895CF93C82F8FEF8C0F30
:10A1A000893060F48AE296E00E94316F8C2F0E9421
:10A1B0009D6F80918D060E94856F03C08C2F0E9439
:10A1C0009D6F81E0CF910895CF93DF932FB7F894DF
:10A1D00094E08902E0011124FE01E355F04F608113
:10A1E0007181828193812FBF0F94EA19CF56D84F86
:10A1F000288139814A815B810F94491ADF91CF917F
:10A2000008952FB7F894909105019B7F90930501D5
:10A210002FBF87FD96C0A3982FB7F89490910501A2
:10A220009460909305012FBF880F2FB7F8949091F9
:10A2300005019B7F909305012FBF87FD8EC0A398DA
:10A240002FB7F894909105019460909305012FBF6A
:10A25000880F2FB7F894909105019B7F909305018B
:10A260002FBF87FD78C0A3982FB7F8949091050170
:10A270009460909305012FBF880F2FB7F8949091A9
:10A2800005019B7F909305012FBF87FD62C0A398B6
:10A290002FB7F894909105019460909305012FBF1A
:10A2A000880F2FB7F894909105019B7F909305013B
:10A2B0002FBF87FD4CC0A3982FB7F894909105014C
:10A2C0009460909305012FBF880F2FB7F894909159
:10A2D00005019B7F909305012FBF87FD36C0A39892
:10A2E0002FB7F894909105019460909305012FBFCA
:10A2F000982F990F2FB7F894809105018B7F809349
:10A3000005012FBF97FD1FC0A3982FB7F894809128
:10A3100005018460809305012FBF2FB7F8948091C9
:10A3200005018B7F809305012FBF96FD18C0A39870
:10A330009FB7F894809105018460809305019FBFC9
:10A340000895A39A69CFA39AE0CFA39AC9CFA39AFD
:10A35000B3CFA39A9DCFA39A87CFA39A71CFA39A85
:10A36000E7CFFC0120E03EE2DB014C91403241F0BE
:10A37000283011F430833196DB014C9140833196C3
:10A380002F5F6F5F7F4F2B3079F710820895CF9248
:10A39000DF92EF92FF92C0906406D0906506E09045
:10A3A0006606F09067066091EE0F7091EF0F6850AF
:10A3B0007109882777FD8095982F0F94EA199B01E2
:10A3C000AC01C701B6010F94E41987FF1DC020E05E
:10A3D00030E040E050E4C701B6010F94171E0F941F
:10A3E000601F7093E1066093E0060F941C0A605AA8
:10A3F00075418F4F9F4F6093E2067093E306809301
:10A40000E4069093E50608C01092E2061092E30677
:10A410001092E4061092E506FF90EF90DF90CF9047
:10A420000895CF92DF92EF92FF92C0906006D09095
:10A430006106E0906206F09063066091F20F709101
:10A44000F30F65517109882777FD8095982F0F9438
:10A45000EA199B01AC01C701B6010F94E41987FF0B
:10A460001DC020E030E040E251E4C701B6010F9486
:10A47000171E0F94601F7093E7066093E6060F9413
:10A480001C0A605C73468F4F9F4F6093E806709381
:10A49000E9068093EA069093EB0608C01092E8065E
:10A4A0001092E9061092EA061092EB06FF90EF90E8
:10A4B000DF90CF9008954F925F926F927F928F922C
:10A4C0009F92AF92BF92CF92DF92EF92FF920F9343
:10A4D0001F93CF93DF932C012EE636E181E090E0CD
:10A4E000F90145915491441655060CF062C0AC0137
:10A4F00041505109DA01AA0FBB1FAA0FBB1FA45973
:10A50000B94EFD0165917491440F551F440F551FBD
:10A510004659594EFA0165907490FC01EE0FFF1FE9
:10A52000EE0FFF1FE459F94EA590B490FD0105917F
:10A530001491F901C591D491FA01859094908827DE
:10A5400077FD8095982F0F94EA196B017C01B20179
:10A5500066197709882777FD8095982F0F94EA1957
:10A560002B013C01B501601B710B882777FD80959D
:10A57000982F0F94EA199B01AC01C301B2010F940B
:10A58000491A2B013C01BE0168197909882777FD1A
:10A590008095982F0F94EA199B01AC01C301B20179
:10A5A0000F94F31E9B01AC01C701B6010F94171E57
:10A5B00011C001962C5F3F4F8A33910509F090CF6F
:10A5C000E0E5F7E165917491882777FD8095982FF4
:10A5D0000F94EA19DF91CF911F910F91FF90EF90A7
:10A5E000DF90CF90BF90AF909F908F907F906F90B3
:10A5F0005F904F9008954F925F926F927F928F92EB
:10A600009F92AF92BF92CF92DF92EF92FF92CF9341
:10A61000DF93CDB7DEB72C970FB6F894DEBF0FBE31
:10A62000CDBF8091640690916506A0916606B091B9
:10A63000670689839A83AB83BC836091EE0F709128
:10A64000EF0F882777FD8095982F0F94EA192981BD
:10A650003A814B815C810F94161E6B017C016093E3
:10A66000CE067093CF068093D0069093D1062091AA
:10A6700055103091561040915710509158100F942A
:10A68000491A6D837E838F8398876093CA0670937F
:10A69000CB068093CC069093CD062091C6063091D0
:10A6A000C7064091C8065091C906C701B6010F946C
:10A6B000171E4B015C016093C6067093C70680931A
:10A6C000C8069093C90620915110309152104091C4
:10A6D0005310509154100F94491A69877A878B87C9
:10A6E0009C876093C2067093C3068093C4069093C0
:10A6F000C50620ED3CEC4CE45DE360914D1070919B
:10A700004E1080914F10909150100F94491A2B01C8
:10A710003C012091BE063091BF064091C006509189
:10A72000C10669817A818B819C810F94161E9B01E1
:10A73000AC01C301B2010F94491A2B013C0123E380
:10A7400033E343E75FE36091BA067091BB06809103
:10A75000BC069091BD060F94491A9B01AC01C30140
:10A76000B2010F94171E2B013C016093BA0670933F
:10A77000BB068093BC069093BD0689819A81AB810C
:10A78000BC818093BE069093BF06A093C006B09391
:10A79000C10629853A854B855C856D817E818F81D7
:10A7A00098850F94171EA30192010F94161E2B017A
:10A7B0003C0120E030E04EE453E40F943D2020E0E3
:10A7C00030E0A9011816ACF4C701B6010F943D2082
:10A7D00018166CF5A7019601C501B4010F94161E59
:10A7E0006093C6067093C7068093C8069093C90607
:10A7F0001EC0C301B2010F94E41987FF22C020E0FC
:10A8000030E0A901C701B6010F94E41987FF16C013
:10A81000A7019601C501B4010F94161E6093C606E8
:10A820007093C7068093C8069093C90607C0412C51
:10A83000512C8EE4682E83E4782E03C0412C512CD9
:10A840003201C301B2012C960FB6F894DEBF0FBEE1
:10A85000CDBFDF91CF91FF90EF90DF90CF90BF9071
:10A86000AF909F908F907F906F905F904F900895E2
:10A870004F925F926F927F928F929F92AF92BF9210
:10A88000CF92DF92EF92FF920F931F93CF93DF93BC
:10A8900000D01F92CDB7DEB70091F20F1091F30FE9
:10A8A0008090600690906106A0906206B09063066A
:10A8B000B801882777FD8095982F0F94EA19A50194
:10A8C00094010F94161E6B017C016093B606709381
:10A8D000B7068093B8069093B90620ED3CEC4CE4A3
:10A8E0005DE360914110709142108091431090910E
:10A8F00044100F94491A2B013C012091B20630916B
:10A90000B3064091B4065091B506C501B4010F9449
:10A91000161E9B01AC01C301B2010F94491A2B0111
:10A920003C0123E333E343E75FE36091AE067091BC
:10A93000AF068091B0069091B1060F94491A9B0121
:10A94000AC01C301B2010F94171E69837A838B8314
:10A950009C836093AE067093AF068093B00690938D
:10A96000B1068092B2069092B306A092B406B0925D
:10A97000B50680917206882321F081E08093AD06B0
:10A98000B9C020E030E040E251E4C701B6010F94C5
:10A990003D20181624F481E08093AD06A4C020E089
:10A9A00030E040E251ECC701B6010F94E41987FD95
:10A9B000E4CF012B11F38091AD06882351F0109262
:10A9C000A9061092AA061092AB061092AC0610923D
:10A9D000AD062091491030914A1040914B10509192
:10A9E0004C10C701B6010F94491A2B013C0160932A
:10A9F000A5067093A6068093A7069093A8062091BB
:10AA0000A9063091AA064091AB065091AC06C70149
:10AA1000B6010F94171E4B015C016093A906709359
:10AA2000AA068093AB069093AC0620914510309116
:10AA3000461040914710509148100F94491A9B01BD
:10AA4000AC016093A1067093A2068093A306909335
:10AA5000A406C301B2010F94171E29813A814B81CC
:10AA60005C810F94161E2B013C0120E030E04FE783
:10AA700053E40F943D2020E030E0A9011816ACF417
:10AA8000C701B6010F943D2018166CF5A701960179
:10AA9000C501B4010F94161E6093A9067093AA060F
:10AAA0008093AB069093AC061EC0C301B2010F9415
:10AAB000E41987FF22C020E030E0A901C701B601F8
:10AAC0000F94E41987FF16C0A7019601C501B401D0
:10AAD0000F94161E6093A9067093AA068093AB0686
:10AAE0009093AC0607C0412C512C9FE7692E93E44C
:10AAF000792E03C0412C512C3201C301B2010F90B9
:10AB00000F900F900F90DF91CF911F910F91FF90B9
:10AB1000EF90DF90CF90BF90AF909F908F907F90FD
:10AB20006F905F904F9008956091640670916506F4
:10AB3000809166069091670608954F925F926F929A
:10AB40007F928F929F92AF92BF92CF92DF92EF92BD
:10AB5000FF920F931F93CF93DF932C012BED33E1E3
:10AB600081E090E0F90145915491441655060CF0AE
:10AB700062C0AC0141505109DA01AA0FBB1FAA0FF4
:10AB8000BB1FA752BC4EFD0165917491440F551F28
:10AB9000440F551F49525C4EFA0165907490FC01B8
:10ABA000EE0FFF1FEE0FFF1FE752FC4EA590B49073
:10ABB000FD0105911491F901C591D491FA01859097
:10ABC0009490882777FD8095982F0F94EA196B0150
:10ABD0007C01B20166197709882777FD8095982F47
:10ABE0000F94EA192B013C01B501601B710B8827FA
:10ABF00077FD8095982F0F94EA199B01AC01C30152
:10AC0000B2010F94491A2B013C01BE016819790960
:10AC1000882777FD8095982F0F94EA199B01AC0146
:10AC2000C301B2010F94F31E9B01AC01C701B60131
:10AC30000F94171E11C001962C5F3F4F8032910573
:10AC400009F090CFE5E5F4E165917491882777FDEF
:10AC50008095982F0F94EA19DF91CF911F910F9152
:10AC6000FF90EF90DF90CF90BF90AF909F908F902C
:10AC70007F906F905F904F90089560916006709103
:10AC800061068091620690916306089567FD5CC03D
:10AC9000823021F128F4882349F0813069F054C0D2
:10ACA000833071F1843009F43DC04EC0662311F049
:10ACB000A19A8FC0A1988DC09FB7662329F0F89400
:10ACC00080910801806804C0F894809108018F7712
:10ACD000809308019FBF47FF4CC07FC09FB766238A
:10ACE00029F0F89480910801806404C0F894809160
:10ACF00008018F7B809308019FBF47FF40C06FC052
:10AD00009FB7662329F0F89480910801886004C0F9
:10AD1000F89480910801877F809308019FBF47FFC7
:10AD20003EC05AC09FB7662329F0F894809108016D
:10AD3000826004C0F894809108018D7F809308019F
:10AD40009FBF47FF39C04AC047FD49C08230B9F0B4
:10AD500028F4882341F0813061F008958330F9F0C0
:10AD6000843051F10895442311F0A09A0895A098D9
:10AD70000895442311F0A29A0895A29808959FB7C8
:10AD8000442329F0F89480910801806204C0F8946B
:10AD9000809108018F7D809308019FBF08959FB720
:10ADA000442329F0F894809108018061F4CFF8944D
:10ADB000809108018F7EEFCF9FB7442329F0F8944C
:10ADC000809108018460E7CFF894809108018B7F1F
:10ADD000E2CF47FFC8CF08950895089508950895D4
:10ADE000643079F028F4613041F0623041F0089528
:10ADF000683051F0603141F0089540E003C040E018
:10AE000004C041E060E002C041E061E03FCF24E0E7
:10AE10008202C0011124FC01E355F04F40815181B1
:10AE200062817381FC01EF55F84F40835183628347
:10AE30007383E091E00FF091E10F82899389A489F7
:10AE4000B5898093BD0F9093BE0FA093BF0FB093B1
:10AE5000C00F089580E0B8D9609307077093080782
:10AE60008093090790930A0781E0AED960930B079E
:10AE700070930C0780930D0790930E0782E0A4D97E
:10AE800060930F0770931007809311079093120738
:10AE900008958091DF0F9FB780FF09C0F8948091DB
:10AEA0000B018D7F80930B019FBF8FEF08C0F8943B
:10AEB00080910B01826080930B019FBF81E08093A2
:10AEC0008A028091DF0F9FB781FF09C0F8948091BB
:10AED0000B01816080930B019FBF8FEF08C0F89436
:10AEE00080910B018E7F80930B019FBF81E0809347
:10AEF0008B028091DF0F9FB782FF09C0F894809189
:10AF00000B018B7F80930B019FBF8FEF08C0F894DC
:10AF100080910B01846080930B019FBF81E080933F
:10AF20008C028091DF0F9FB783FF09C0F894809156
:10AF30000B01806480930B019FBF8FEF08C0F894D2
:10AF400080910B018F7B80930B019FBF81E08093E9
:10AF50008D0208954F925F926F927F92AF92BF924F
:10AF6000CF92DF92EF92FF920F931F93CF93DF93D5
:10AF70008C01EB01FC0147A050A461A472A4AFA016
:10AF8000B8A4C9A4DAA49501A601C301B2010F9423
:10AF9000E41987FF40C0A3019201C301B2010F94DD
:10AFA000491A2B013C01F80183A994A9A5A9B6A9C6
:10AFB000BC01CD0190589B01AC010F94171EF80104
:10AFC00027A530A941A952A90F94491A9B01AC01A8
:10AFD000C301B2010F94161E0F9482207B018C01D5
:10AFE0009B01AC01B501C6010F94E41987FF02C0B3
:10AFF000750186019701A801B501C6010F94E419F6
:10B00000882349F0A701B8014FA358A769A77AA7D9
:10B01000888181608883DF91CF911F910F91FF908C
:10B02000EF90DF90CF90BF90AF907F906F905F9048
:10B030004F9008958F929F92AF92BF92CF92DF92DE
:10B04000EF92FF920F931F93CF93DF9300D01F9245
:10B05000CDB7DEB719E6812E11E1912E0AEFA02EB1
:10B0600000E1B02E04E311E1C12CD12C7601C39490
:10B07000F40161917191819191914F01F5012191BB
:10B080003191419151915F0129833A834B835C83D4
:10B090000F94E81929813A814B815C810F94491AF8
:10B0A0000F94601FF80161937193819391938F01C5
:10B0B000C616D706E806F90610F46B017C01F9E71D
:10B0C0008F16F1E19F06A1F66FEF7FEFCB01A7018D
:10B0D00096010F94B91D20930E1030930F104093DA
:10B0E0001010509311100F900F900F900F90DF9150
:10B0F000CF911F910F91FF90EF90DF90CF90BF9075
:10B10000AF909F908F9008950F931F93CF93DF93ED
:10B11000C8E2D3E009E611E189910F94B2078823D0
:10B1200049F00F9444060F94601FF8016083718307
:10B13000828393830C5F1F4FF3E0CC32DF0761F70C
:10B14000DF91CF911F910F9175CF61E0FC0180815C
:10B150000D94E7098EBD0DB407FEFDCF08958FEF66
:10B160008EBD0DB407FEFDCF8EB508950F931F93CE
:10B17000CF93DF93EB010F941C0A8B01F0DF8F3F1D
:10B1800049F00F941C0A601B710B6C177D07B0F31C
:10B1900080E001C081E0DF91CF911F910F91089570
:10B1A000CF92DF92FF920F931F93CF93DF9300D044
:10B1B0001F92CDB7DEB76C01F62EFC018281982F6D
:10B1C000906A96959CBD80FD06C091E0863009F49A
:10B1D00090E0892F01C080E08DBD60E0F6018081A4
:10B1E00029833A834B835C830F94E7096CE271E017
:10B1F000C601BCDF8F2D8064ADDF08E110E05C810B
:10B200004B813A812981DA01C901002E04C0B6952B
:10B21000A795979587950A94D2F729833A834B830C
:10B220005C8398DF0850110929813A814B815C8148
:10B23000083FFFEF1F0739F7FF2029F088E0F816D5
:10B2400021F08FEF03C085E901C087E883DFECE0E0
:10B25000FE1201C084DF10E082DFF601838387FFE6
:10B2600004C01F3F11F01F5FF7CF0F900F900F909A
:10B270000F90DF91CF911F910F91FF90DF90CF90B2
:10B2800008959091C00095FFFCCF8093C60008956B
:10B29000EF92FF921F93CF93DF931F92CDB7DEB74C
:10B2A000182FE2E6F6E184917F012FEFE21AF20A0D
:10B2B000882329F09983E5DFF7019981F4CFE12F05
:10B2C000F92F84917F019FEFE91AF90A882319F079
:10B2D000D8DFF701F6CFE9E4F6E184917F01AFEF23
:10B2E000EA1AFA0A882319F0CCDFF701F6CF0F909B
:10B2F000DF91CF911F91FF90EF900895CF93DF934F
:10B3000083E50F941308882319F00F94340602C0C4
:10B3100060E070E0EB01DD27C230D105A8F0E3E08A
:10B32000F2E48491EF012196882319F0AADFFE014F
:10B33000F8CFE7E2F6E18491EF012196882309F442
:10B340004DC09FDFFE01F7CF88E40F9413088823D8
:10B35000A9F00F943406683771053CF0633281E040
:10B3600078072CF062E271E002C068E770E0FE014D
:10B37000EE0FFF1FEE5AFE4E7183608386E40F943A
:10B380001308882399F00F9434066F3F710519F064
:10B3900014F06FEF70E0FE01EE0FFF1FE65BFE4E54
:10B3A00077FF02C060E070E07183608382E40F94F5
:10B3B0001308882399F00F9434066530710534F032
:10B3C000683871052CF067E870E002C065E070E055
:10B3D000CC0FDD1FC25BDE4E79836883DF91CF9196
:10B3E0000895CF93DF93E2E3F5E18491EF01219695
:10B3F000882319F046DFFE01F8CFE4E2F5E18491FD
:10B40000EF012196882319F03CDFFE01F8CFEDE033
:10B41000F5E18491EF012196882319F032DFFE01D6
:10B42000F8CFEDEFF4E18491EF012196882319F034
:10B4300028DFFE01F8CFECEEF4E18491EF012196D4
:10B44000882319F01EDFFE01F8CFEBEDF4E18491C3
:10B45000EF012196882319F014DFFE01F8CFECEC00
:10B46000F4E18491EF012196882319F00ADFFE01AF
:10B47000F8CFE7EBF4E18491EF012196882319F0EE
:10B4800000DFFE01F8CFE1EAF4E18491EF012196BB
:10B49000882319F0F6DEFE01F8CFECE8F4E18491A0
:10B4A000EF012196882319F0ECDEFE01F8CFEFE6DC
:10B4B000F4E18491EF012196882319F0E2DEFE0188
:10B4C000F8CFE7E5F4E18491EF012196882319F0A4
:10B4D000D8DEFE01F8CFDF91CF9108953FB7F89401
:10B4E0002091B60A8091B50A821759F0E22FF0E058
:10B4F000EB5CF54F808190E02F5F2F772093B60AA9
:10B5000002C08FEF9FEF3FBF0895CF93FC01C62F7E
:10B5100080818B33A1F080912F09843080F42091B9
:10B520005A1030E6239FC0011124BF018255984F65
:10B530000F9457218C2F0F949D0781E001C080E06C
:10B54000CF91089580919F069091A006009731F0C9
:10B550004AE050E060E070E00D94241860E070E094
:10B56000CB01089583E50F94B207882351F00F941F
:10B5700044066093E2107093E3108093E41090937C
:10B58000E51084E50F94B207882351F00F94440628
:10B590006093DE107093DF108093E0109093E110C1
:10B5A00082E40F94B207882349F0CCDF60935611F0
:10B5B00070935711809358119093591188E50F9407
:10B5C000B207882351F00F944406609317117093CB
:10B5D00018118093191190931A1189E50F94B207ED
:10B5E000882351F00F94440660931B1170931C1133
:10B5F00080931D1190931E118AE50F94B207882342
:10B6000051F00F94440660931F11709320118093A2
:10B6100021119093221185E40F94B207882351F0F1
:10B620000F94440660932311709324118093251185
:10B630009093261108950F94340697FD0EC00F9431
:10B6400034066F3F71058105910509F01CF40F94D4
:10B65000340601C06FEF862F089580E00895809131
:10B660009F069091A006892B39F0E5DF91E08111CA
:10B6700001C090E0892F089581E0089583E50F943B
:10B68000B207882319F0EBDF809390070895CF93DA
:10B69000DF93C0912814CC23C1F0C150C09328146B
:10B6A0008FE1C89FE0011124CE50DD4E8BE1FE01F9
:10B6B0003496A7EDB2E101900D928A95E1F78A8167
:10B6C0009B819093D6128093D5121092861181E0BF
:10B6D0008093871183E08093A802DF91CF91089532
:10B6E0005F988EBD00000DB407FEFDCF8EB56EBD18
:10B6F00000000DB407FEFDCF8EB55F9A0895CF927E
:10B70000DF92EF92FF920F931F93CF93DF93EC01A1
:10B710000F941C0A0E811F8128853985011511059A
:10B720002105310559F53C853323A9F12A8531508E
:10B730003C8731E0320F3A874D85341301C01A86B9
:10B74000FE0134E0239FE00DF11D112406851785CD
:10B75000208931890A831B832C833D836B017C0103
:10B76000C00ED11EE11CF11CCE82DF82E886F98674
:10B770008C819D81892B79F0769A0DC06B017C01BB
:10B78000C01AD10AE20AF30AF7FC05C076981E82B5
:10B790001F8218861986DF91CF911F910F91FF901C
:10B7A000EF90DF90CF9008950F931F93CF93DF9387
:10B7B0008C01EB01DC0113968C918823C1F182503E
:10B7C000823028F48FE28883198281E031C0F80149
:10B7D000648575858685978540E00E94D4708823AE
:10B7E00039F1D8015096EC91B0E2EB9FF0011124B1
:10B7F000E95AFB4F3097D9F090E020E03EE24081DB
:10B80000403269F0283029F4DE01A90FB11D3C93C4
:10B810009F5F4081DE01A90FB11D4C939F5F2F5F99
:10B8200031962B3061F7C90FD11D188201C080E01D
:10B83000DF91CF911F910F910895CF93DF93809166
:10B84000E611811107C081E08093E6118DEA91E154
:10B850000F942409C091AF11D091B011E091DE1185
:10B86000F091DF1182E01995E091DE11F091DF1186
:10B8700081E0199520E030E044E1BE018DEA91E1DC
:10B880000F94200920EE31E147E1BE018DEA91E1FC
:10B890000F942009E091DE11F091DF1180E0DF913B
:10B8A000CF9119941092F30F1092F20F80E00E9442
:10B8B00011521092EF0F1092EE0F0E94C7510E948A
:10B8C00045771092F30F1092F20F80E00E94115210
:10B8D000109208109FB7F894E2E0F1E080818F7B2E
:10B8E00080839FBF1092EF0F1092EE0F1092061000
:10B8F0007598089510926111109260111092631161
:10B9000010926211CFDF0C9445A790912F12809175
:10B910003012981731F0809130128F5F8F708093C2
:10B92000301208950F931F93CF93DF93EC01FC0126
:10B93000E65AFF4F1082138234971382128280E2FC
:10B9400093E091838083B59610821382349713829B
:10B950001282918380838E010A561F4F9E012453C9
:10B960003E4FF801B8016C5F7F4FAC01CF01801BE7
:10B97000910B860F971FDC011C9213961C92138269
:10B980001282518340837F96E217F30779F7CE0145
:10B9900083539E4F29E1DC0111962C931197149645
:10B9A0001C920596DC0157961C928296DC011C9233
:10B9B00013961C920497DC0113961C921E92129708
:10B9C00020E233E02D933C93198218821B821A8265
:10B9D0008F549F4FDC011D921D921D921C92139754
:10B9E0000496DC011D921D921D921C9213971082E9
:10B9F000FE01E15FFD4F108286E391E0F8019C01BA
:10BA0000119221503040E1F7FE01E355FD4F81E0F6
:10BA10008083E955F240118210820F941C0AC755A9
:10BA2000DD4F68577C4E8F4F9F4F688379838A83A1
:10BA30009B83DF91CF911F910F9108952F923F9299
:10BA40004F925F926F927F928F929F92AF92BF922E
:10BA5000CF92DF92EF92FF920F931F93CF93DF93DA
:10BA6000CDB7DEB768970FB6F894DEBF0FBECDBF77
:10BA70001C015B018A01DC01D7966D917D918D914E
:10BA80009C91DA970F94E8196B017C01F5012081F4
:10BA90003181428153810F94491A0F94DD1E0F9416
:10BAA000601F69877A878B879C87D8012D913D918C
:10BAB0004D915C91C701B6010F94491A0F94DD1E98
:10BAC0000F94601F6D877E878F87988B29853A85B5
:10BAD0004B855C85283731054105510540F488E7E1
:10BAE00090E0A0E0B0E089879A87AB87BC872D857E
:10BAF0003E854F855889283731054105510540F469
:10BB000088E790E0A0E0B0E08D879E87AF87B88B94
:10BB100091012D5B3F4FD9018D919D910D90BC916D
:10BB2000A02D8D839E83AF83B887BC01CD010F9478
:10BB3000EA1969837A838B839C8369857A858B85EF
:10BB40009C850F94E819698B7A8B8B8B9C8B20E0FA
:10BB500030E0A90169817A818B819C810F94E4197D
:10BB6000882339F1A7019601C701B6010F94491A3C
:10BB70004B015C0129893A894B895C89CA01B90169
:10BB80000F94491A9B01AC01C501B4010F94161E14
:10BB90004B015C0129813A814B815C81CA01B90169
:10BBA0000F94171E9B01AC01C501B4010F94F31E45
:10BBB00003C060E070E0CB010F94DD1E0F945B1FAB
:10BBC0002B013C016D817E818F81988590958095B8
:10BBD000709561957F4F8F4F9F4F0F94EA194B01DE
:10BBE0005C016D857E858F8598890F94E8196D833A
:10BBF0007E838F83988720E030E0A901C501B401DE
:10BC00000F94E419882349F12D813E814F81588595
:10BC1000CA01B9010F94491A6D8B7E8B8F8B988F57
:10BC2000A7019601C701B6010F94491A9B01AC0107
:10BC30006D897E898F89988D0F94161E6B017C010A
:10BC4000A5019401C501B4010F94171E9B01AC011D
:10BC5000C701B6010F94F31E03C060E070E0CB0192
:10BC60000F948C1FF10182889388A488B588750190
:10BC70006401C418D508E608F7080F945B1FC61ABC
:10BC8000D70AE80AF90AF7FE6BC020E030E0A90104
:10BC900069817A818B819C810F94E419882309F44E
:10BCA00047C029813A814B815C81CA01B9010F9457
:10BCB000171E6B017C01C501B4010F94E8199B01AB
:10BCC000AC01C701B6010F94491A6B017C012989A7
:10BCD0003A894B895C89CA01B9010F94491A9B01C1
:10BCE000AC01C701B6010F94161E6B017C012D81BA
:10BCF0003E814F815885CA01B9010F94491A9B01B1
:10BD0000AC01C701B6010F94171E6B017C0120E046
:10BD100030E040E850E469817A818B819C810F9406
:10BD2000491A9B01AC01C701B6010F94F31E03C071
:10BD300060E070E0CB010F94DD1E0F945B1F2B01C0
:10BD40003C0197FF03C0412C512C32014814590487
:10BD50006A047B0410F024013501C12CD12C76013A
:10BD60008FB7F894D1019C9193FD22C0F101468ACE
:10BD7000578A608E718EC40CD51CE61CF71C5A962F
:10BD8000CD92DD92ED92FC925D9729853A854B85A7
:10BD90005C85DB962D933D934D935C93DE97FF96E8
:10BDA0002D853E854F855889208331834283538377
:10BDB0008FBF68960FB6F894DEBF0FBECDBFDF9180
:10BDC000CF911F910F91FF90EF90DF90CF90BF9098
:10BDD000AF909F908F907F906F905F904F903F902B
:10BDE0002F900895CF93DF9383E50F941308882352
:10BDF00021F00F943406EB0102C0C0E0D0E080E5F2
:10BE00000F941308882321F00F943406CB0102C04D
:10BE100080E090E0BE01DF91CF9162CCCF93DF93C1
:10BE200000D01F921F92CDB7DEB795E0E9EAF2E0AD
:10BE3000DE01119601900D929A95E1F7E1E0F0E0B4
:10BE4000EC0FFD1FE80FF11D808190E00F900F9027
:10BE50000F900F900F90DF91CF9142CC1F93CF9313
:10BE6000DF93C8E2D3E010E089910F94B2078823F2
:10BE700021F00F943406812FD1DF1F5F1430A1F71A
:10BE800082E40F94B207882321F00F94340684E0F3
:10BE9000C5DF83E50F94B207882341F0C0E00F941B
:10BEA00034068C2FBBDFCF5FC530C9F7DF91CF9150
:10BEB0001F9108958F929F92AF92BF92CF92DF927F
:10BEC000EF92FF92CF93C82FC0905802D0905902A2
:10BED000E0905A02F0905B02A7019601C701B601FB
:10BEE0000F94C3208090FA069090FB06A090FC0669
:10BEF000B090FD06811129C0C11127C080916B0649
:10BF0000882319F1A7019601C501B4010F94161EEB
:10BF100020910211309103114091041150910511AB
:10BF20000F94491A0F944820719561957109809179
:10BF30006C07882351F08091EC0F9091ED0F860FE4
:10BF4000971F9093ED0F8093EC0F80925802909280
:10BF50005902A0925A02B0925B02CF91FF90EF90EB
:10BF6000DF90CF90BF90AF909F908F900895CF9229
:10BF7000DF92EF92FF92EEE3F2E484917F019FEF74
:10BF8000E91AF90A882319F07CD9F701F6CFE4EF12
:10BF9000F9E184917F019FEFE91AF90A882319F0EA
:10BFA00070D9F701F6CF8AE50F94B2078823C1F163
:10BFB0000F9444066B017C0120E030E040E050EC3F
:10BFC0000F943D2087FD20C020E030E040EA50E49F
:10BFD000C701B6010F94E4191816B4F0C092FA061E
:10BFE000D092FB06E092FC06F092FD0680E062DF54
:10BFF0006091FA067091FB068091FC069091FD0617
:10C0000042E00E941D4D18C0EFEDF9E184917F01DF
:10C010009FEFE91AF90A882379F033D9F701F6CFAF
:10C020004091FA065091FB066091FC067091FD0666
:10C030008CED99E10E946BBD8AE0FF90EF90DF905C
:10C04000CF901FC9AF92BF92CF92DF92EF92FF9233
:10C050000F931F93CF93C82F882319F0E4ECF9E1D5
:10C060000BC0EEE3F2E484918F010F5F1F4F882332
:10C07000A9F307D9F801F7CF84918F010F5F1F4F04
:10C08000882319F0FED8F801F7CFCC2319F0E7EA9E
:10C09000F9E10BC0EEE3F2E484918F010F5F1F4FD3
:10C0A0008823A9F3EED8F801F7CF84918F010F5FB1
:10C0B0001F4F882319F0E5D8F801F7CF8AE0E1D8BF
:10C0C000C11129C0EEE3F2E484918F010F5F1F4F8D
:10C0D000882319F0D6D8F801F7CFE4E9F9E1849183
:10C0E0008F010F5F1F4F882319F0CBD8F801F7CFCE
:10C0F00080914911882319F08AE0C3D8BCC3E9E8CC
:10C10000F9E184918F010F5F1F4F882309F4B3C3B6
:10C11000B8D8F801F6CF4091451150914611609181
:10C1200047117091481180E899E10E946BBD8AE047
:10C13000A8D880914911811119C0CC2319F0E5E7E5
:10C14000F9E10BC0EEE3F2E484918F010F5F1F4F22
:10C150008823A9F396D8F801F7CF84918F010F5F58
:10C160001F4F882319F08DD8F801F7CFC11121C0D6
:10C17000EEE3F2E484918F010F5F1F4F882319F0E3
:10C1800080D8F801F7CFE4E6F9E184918F010F5FE1
:10C190001F4F882319F075D8F801F7CFEEE3F2E4CA
:10C1A00084918F010F5F1F4F882319F06AD8F8011F
:10C1B000F7CF4091FA105091FB106091FC107091F4
:10C1C000FD108CE599E10E946BBD4091FE105091ED
:10C1D000FF10609100117091011189E599E10E94B1
:10C1E0006BBD409102115091031160910411709147
:10C1F000051186E599E10E946BBD409106115091B1
:10C200000711609108117091091183E599E10E946D
:10C210006BBD8AE036D8C11121C0EEE3F2E484910F
:10C220008F010F5F1F4F882319F02BD8F801F7CF2C
:10C23000E5E3F9E184918F010F5F1F4F882319F027
:10C2400020D8F801F7CFEEE3F2E484918F010F5F7D
:10C250001F4F882319F015D8F801F7CF4091E61049
:10C260005091E7106091E8107091E9108CE299E12B
:10C270000E946BBD4091EA105091EB106091EC1060
:10C280007091ED1089E299E10E946BBD4091EE1032
:10C290005091EF106091F0107091F11086E299E1E9
:10C2A0000E946BBD4091F2105091F3106091F41018
:10C2B0007091F51083E299E10E946BBD8AE00E94C3
:10C2C0004159C11124C0EEE3F2E484918F010F5F64
:10C2D0001F4F882321F00E944159F801F6CFE1E079
:10C2E000F9E184918F010F5F1F4F882321F00E9495
:10C2F0004159F801F6CFEEE3F2E484918F010F5F2C
:10C300001F4F882321F00E944159F801F6CF409138
:10C31000691150916A1160916B1170916C1188EFE5
:10C3200098E10E9467C140916D1150916E1160912A
:10C330006F117091701185EF98E10E9467C1409173
:10C34000711150917211609173117091741182EF9B
:10C3500098E10E9467C140917511509176116091EA
:10C360007711709178118FEE98E10E9467C18AE091
:10C370000E944159C11124C0EEE3F2E484918F017F
:10C380000F5F1F4F882321F00E944159F801F6CF1B
:10C39000E5EAF8E184918F010F5F1F4F882321F0B8
:10C3A0000E944159F801F6CFEEE3F2E484918F0147
:10C3B0000F5F1F4F882321F00E944159F801F6CFEB
:10C3C000409181115091821160918311709184117B
:10C3D0008CE998E10E946BBD40917D1150917E11D6
:10C3E00060917F117091801189E998E10E946BBD85
:10C3F0004091791150917A1160917B1170917C116B
:10C4000086E998E10E946BBD8AE00E944159C11102
:10C4100024C0EEE3F2E484918F010F5F1F4F882365
:10C4200021F00E944159F801F6CFE2E2F8E184914F
:10C430008F010F5F1F4F882321F00E944159F8019F
:10C44000F6CFEEE3F2E484918F010F5F1F4F882354
:10C4500021F00E944159F801F6CF4091E21050912D
:10C46000E3106091E4107091E51089E198E10E9479
:10C470006BBD4091DE105091DF106091E010709123
:10C48000E11086E198E10E946BBD409156115091F8
:10C490005711609158117091591183E198E10E94F0
:10C4A00067C1409117115091181160911911709145
:10C4B0001A1180E198E10E946BBD40911B115091CF
:10C4C0001C1160911D1170911E118DE098E10E9468
:10C4D0006BBD40911F1150912011609121117091FD
:10C4E00022118AE098E10E946BBD40912311509186
:10C4F0002411609125117091261187E098E10E9426
:10C500006BBD8AE00E944159C11124C0EEE3F2E400
:10C5100084918F010F5F1F4F882321F00E944159A2
:10C52000F801F6CFE9EFF7E184918F010F5F1F4F1C
:10C53000882321F00E944159F801F6CFEEE3F2E49E
:10C5400084918F010F5F1F4F882321F00E94415972
:10C55000F801F6CF40917007509171076091720712
:10C560007091730780EF97E10E946BBD4091740753
:10C570005091750760917607709177078DEE97E17E
:10C580000E946BBD409178075091790760917A07BE
:10C5900070917B078AEE97E10E946BBD8AE00E9452
:10C5A0004159C11124C0EEE3F2E484918F010F5F81
:10C5B0001F4F882321F00E944159F801F6CFE6ED84
:10C5C000F7E184918F010F5F1F4F882321F00E94B4
:10C5D0004159F801F6CFEEE3F2E484918F010F5F49
:10C5E0001F4F882321F00E944159F801F6CF609136
:10C5F0006B0670E08DEC97E10E943F4F8AE00E944D
:10C600004159CC2379F082E5A82E81E1B82E9EE431
:10C61000C92E91E1D92E2AE4E22E21E1F22E00E08A
:10C6200010E024C0EEE3F2E484918F010F5F1F4F0E
:10C63000882321F00E944159F801F6CFE0EBF7E1A1
:10C6400084918F010F5F1F4F882321F00E94415971
:10C65000F801F6CFEEE3F2E484918F010F5F1F4FF4
:10C66000882389F20E944159F801F6CFB80187EA80
:10C6700097E10E943F4FF501619171915F0184EA5A
:10C6800097E10E943F4FF601619171916F0181EA3C
:10C6900097E10E943F4FF701619171917F018EE90F
:10C6A00097E10E943F4F8AE00E9441590F5F1F4F60
:10C6B00002301105D9F6C11124C0EEE3F2E48491F1
:10C6C0008F010F5F1F4F882321F00E944159F8010D
:10C6D000F6CFEFE8F7E184918F010F5F1F4F8823BA
:10C6E00021F00E944159F801F6CFEEE3F2E4849183
:10C6F0008F010F5F1F4F882321F00E944159F801DD
:10C70000F6CF4091491050914A1060914B107091B2
:10C710004C1086E897E10E946BBD2CEA35EC47E2AD
:10C720005EE36091451070914610809147109091A2
:10C7300048100F94F31EAB01BC0183E897E10E94FF
:10C740004EBD2CEA35EC47E25EE3609141107091FA
:10C75000421080914310909144100F94491AAB01FC
:10C76000BC0180E897E10E944EBD8AE00E944159D9
:10C77000C1110CC0EEE3F2E484918F010F5F1F4FF3
:10C78000882321F00E944159F801F6CF40915510BD
:10C7900050915610609157107091581087E797E1AB
:10C7A0000E946BBD2CEA35EC47E25EE360915110CC
:10C7B0007091521080915310909154100F94F31E69
:10C7C000AB01BC0184E797E10E944EBD2CEA35EC39
:10C7D00047E25EE360914D1070914E1080914F10D2
:10C7E000909150100F94491AAB01BC0181E797E179
:10C7F0000E944EBD8AE00E944159C11124C0EEE35F
:10C80000F2E484918F010F5F1F4F882321F00E9473
:10C810004159F801F6CFEBE5F7E184918F010F5F05
:10C820001F4F882321F00E944159F801F6CFEEE313
:10C83000F2E484918F010F5F1F4F882321F00E9443
:10C840004159F801F6CF4091FA065091FB066091EC
:10C85000FC067091FD0682E597E10E946BBD8AE0BF
:10C86000CF911F910F91FF90EF90DF90CF90BF90ED
:10C87000AF900C944159EEE3F2E484918F010F5F85
:10C880001F4F882309F447CC0E944159F801F5CF86
:10C8900083E50F94B207882319F00E942F5B01C033
:10C8A00081E091E08927CECBCF92DF92EF92FF9289
:10C8B0001F93CF93DF9300D01F92CDB7DEB7809147
:10C8C000891190918A11A0918B11B0918C11B7FFB1
:10C8D00008C01092891110928A1110928B11109237
:10C8E0008C1180910B1190910C11A0910D11B091B0
:10C8F0000E114091891150918A1160918B117091A4
:10C900008C1184179507A607B70744F48093891103
:10C9100090938A11A0938B11B0938C118091A802EF
:10C92000882359F16091891170918A1180918B113E
:10C9300090918C11C0900F11D0901011E0901111B6
:10C94000F09012116C0D7D1D8E1D9F1D0F94E81926
:10C9500020E030E048EC52E40F94491A69837A836E
:10C960008B839C83CE0101960E94209DBC01809107
:10C970001511909116110E94A1A880918511109116
:10C98000F710811106C01123C1F18091A8028823FC
:10C99000A1F16091891170918A1180918B11909110
:10C9A0008C11C0900F11D0901011E0901111F090E7
:10C9B00012116C0D7D1D8E1D9F1D0F94E81920E036
:10C9C00030E048EC52E40F94491A0F94601FE09154
:10C9D0001311F0911411309721F0608371838283D9
:10C9E0009383112329F0E091F810F091F910199533
:10C9F0008091851181110E944BA780918511882318
:10CA000029F0E091F810F091F91019950F900F901E
:10CA10000F900F90DF91CF911F91FF90EF90DF90DB
:10CA2000CF900895CF92DF92EF92FF921F93CF9312
:10CA3000DF9300D01F92CDB7DEB78091891190911E
:10CA40008A11A0918B11B0918C11B7FF08C0109280
:10CA5000891110928A1110928B1110928C11809171
:10CA60000B1190910C11A0910D11B0910E114091EC
:10CA7000891150918A1160918B1170918C118417DA
:10CA80009507A607B70744F48093891190938A11FC
:10CA9000A0938B11B0938C118091A802882359F137
:10CAA0006091891170918A1180918B1190918C11F4
:10CAB000C0900F11D0901011E0901111F090121150
:10CAC0006C0D7D1D8E1D9F1D0F94EA1920E030E036
:10CAD00048EC52E40F94491A69837A838B839C83D0
:10CAE000CE0101960E94209DBC018091151190916C
:10CAF00016110E94A1A8809185111091F710811143
:10CB000006C01123B1F18091A802882391F16091B0
:10CB1000891170918A1180918B1190918C11C09024
:10CB20000F11D0901011E0901111F09012116C0DB6
:10CB30007D1D8E1D9F1D0F94EA1920E030E048EC0A
:10CB400052E40F94491AE0911311F09114113097A7
:10CB500021F06083718382839383112329F0E09114
:10CB6000F810F091F91019958091851181110E94AA
:10CB70004BA70F900F900F900F90DF91CF911F91C7
:10CB8000FF90EF90DF90CF900895CF92DF92EF92D9
:10CB9000FF921F93CF93DF9300D01F92CDB7DEB7E4
:10CBA0008091891190918A11A0918B11B0918C1173
:10CBB000B7FF08C01092891110928A1110928B1140
:10CBC00010928C1180910B1190910C11A0910D116C
:10CBD000B0910E114091891150918A1160918B1181
:10CBE00070918C1184179507A607B70744F48093BA
:10CBF000891190938A11A0938B11B0938C1180911D
:10CC0000A802882359F16091891170918A1180914D
:10CC10008B1190918C11C0900F11D0901011E09059
:10CC20001111F09012116C0D7D1D8E1D9F1D0F9422
:10CC3000EA192AE037ED43E25CE30F94491A69836D
:10CC40007A838B839C83CE0101960E94EA9BBC0170
:10CC500080911511909116110E94A1A880918511C3
:10CC60001091F710811106C01123B1F18091A80233
:10CC7000882391F16091891170918A1180918B11B3
:10CC800090918C11C0900F11D0901011E090111163
:10CC9000F09012116C0D7D1D8E1D9F1D0F94EA19D1
:10CCA0002AE037ED43E25CE30F94491AE091131157
:10CCB000F0911411309721F0608371838283938304
:10CCC000112329F0E091F810F091F9101995809155
:10CCD000851181110E944BA780918511882329F02D
:10CCE000E091F810F091F91019950F900F900F90B6
:10CCF0000F90DF91CF911F91FF90EF90DF90CF9039
:10CD00000895CF92DF92EF92FF921F93CF93DF931C
:10CD100000D01F92CDB7DEB78091891190918A1112
:10CD2000A0918B11B0918C11B7FF08C0109289119E
:10CD300010928A1110928B1110928C1180910B110C
:10CD400090910C11A0910D11B0910E11409189118B
:10CD500050918A1160918B1170918C1184179507F5
:10CD6000A607B70744F48093891190938A11A09382
:10CD70008B11B0938C118091A802882359F1609196
:10CD8000891170918A1180918B1190918C11C090B2
:10CD90000F11D0901011E0901111F09012116C0D44
:10CDA0007D1D8E1D9F1D0F94EA192AE037ED43E289
:10CDB0005CE30F94491A69837A838B839C83CE0149
:10CDC00001960E949F9CBC018091151190911611B3
:10CDD0000E94A1A8809185111091F710811106C0C1
:10CDE0001123B1F18091A802882391F160918911FA
:10CDF00070918A1180918B1190918C11C0900F11BC
:10CE0000D0901011E0901111F09012116C0D7D1D59
:10CE10008E1D9F1D0F94EA192AE037ED43E25CE373
:10CE20000F94491AE0911311F0911411309721F0E9
:10CE30006083718382839383112329F0E091F8103A
:10CE4000F091F91019958091851181110E944BA7DD
:10CE50000F900F900F900F90DF91CF911F91FF9047
:10CE6000EF90DF90CF9008950F931F93CF93809111
:10CE7000891190918A11A0918B11B0918C11B7FFFB
:10CE800008C01092891110928A1110928B11109281
:10CE90008C1180910B1190910C11A0910D11B091FA
:10CEA0000E114091891150918A1160918B117091EE
:10CEB0008C1184179507A607B70744F4809389114E
:10CEC00090938A11A0938B11B0938C118091A8023A
:10CED000882311F16091891170918A1180918B11D1
:10CEE00090918C1100910F1110911011209111113E
:10CEF00030911211600F711F821F931F0F94EA1956
:10CF00000F945B1FCB010E94739EBC018091151191
:10CF1000909116110E94A1A880918511C091F710DF
:10CF2000811106C0CC2381F18091A802882361F190
:10CF30006091891170918A1180918B1190918C115F
:10CF400000910F11109110112091111130911211B7
:10CF5000600F711F821F931F0F94EA19E091131144
:10CF6000F0911411309721F0608371838283938351
:10CF7000CC2329F0E091F810F091F91019958091E7
:10CF8000851181110E944BA780918511CF911F912E
:10CF90000F91089569DF882329F0E091F810F0914E
:10CFA000F9101994089560CF0E942CA9882329F0C4
:10CFB000E091F810F091F910199408950C942CA9AF
:10CFC000EC01E3E0F2E484918F010F5F1F4F8823AF
:10CFD00021F00E944159F801F6CFEAE1FAE184918B
:10CFE0008F010F5F1F4F882321F00E944159F801E4
:10CFF000F6CF0E94525C0F947B060E9408AD61E060
:10D00000CE010E942CA40E9445A70E941D5C84E0D2
:10D010007CD78091AE11869586951092E41180930D
:10D02000E5110E941B708091AE1186958695880F40
:10D030001092E4118093E5118BE09AE19BD78091E7
:10D04000AE1186958695982F990F980F1092E4113E
:10D050009093E5118EEF99E18DD70E949250811146
:10D06000D6CF2FEF8BE49DE1215080409040E1F737
:10D0700000C00000F8942FEF84E39CE02150804032
:10D080009040E1F700C000000E94525CA895FECFDE
:10D090006F927F928F929F92AF92BF92DF92EF92A8
:10D0A000FF920F931F93CF93DF93CDB7DEB7AD976A
:10D0B0000FB6F894DEBF0FBECDBF7C01D62E809197
:10D0C0005F12882309F4F7C180915314882309F46F
:10D0D0009DC0442309F4C4C180916B14882321F1BD
:10D0E000E3E0F2E484918F010F5F1F4F882321F06A
:10D0F0000E944159F801F6CFEDE9FBE184918F01DF
:10D100000F5F1F4F882321F00E944159F801F6CF8D
:10D1100061E070E080E090E00E94024D8AE00E94B1
:10D12000415984E99BE14CDF8FE280937014B12C6C
:10D1300021E001E714E19FE1A92E80912814B8169F
:10D14000B8F4AB9CC0011124B8018A509D4E2DA7A4
:10D150000E94D45BC8012DA58C010196F801308195
:10D16000332321F02D3810F42F5FF6CFB394E5CFA1
:10D1700027FD06C0B80180E594E10E94D45B02C09F
:10D18000F8011082EEE3F2E484918F010F5F1F4FEC
:10D19000882321F00E944159F801F6CFB7018BE7AF
:10D1A0009BE10E94A29B60916B14FDE86F9FB00110
:10D1B000112460597B4E80E79BE10E94A29B409125
:10D1C00001155091021560910315709104158AE6BE
:10D1D0009BE10E9467C18AE00E94415980916B14D3
:10D1E00094E0899FF0011124E459FB4E4091011510
:10D1F000509102156091031570910415408351837D
:10D20000628373838F5F80936B140DC010926B14D5
:10D2100082E0B82E27C1B7018DE59BE10E94A29B59
:10D220008AE00E9441590E942E901D8218861C821D
:10D230001B8280E293E09A83898382EB92E1909350
:10D24000D2128093D112F70180818F3209F06DC024
:10D2500087010F5F1F4FCE0101963C01011511059B
:10D2600009F469C06FE270E0C8010F944C215C01C1
:10D27000009709F461C00817190708F05DC04C0158
:10D28000801A910AA401B801CE0180960F946C21F6
:10D29000E0E2F0E0EC0FFD1FE80DF91D10828E01B9
:10D2A000005E1F4FF80181918F01882319F00E94C1
:10D2B0004159F8CF8AE00E9441596091D112709192
:10D2C000D2126115710519F06C5F7F4F02C060E0EA
:10D2D00070E021E0AE01405E5F4FCE0105960E94F6
:10D2E0002FAD81111AC0E9E4FBE184918F010F5F3A
:10D2F0001F4F811104C08E01005E1F4F04C00E94A9
:10D300004159F801F2CFF80181918F01882319F07A
:10D310000E944159F8CF8EE28CC07092D212609276
:10D32000D11285010F5F1F4F99CF83ED92E190934A
:10D33000D2128093D11287016091D1127091D212D2
:10D34000DD2009F45DC06115710519F06C5F7F4F38
:10D3500002C060E070E021E0A80180E594E10E9455
:10D360002FAD882309F448C0809161149091621414
:10D37000A0916314B09164148093FD149093FE14F3
:10D38000A093FF14B0930015B8018BE39BE10E94BA
:10D39000A29B4091FD145091FE146091FF14709176
:10D3A000001583E39BE10E9467C18AE00E94415916
:10D3B0001092011510920215109203151092041587
:10D3C000E4E2FBE184917F019FEFE91AF90A8823E7
:10D3D00021F00E944159F701F5CFB80180E090E0BB
:10D3E0000E94E9AF80916E12811102C0C80102C093
:10D3F0008EE692E160E02DC0B80180E19BE113C0B0
:10D400006115710519F06C5F7F4F02C060E070E03C
:10D4100026E5A80180E594E10E942FAD81110CC0A2
:10D42000B8018CEF9AE10E94A29B8EE20E944159C2
:10D430008AE00E9441590FC081E080935C12B701DD
:10D440008AEE9AE10E94A29B8AE00E94415960E024
:10D45000C8010E941CA4CE0101960E9485912BC098
:10D46000BB24B394EEE3F2E484918F010F5F1F4F6E
:10D47000882321F00E944159F801F6CFE5E6FBE14F
:10D4800084918F010F5F1F4F882321F00E94415923
:10D49000F801F6CFE1E0BE1203C006E313E002C0DC
:10D4A00000E313E0F80181918F01882309F4B3CEE2
:10D4B0000E944159F7CFAD960FB6F894DEBF0FBE6C
:10D4C000CDBFDF91CF911F910F91FF90EF90DF9033
:10D4D000BF90AF909F908F907F906F90089560E085
:10D4E0008091F40F9091F50F0E949D556093600616
:10D4F0007093610680936206909363068091F00FAB
:10D500009091F10F0E945B526093640670936506E0
:10D510008093660690936706A8958FB7F89410924B
:10D52000F60F8FBF0895CF92DF92FF920F931F9354
:10D53000CF93DF931F921F92CDB7DEB7F82E6A010B
:10D5400080915702882309F441C0E3E0F2E484911A
:10D550008F010F5F1F4F882341F069837A830E94F8
:10D560004159F80169817A81F2CFFB0184918F01E1
:10D570000F5F1F4F882321F00E944159F801F6CF19
:10D58000EFE3FAE184918F010F5F1F4F882321F0B1
:10D590000E944159F801F6CFF7FC0CC06F2D772798
:10D5A00067FD7095872F972F0E94024D8AE00E9499
:10D5B00041590CC0EAE3FAE184918F010F5F1F4FDC
:10D5C000882321F00E944159F801F6CF8091D206BC
:10D5D000811107C01092570281E08093D206C601E4
:10D5E000EFDC0F900F90DF91CF911F910F91FF9083
:10D5F000DF90CF900C94525C2F923F924F925F92AB
:10D600006F927F928F929F92AF92BF92CF92DF9252
:10D61000EF92FF920F931F93CF93DF9300D01F924F
:10D62000CDB7DEB74C011B0129833A834B835C8362
:10D6300027013801D7FE12C080918406882309F49F
:10D64000A7C0F40110821092D7061092D80610924B
:10D65000D9061092DA0601E010E015C0F601EE5886
:10D66000F94F8081882309F4BEC0F4011082F601CD
:10D67000EE0FFF1FEE0FFF1FED52F94F10821182C8
:10D68000128213828601F40180818230E1F08330BE
:10D6900009F455C0813009F0A8C0F801EE0FFF1F52
:10D6A000EE0FFF1FED52F94F2081318142815381EE
:10D6B00069817A818B819C810F94E41987FD95C0E3
:10D6C00082E0F4018083000F111F000F111F0D5223
:10D6D000194FB501882777FD8095982F0F94EA1987
:10D6E0009B01AC01F80160817181828193810F946B
:10D6F000161E9B01AC0169817A818B819C810F94FC
:10D700003D2087FD0CC00F941C0A6856754C8F4F46
:10D710009F4FF101608371838283938366C00F946E
:10D720001C0AF1010081118122813381601B710B80
:10D73000820B930B97FD59C083E0F4018083FFEFC8
:10D74000CF16DF0631F0C114D10431F444E95AE1B7
:10D7500005C04DE55AE102C041E85AE161E77AE1CE
:10D760008C2D0F900F900F900F90DF91CF911F9104
:10D770000F91FF90EF90DF90CF90BF90AF909F9070
:10D780008F907F906F905F904F903F902F90CBCE77
:10D7900001E010E07801EE0CFF1CEE0CFF1CC7014D
:10D7A0008D52994F7C01A3019201FC01608171812E
:10D7B000828193810F94E419882309F464CFF701DF
:10D7C0004082518262827382FF24F39420E030E031
:10D7D000A901C301B2010F943D2018160CF0F12CE1
:10D7E000F401F08250CF8601D5CF0F900F900F90AB
:10D7F0000F90DF91CF911F910F91FF90EF90DF90ED
:10D80000CF90BF90AF909F908F907F906F905F90E0
:10D810004F903F902F9008958F3F29F0811106C0BF
:10D8200045E95CE405C042E65CE402C045E85CE42E
:10D8300063E77CE478CE8F3F29F0811106C048ED84
:10D840005CE405C045EA5CE402C048EC5CE466EBDD
:10D850007CE469CE4F925F926F927F92AF92BF92BB
:10D86000CF92DF92EF92FF920F931F93CF93DF93AC
:10D8700000D01F92CDB7DEB78091F60F811113C093
:10D880000F900F900F900F90DF91CF911F910F91FC
:10D89000FF90EF90DF90CF90BF90AF907F906F9010
:10D8A0005F904F9008951BDE0F941C0A69837A8362
:10D8B0008B839C8380915C0290915D0218161906FF
:10D8C0000CF026C1019790935D0280935C0240901A
:10D8D00060065090610660906206709063068091C9
:10D8E0007206811119C080916E0690916F06A09109
:10D8F0007006B09171060097A105B10569F0298104
:10D900003A814B815C81281B390B4A0B5B0B57FD1D
:10D9100003C081E0809372066091F20F7091F30F63
:10D92000882777FD8095982F0F94EA191EE1A12E84
:10D93000B12CC12CD12C7B018C01A30192016DEE85
:10D9400076E08CEE96E058DE4090600650906106DE
:10D950006090620670906306609167077091680737
:10D96000882777FD8095982F0F94EA199B01AC01C9
:10D97000C301B2010F943D201816D4F460916802DF
:10D9800070916902882777FD8095982F0F94EA1986
:10D990009B01AC01C301B2010F94E41987FF08C0D9
:10D9A00080E00E9438540F945B1F7595679501C005
:10D9B00060E0609308108091E8069091E906A091DC
:10D9C000EA06B091EB060097A105B10521F1298186
:10D9D0003A814B815C81281B390B4A0B5B0B57FD4D
:10D9E0001AC00E943D562B013C016091E6067091E1
:10D9F000E70680E090E00F94E8199B01AC01C301B9
:10DA0000B2010F94E41987FFA5C048ED5AE169EC13
:10DA10007AE180E088DD8091E2069091E306A091B2
:10DA2000E406B091E5060097A105B10521F1298131
:10DA30003A814B815C81281B390B4A0B5B0B57FDEC
:10DA40001AC00E9494552B013C016091E006709130
:10DA5000E10680E090E00F94E8199B01AC01C3015E
:10DA6000B2010F94E41987FF72C047EA5AE16AEBEA
:10DA70007AE18FEF58DD6091EE0F7091EF0F8827FC
:10DA800077FD8095982F0F94EA19209164063091C4
:10DA900065064091660650916706FAE0AF2EB12CFC
:10DAA000CC24CA94DC2C7B018C016BED76E08FEDED
:10DAB00096E0A2DD80918406811127C04090640623
:10DAC00050906506609066067090670620E030E032
:10DAD00040EA50E4C301B2010F943D2087FF04C027
:10DAE00060E060930610CCCE20E030E046E153E4E5
:10DAF000C301B2010F94E419181694F30E94FB526B
:10DB00000F945B1F75956795ECCF10920610B8CEF9
:10DB100040906006509061066090620670906306C7
:10DB200020E030E848E953E4C301B2010F943D20FE
:10DB30001816A4F020E030E040EA50E4C301B2013E
:10DB40000F94E41987FFCBCE80E066DEC0CE0E9442
:10DB5000C75191CF80E00E9411525DCF80E06BDE13
:10DB60004090600650906106609062067090630677
:10DB7000E1CF0F931F93CF93DF93EC018B01609163
:10DB80003D1240913E12641306C081E392E10E946F
:10DB90007F5B60DEF4CF28813981F801808191813B
:10DBA00050913C1274E0579FF0011124EB5CFD4E44
:10DBB00033872287958784876F5F60933D1281E06A
:10DBC000850F841719F080933C1202C010923C120A
:10DBD000DF91CF911F910F9108950F931F93CF93D2
:10DBE000DF93CDB7DEB728970FB6F894DEBF0FBE30
:10DBF000CDBF8823C1F083E992E098878F8304E644
:10DC000010E01A830983BE01695F7F4FCE01019640
:10DC1000B0DF8AEB92E09E838D831A830983BE0175
:10DC20006B5F7F4F0BC088EB91E09C838B8384E11B
:10DC300090E09A838983BE016D5F7F4FCE0101968C
:10DC400098DF28960FB6F894DEBF0FBECDBFDF91E8
:10DC5000CF911F910F9108950E9484C1BECFAF92C2
:10DC6000BF92CF92DF92FF920F931F93CF93DF93D8
:10DC700000D01F92CDB7DEB7F82E662351F0109278
:10DC8000F5061092F1061092F2061092F306109229
:10DC9000F4060F941C0A0091F1061091F2062091EF
:10DCA000F3063091F4065B016C01A01AB10AC20AB6
:10DCB000D30AD7FC3DC0F7FE05C004EC19E020E014
:10DCC00030E015C0E091F5062F2D332727FD309564
:10DCD0002C5F3F4F4E2F552747FD50952417350792
:10DCE0003CF1EF1554F300E911E020E030E0DC01F5
:10DCF000CB01800F911FA21FB31F8093F106909359
:10DD0000F206A093F306B093F40680ED97E09C83AF
:10DD10008B838CE291E09A838983BE016D5F7F4F94
:10DD2000CE01019626DF8091F5068F5F8093F50680
:10DD30000F900F900F900F90DF91CF911F910F9147
:10DD4000FF90DF90CF90BF90AF900895CF92DF9279
:10DD5000EF92FF926B017C0183E3C816D104E104CA
:10DD6000F10468F082E3C81AD108E108F10862E31F
:10DD700070E080E090E00F9489096CDDEDCFC70181
:10DD8000B6010F948909FF90EF90DF90CF9062CD9C
:10DD9000EF92FF920F931F93CF93DF93EC018901D2
:10DDA0008C81833039F089E0440F551F661F771F3F
:10DDB0008A95D1F79A01AB0161E1CE010E94D0585A
:10DDC000882331F084E08983CE010E94A55841C0A8
:10DDD0000F941C0A7B010E94AF588B838F3F49F43C
:10DDE0000F941C0A6E197F096D327140A0F381E116
:10DDF00003C08E3F49F08FE08983CE010E94A55871
:10DE00008FEF0E94AA5825C08FEF8EBDF80180E0E9
:10DE100090E02FEF0DB407FEFDCF3EB531932EBD40
:10DE200001968F3F31E09307A9F70DB407FEFDCFB0
:10DE30008EB5F801E150FE4F80830E94AF580E94DA
:10DE4000AF58CE010E94A5588FEF0E94AA5881E0DA
:10DE500001C080E0DF91CF911F910F91FF90EF9073
:10DE600008952091B1113091B2112817390709F4A2
:10DE700044C09093B2118093B111009709F437C058
:10DE80002091C411FC01211107C03596E491E09363
:10DE9000C511FC013C960FC0213039F43F96E49146
:10DEA000E093C511FC01709606C03D96E491E093A5
:10DEB000C511FC013E9684918093C6118091C511D5
:10DEC000992787FD90952091C611821B910927FD06
:10DED00093952091C711203441F0829FC0011124F5
:10DEE00026E0969587952A95E1F78093C8118CEEE8
:10DEF00090E09093C3118093C211089580E29CE159
:10DF0000B0DF81E080938D060895CF93C82F8230D3
:10DF100051F020F4813079F4CF91F0CF833031F09B
:10DF2000843021F008C08AE296E002C086EB96E0D9
:10DF300098DFC0938D06CF910895E091A911F091DB
:10DF4000AA110190F081E02D682F89EA91E11994DE
:10DF5000CF93C82F8FEF8C0F893048F48AE296E078
:10DF600080DF8C2FEADF80918D06CF91CECF8C2F72
:10DF7000CF91E3CFCF93DF93EC01FE01849188230F
:10DF800019F0E6DF2196F9CFDF91CF910895CF9375
:10DF9000DF93EC018991882311F0DADFFBCFDF9169
:10DFA000CF9108959CE0899F802D112441E0480F76
:10DFB0004093DB10845F8093DC106091E11170E08E
:10DFC000282F30E02E5F3F4F261737079CF150E097
:10DFD0002091E31130E04217530764F59EE39093DC
:10DFE000E4118093E51185E4B3DF809175068F5CC1
:10DFF000AFDF80E2ADDF60916006709161068091D5
:10E000006206909163060F945B1FCB010E94739E82
:10E01000BEDF8FE29DDF0E9449A4811104C0809180
:10E020007206811107C08091F20F9091F30F0E9448
:10E03000739EADCF0895CF93DF93C0E1D2E0899175
:10E04000882329F07ADF82E0C632D807C1F7DF9152
:10E05000CF9108950F931F93CF93DF93EC01890124
:10E060008C81833039F039E0440F551F661F771FCC
:10E070003A95D1F79A01AB0168E1CE010E94D058E0
:10E08000882311F086E034C08EEF8EBD80E090E0F2
:10E090000DB407FEFDCFF801E80FF91F20812EBD5A
:10E0A0000DB407FEFDCF21812EBD0296811522E021
:10E0B000920771F70DB407FEFDCF8FEF0E94AA58AB
:10E0C0008FEF0E94AA580E94AF588B838F718530C2
:10E0D00031F083E18983CE010E94A5580AC068E52A
:10E0E00072E0CE010E94B658182F811107C087E157
:10E0F0008983CE010E94A55810E012C020E030E0D4
:10E10000A9016DE0CE010E94D058811104C00E9487
:10E11000AF58882311F086E1EBCFCE010E94A558BD
:10E12000812FDF91CF911F910F910895CF9380910F
:10E1300015078823A9F140911607509117076091A0
:10E1400018077091190727E534E080911307909123
:10E15000140780DFC82F882321F14091F6065091E3
:10E16000F7066091F8067091F906411551056105B1
:10E17000710589F027E534E0809113079091140729
:10E1800069DF882359F01092F6061092F706109274
:10E19000F8061092F906109215078C2FC82F01C0AF
:10E1A000C1E08C2FCF910895CF92DF92EF92FF9232
:10E1B000CF936B017C01C42F8091160790911707B4
:10E1C000A0911807B09119078C159D05AE05BF05E4
:10E1D000C1F0ACDF811102C080E017C027E534E058
:10E1E000B701A6018091130790911407D1DD882310
:10E1F00099F3C0921607D0921707E0921807F09291
:10E20000190781E0C11180931507CF91FF90EF901E
:10E21000DF90CF9008958F929F92AF92BF92CF924E
:10E22000DF92EF92FF921F93CF93DF93C82F29E2E3
:10E2300034E130931407209313071092451442E001
:10E2400050E060E070E040932E1450932F146093E0
:10E25000301470933114109215071092F606109234
:10E26000F7061092F8061092F9064FEF5FEFBA0129
:10E270004093160750931707609318077093190778
:10E28000882349F1853008F0F6C040E060E070E096
:10E29000CB018ADF882309F4EEC020E1C29FF001A0
:10E2A0001124EB5FF94F80818F7709F0E4C044853A
:10E2B000558566857785443651056105710508F4F5
:10E2C000DAC0C084D184E284F384C114D104E104AF
:10E2D000F10421F4D0C0C12CD12C760140E0C7015B
:10E2E000B60162DF182F882309F4C5C0809162044B
:10E2F000909163048115924009F0BDC0A09167041C
:10E30000AA2309F4B8C0809165049091660400972F
:10E3100009F4B1C040916404442309F4ACC0A09353
:10E32000401440933214E0E050E061E070E0CE2F02
:10E330009B010E2E02C0220F331F0A94E2F74217F0
:10E34000530749F021E02E0FE83018F020933B14DA
:10E3500092C0E22FECCFE0933B1420916D043091FA
:10E360006E042115310519F040E050E008C02091FD
:10E370007B0430917C0440917D0450917E04209375
:10E3800033143093341440933514509336144601AB
:10E390005701880E991EA11CB11C809241149092C5
:10E3A0004214A0924314B0924414E0916804F09196
:10E3B0006904F0934714E0934614B0E00F94F71DFE
:10E3C000680D791D8A1D9B1D609348147093491434
:10E3D00080934A1490934B1445E0EE0FFF1F4A952B
:10E3E000E1F7E150FE4FEF2FFF27E695DC01CB016F
:10E3F0008E0F9F1FA11DB11D80933C1490933D145F
:10E40000A0933E14B0933F1480906A0490906B04E4
:10E410008114910419F0A12CB12C08C080907704CC
:10E4200090907804A0907904B0907A04A7019601A6
:10E43000281B390B4A0B5B0BDA01C901880D991DAA
:10E44000AA1DBB1D0C2E04C0B695A7959795879560
:10E450000A94D2F78093371490933814A093391408
:10E46000B0933A14853F4FE09407A105B10528F415
:10E470008CE08093451410E01AC0853F9F4FA105A2
:10E48000B10510F480E111C080918304909184045F
:10E49000A0918504B0918604809348149093491408
:10E4A000A0934A14B0934B1480E280934514812FBB
:10E4B000DF91CF911F91FF90EF90DF90CF90BF90B1
:10E4C000AF909F908F9008958F929F92AF92BF923E
:10E4D000CF92DF92EF92FF920F931F93CF93DF9330
:10E4E000EC016A017B01890189859A85AB85BC8530
:10E4F0000196A11DB11D84179507A607B70710F453
:10E5000080E054C08F89803129F49927872F762F96
:10E51000652F0BC08032A1F7CB01BA01E7E09695D9
:10E52000879577956795EA95D1F78B889C88AD8814
:10E53000BE88680D791D8A1D9B1D809016079090DE
:10E540001707A0901807B0901907681579058A0574
:10E550009B0581F48F89803191F4DD24EE24FF2422
:10E56000F601EE0FFF1FE95AFB4F80819181A0E079
:10E57000B0E016C040E018DE8111ECCFC1CFE894C6
:10E58000C7F8DD24EE24FF24F601EE0FFF1FEE0F87
:10E59000FF1FE95AFB4F80819181A281B381BF7037
:10E5A000F80180839183A283B38381E0DF91CF91CF
:10E5B0001F910F91FF90EF90DF90CF90BF90AF90A1
:10E5C0009F908F9008952F923F924F925F926F92FB
:10E5D0007F928F929F92AF92BF92CF92DF92EF92F3
:10E5E000FF920F931F93CF93DF93EC015B016A01BE
:10E5F0008B81811103C08FEF9FEFC6C0898180FF9F
:10E60000FACF49895A896B897C8988859985AA8539
:10E61000BB852601612C712C8A019B01081B190BFB
:10E620002A0B3B0B041515052605370518F46A015E
:10E63000C81AD90A76013E0124E0620E711CE11469
:10E64000F10409F476C0488559856A857B854A01BD
:10E6500081E098222B811A012B01A9E0569447945E
:10E6600037942794AA95D1F7898D9A8DFC01223091
:10E6700049F4628D738D848D958D620D731D841D9B
:10E68000951D3CC014811150122181149104C1F4D4
:10E69000111116C0452B462B472B49F48D899E89B5
:10E6A000AF89B88D8C839D83AE83BF8309C04C81B5
:10E6B0005D816E817F81930107DF882309F49BCF01
:10E6C000E98DFA8D6C817D818E819F816250710907
:10E6D00081099109058404C0660F771F881F991F5F
:10E6E0000A94D2F72685378540895189620F731FB6
:10E6F000841F951F610F711D811D911D20E032E067
:10E700002819390987012E153F0508F489010115DB
:10E71000F2E01F0761F5209116073091170740912D
:10E72000180750911907621773078407950719F4A2
:10E730001EC0C60129C09501AB01BC018091130721
:10E740009091140725DB882309F455CFA00EB11E44
:10E7500088859985AA85BB85800F911FA11DB11D54
:10E7600088879987AA87BB87E01AF10A68CF40E0BB
:10E770001BDD882309F43FCFB401695A7B4FA80100
:10E78000C5010F942521E2CFDF91CF911F910F9109
:10E79000FF90EF90DF90CF90BF90AF909F908F90C1
:10E7A0007F906F905F904F903F902F900895AF9221
:10E7B000BF92CF92DF92EF92FF920F931F93CF936E
:10E7C000DF936C01EB017A01DC0113968C911397B6
:10E7D000823070F018960D911D912D913C911B97F0
:10E7E0000F71112722273327012B022B032B11F046
:10E7F0008FEF58C04115510511F0F70110821DE04F
:10E8000040E250E0BE01C601DEDE9C01803291058F
:10E8100031F081E0232B09F480E0819543C08881A9
:10E820008823C1F1853E61F38E3251F3E114F10486
:10E8300061F19B859F739F3041F54A8D5B8D452B20
:10E8400021F58F719FEF980F9530F8F490E00197C4
:10E85000189F9001199F300D1124FE0180E090E077
:10E860005701A20EB31E8530B8F46181A501480F8F
:10E87000591FDA016C93019632968D30910599F704
:10E88000888186FF02C0F50115868B8583FDB8CF90
:10E89000822F08C080E006C08B3010F46481E6CF80
:10E8A0006681E4CFDF91CF911F910F91FF90EF90A0
:10E8B000DF90CF90BF90AF9008954F925F926F928C
:10E8C0007F92AF92BF92CF92DF92EF92FF920F931F
:10E8D0001F93CF93DF93EC016A017B012B812223ED
:10E8E00049F089899A89AB89BC8984179507A6075D
:10E8F000B70710F480E06BC0223009F463C0C11484
:10E90000D104E104F10449F41C821D821E821F829D
:10E91000188619861A861B8659C088859985AA8506
:10E92000BB85E98DFA8DE585F0E03996AC01BD0136
:10E9300041505109610971090E2E04C07695679501
:10E94000579547950A94D2F797018601015011090E
:10E950002109310904C03695279517950795EA9541
:10E96000D2F7041715072607370720F0892B8A2BC3
:10E970008B2B49F48D899E89AF89B88D8C839D83BB
:10E98000AE83BF8304C0041B150B260B370B280175
:10E9900039015E0184E0A80EB11C411451046104E8
:10E9A000710481F04C815D816E817F819501898D3B
:10E9B0009A8D8ADD91E0491A510861087108811128
:10E9C000ECCF05C0C886D986EA86FB8681E0DF9158
:10E9D000CF911F910F91FF90EF90DF90CF90BF905C
:10E9E000AF907F906F905F904F9008954F925F929D
:10E9F0006F927F92AF92BF92CF92DF92EF92FF928F
:10EA00000F931F93CF93DF9300D01F92CDB7DEB744
:10EA10008C0149835A836B837C835901C12CD12C8F
:10EA20007601412CB2E05B2E612C712C49815A8118
:10EA30006B817C819E012F5F3F4FC80145DD88239C
:10EA400041F1D301C201F801058404C0880F991F68
:10EA5000AA1FBB1F0A94D2F7C80ED91EEA1EFB1EBE
:10EA600049815A816B817C818789803139F481E0C9
:10EA7000483F5F4F6105710538F4D8CF81E0483FCA
:10EA80005F4F6F4F7F4090F2F501C082D182E282EA
:10EA9000F3820F900F900F900F90DF91CF911F9105
:10EAA0000F91FF90EF90DF90CF90BF90AF907F904D
:10EAB0006F905F904F9008950F931F93CF93DF93C4
:10EAC000EC018B018B81882311F080E041C0FB01B8
:10EAD0008789803131F18032C1F783E08B83F8017F
:10EAE000428D538D648D758D4D8B5E8B6F8B788FC2
:10EAF0009E012F5E3F4FC80179DF882331F31A8FC3
:10EB0000098F81E089831C821D821E821F821886E4
:10EB100019861A861B861C861D861E861F86188AE5
:10EB200017C082E08B831D8A1E8A1F8A188EFB0104
:10EB3000408D518D60E070E085E0440F551F661FE9
:10EB4000771F8A95D1F7498B5A8B6B8B7C8BD7CFEC
:10EB5000DF91CF911F910F9108954F925F926F9225
:10EB60007F928F929F92AF92BF92CF92DF92EF925D
:10EB7000FF920F931F93CF93DF93EC014A015B0148
:10EB800028013901423051056105710508F462C060
:10EB900049855A856B857C854F5F5F4F6F4F7F4FEF
:10EBA000481559056A057B0508F454C08F898031E2
:10EBB00029F4FF24EB2CDA2CC92C0CC0803209F08C
:10EBC00049C07501640137E0F694E794D794C7947F
:10EBD0003A95D1F74B895C896D897E89C40ED51E23
:10EBE000E61EF71E41E0C701B601DEDA882391F187
:10EBF0009F89903159F49924AA24BB24F401EE0F83
:10EC0000FF1FE95AFB4F5182408210C0E89487F8F9
:10EC10009924AA24BB24F401EE0FFF1FEE0FFF1F5F
:10EC2000E95AFB4F40825182628273829A89923004
:10EC300090F04D815E816F8178854C0D5D1D6E1D5C
:10EC40007F1D4093F6065093F7066093F806709385
:10EC5000F90601C080E0DF91CF911F910F91FF90E5
:10EC6000EF90DF90CF90BF90AF909F908F907F906C
:10EC70006F905F904F900895AF92BF92CF92DF92C6
:10EC8000EF92FF920F931F93CF93DF9300D01F92C9
:10EC9000CDB7DEB75C016A017B0182E090E0A0E0C5
:10ECA000B0E0F50180839183A283B3839E012F5F3F
:10ECB0003F4FB701A601C50107DC811102C080E00A
:10ECC00023C000E010E09801B701A601C50145DFAF
:10ECD0008823A9F3C980DA80EB80FC80F50187895D
:10ECE000803149F481E0F8EFCF16FFEFDF06E10451
:10ECF000F10450F4DBCF81E098EFC9169FEFD906FD
:10ED0000E9069FE0F90690F20F900F900F900F9098
:10ED1000DF91CF911F910F91FF90EF90DF90CF90F7
:10ED2000BF90AF900895CF93DF93CDB7DEB78091BA
:10ED30007406811110C09E01275F3F4F4F81588597
:10ED400062E470E080E192E00F94AC190E94FDA3B0
:10ED500083E08093A802DF91CF910895FF920F93F3
:10ED60001F93CF93DF93C091A31181E0C827D09167
:10ED7000A411D827F090A511F826C11102C0DD23F7
:10ED800019F0EEE3F2E404C0F110FBCF80E077C0AD
:10ED900084918F010F5F1F4F882321F00E944159FA
:10EDA000F801F6CFEAE1FCE184918F010F5F1F4F7C
:10EDB000882321F00E944159F801F6CFCC2361F05D
:10EDC000E8E1FCE184918F010F5F1F4F882321F060
:10EDD0000E944159F801F6CFDD2361F0E6E1FCE144
:10EDE00084918F010F5F1F4F882321F00E944159AA
:10EDF000F801F6CFF11003C0ECE0FCE10CC0E4E157
:10EE0000FCE184918F010F5F1F4F8823A9F30E94BB
:10EE10004159F801F6CF84918F010F5F1F4F88236E
:10EE200021F00E944159F801F6CFFF2019F04CE380
:10EE300053E002C04CEB53E0DD2319F02EE333E046
:10EE400002C02CEB33E0CC2319F080E493E002C045
:10EE50008CEB93E05F934F933F932F939F938F930C
:10EE60008AEF9BE19F938F931F925DDF8DB79EB7D3
:10EE700009960FB6F8949EBF0FBE8DBF81E0DF915B
:10EE8000CF911F910F91FF90089580914F12815063
:10EE9000823010F080E0089510924F120F941C0AF7
:10EEA000609358127093591280935A1290935B1288
:10EEB00081E008950F931F9380914F12813019F4D0
:10EEC0000F941C0A08C060915812709159128091D9
:10EED0005A1290915B120091541210915512209188
:10EEE000561230915712601B710B820B930B28EE58
:10EEF00033E040E050E00F94B91D809150129091A2
:10EF00005112A0915212B0915312280F391F4A1F6B
:10EF10005B1FCA01B9011F910F91089580914F1293
:10EF2000813099F1823051F4C5DF609350127093B3
:10EF30005112809352129093531218C0109254128F
:10EF40001092551210925612109257121092581297
:10EF50001092591210925A1210925B121092501283
:10EF600010925112109252121092531281E080931B
:10EF70004F120F941C0A6093541270935512809391
:10EF800056129093571281E0089580E00895CF9231
:10EF9000DF92EF92FF92C0908807D0908907E090AF
:10EFA0008A07F0908B07209106113091071140914C
:10EFB000081150910911C701B6010F94491A0F9415
:10EFC000482060932B1270932C1280932D129093F3
:10EFD0002E12C701B6010F945B1F2FB7F8946093F0
:10EFE000B90F7093BA0F8093BB0F9093BC0F2FBFD4
:10EFF00010921B1210921C1210921D1210921E12CF
:10F00000FF90EF90DF90CF90089580914F12813064
:10F0100079F482E080934F120F941C0A6093581287
:10F020007093591280935A1290935B1281E0089565
:10F0300080E00895E82FF0E0ED5CFC4E849190E0D4
:10F04000FC013797EC30F105F8F4EC57FF4F0D94C5
:10F0500006218091B100887F84608093B10008957B
:10F0600080919100887F84608093910008958091C1
:10F07000A100887F84608093A10008958091210180
:10F08000887F84608093210108958F929F92AF9230
:10F09000BF92CF92DF92EF92FF920F931F93CF9385
:10F0A000DF931F921F92CDB7DEB77C01490180919B
:10F0B0004411811148C08B015B01A40EB51E0A15D5
:10F0C0001B0509F440C0F701C080D180F8016191AF
:10F0D0008F016983C6016A830F949A1C6A8168173D
:10F0E00029F1C6010F94A21CC6010F949A1C9981A4
:10F0F0008917E1F0EEE3F2E484918F010F5F1F4F77
:10F10000882321F00E944159F801F6CFE0EEFBE19F
:10F1100084918F010F5F1F4F882321F00E94415976
:10F12000F801F6CF81E0809344110DC0BE016F5FFE
:10F130007F4FC4010E94D89AF70180819181019686
:10F1400091838083BCCF0F900F90DF91CF911F915F
:10F150000F91FF90EF90DF90CF90BF90AF909F9076
:10F160008F9008952F923F924F925F926F927F926D
:10F170008F929F92AF92BF92CF92DF92EF92FF92C7
:10F180000F931F93CF93DF93CDB7DEB76B970FB677
:10F19000F894DEBF0FBECDBF9F8B8E8B1B01488FB7
:10F1A000298FFC016081718182819381698B7A8BC7
:10F1B0008B8B9C8BF101C080D180E280F380CD8667
:10F1C000DE86EF86F88A40904B0450904C046090A5
:10F1D0004D0470904E0420914704309148044091B2
:10F1E000490450914A040F94161E4B015C012CE017
:10F1F00032E040EA51EC0F943D2087FD24C021E22B
:10F2000030E041E953E4C501B4010F94E419181644
:10F21000D4F0A3019201C701B6010F94161E6B0131
:10F220007C012CE032E040EA51EC0F943D2087FD58
:10F230000AC021E230E847E953E4C701B6010F9460
:10F24000E41918162CF4612C712C00EC1FE74AC34A
:10F25000C0900C02D0900D02E0900E02F0900F02D0
:10F260008091FF06811107C080915E028093FE06A7
:10F2700081E08093FF0680915F0290916002A091EF
:10F280006102B091620280930C0290930D02A093F0
:10F290000E02B0930F020E94B1EA19821A821B82F9
:10F2A0001C82AE014F5F5F4FBE01635F7F4FCE0197
:10F2B00041960E949DE881E00E940BEB811197C26C
:10F2C0000F94280A04E010E0812C912CA12CE1E499
:10F2D000BE2E412C512CF0E26F2EF1E47F2E60E027
:10F2E00070E080EF93E40E9450EB882309F401C1A1
:10F2F000015011090115110509F0C1C0EDE8F5E251
:10F3000084918F010F5F1F4F882321F00E94415984
:10F31000F801F6CF60E08EE795E20E942CA450E75A
:10F32000C52E53E0D52EDE82CD8269E1E62EF12C8A
:10F33000FA82E982BE016B5F7F4FCE0101960E9487
:10F34000B96D1E821D8202E310E01A830983BE019B
:10F350006B5F7F4FCE0101960E94B96DDE82CD8238
:10F36000FA82E982BE016B5F7F4FCE0101960E9457
:10F37000B96D1E821D821A830983BE016B5F7F4FA8
:10F38000CE0101960E94B96DDE82CD82FA82E982B9
:10F39000BE016B5F7F4FCE0101960E94B96D1E8248
:10F3A0001D821A830983BE016B5F7F4FCE010196D8
:10F3B0000E94B96D80E090E0A0E0B1E48D839E836F
:10F3C000AF83B88780E090E0A8ECB2E489839A83A9
:10F3D000AB83BC83BE016B5F7F4FCE0101960E9461
:10F3E000A1E8109288071092890710928A0710925C
:10F3F0008B07C09075068091840790918507A09136
:10F400008607B091870740918007509181076091EE
:10F4100082077091830700917C0710917D072091EE
:10F420007E0730917F0709831A832B833C834D83AA
:10F430005E836F83788789879A87AB87BC87AE01A5
:10F44000475F5F4FBE016B5F7F4FCE0101960E9409
:10F45000D5A2E12CF12C00EA1FE328E837E0AE0149
:10F46000475F5F4FBE016B5F7F4FCE0101960E94E9
:10F470003ECF8DDD0E947EFB8FE695E21EC1E6EA5F
:10F48000F5E284919F012F5F3F4F882341F02A8F3F
:10F490003B8F0E9441592A8D3B8DF901F2CF60E0EC
:10F4A00086E695E20E942CA48D829E82AF82B88669
:10F4B00049825A826B827C82BE016B5F7F4FCE0194
:10F4C00001960E94A1E81D8A19821A821B821C8261
:10F4D000FCE0F9871D829E012B5E3F4FAE014F5F1E
:10F4E0005F4FBE01675F7F4FCE0105960E94A8E87F
:10F4F000F6CE80E090E0A0E0B1E48D839E83AF8300
:10F50000B88720E030E040EA50E4609184077091D1
:10F51000850780918607909187070F94171E69834E
:10F520007A838B839C83BE016B5F7F4FCE010196F4
:10F530000E94A1E804E010E0812C912C30E8A32E79
:10F540003FE3B32E412C512C40E2642E41E4742E53
:10F55000DFC060E084E395E20E942CA480E7C82E1F
:10F5600083E0D82EDE82CD8299E1E92EF12CFA8259
:10F57000E982BE016B5F7F4FCE0101960E94B96D9B
:10F580001E821D8202E310E01A830983BE016B5FB5
:10F590007F4FCE0101960E94B96DDE82CD82FA8244
:10F5A000E982BE016B5F7F4FCE0101960E94B96D6B
:10F5B0001E821D821A830983BE016B5F7F4FCE01BD
:10F5C00001960E94B96DDE82CD82FA82E982BE0187
:10F5D0006B5F7F4FCE0101960E94B96D1E821D8226
:10F5E0001A830983BE016B5F7F4FCE0101960E9493
:10F5F000B96D80E090E0A0E0B1E48D839E83AF839D
:10F60000B88780E090E0A8ECB2E489839A83AB836A
:10F61000BC83BE016B5F7F4FCE0101960E94A1E8C3
:10F62000109288071092890710928A0710928B0710
:10F63000C09075068091840790918507A0918607F8
:10F64000B0918707409180075091810760918207B0
:10F650007091830700917C0710917D0720917E07B0
:10F6600030917F0709831A832B833C834D835E830C
:10F670006F83788789879A87AB87BC87AE01475F9E
:10F680005F4FBE016B5F7F4FCE0101960E94D5A2F6
:10F69000E12CF12C00EA1FE328E837E0AE01475FD8
:10F6A0005F4FBE016B5F7F4FCE0101960E943ECF40
:10F6B0006EDC0E947EFB85E295E20E94E06760E0DE
:10F6C0008CE195E20E942CA48D829E82AF82B88646
:10F6D00049825A826B827C82BE016B5F7F4FCE0172
:10F6E00001960E94A1E81D8A19821A821B821C823F
:10F6F0008CE089871D829E012B5E3F4FAE014F5FDC
:10F700005F4FBE01675F7F4FCE0105960E94A8E85C
:10F7100060E070E080E792E40E9450EB882319F1EA
:10F72000015011090115110569F4E3E4F5E2849132
:10F730008F010F5F1F4F882309F40BCF0E9441599F
:10F74000F801F5CFECE5F5E284919F012F5F3F4F83
:10F75000882309F4B4CF2A8F3B8F0E9441592A8D08
:10F760003B8DF901F1CF8090840790908507A090A0
:10F770008607B090870720914F0430915004409144
:10F78000510450915204C501B4010F94161E2091EA
:10F79000FA063091FB064091FC065091FD060F944D
:10F7A000171E3B018C01988D91111CC080E090E0E8
:10F7B000A0E0B1E489839A83AB83BC8320E030E08E
:10F7C00040EA50E4C501B4010F94171E6D837E8397
:10F7D0008F839887BE016F5F7F4FCE0105960E9491
:10F7E000A1E809C080E00E940BEB882321F0612C86
:10F7F000712C00EC1FE78091FE0680935E02E98D7C
:10F80000E33008F440C0E9EDF5E284915F019FEF39
:10F81000A91AB90A882321F00E944159F501F5CFB0
:10F82000EE89FF89608171818281938143E00E942A
:10F830001D4DE4EDF5E284915F019FEFA91AB90A2D
:10F84000882321F00E944159F501F5CFF101608133
:10F8500071818281938143E00E941D4DEFECF5E2BE
:10F8600084915F019FEFA91AB90A882321F00E94B1
:10F870004159F501F5CF43E0B301C8010E941D4D88
:10F880008AE00E944159C0920C02D0920D02E0928F
:10F890000E02F0920F029301A801B301C8010F9468
:10F8A000C3208823F9F060E080EC95E20E942CA44C
:10F8B000E3E0F2E484917F019FEFE91AF90A8823DB
:10F8C00021F00E944159F701F5CFE0EBF5E2849178
:10F8D0007F019FEFE91AF90A882321F00E9441591C
:10F8E000F701F5CFB301C8016B960FB6F894DEBFF0
:10F8F0000FBECDBFDF91CF911F910F91FF90EF9081
:10F90000DF90CF90BF90AF909F908F907F906F903F
:10F910005F904F903F902F9008952F923F924F927B
:10F920005F926F927F928F929F92AF92BF92CF928F
:10F93000DF92EF92FF920F931F93CF93DF93CDB798
:10F94000DEB7CF5FD1090FB6F894DEBF0FBECDBFD3
:10F9500005DA81110C94088BFE0131968CE3DF01EE
:10F960001D928A95E9F7C0906B06C652DF4FC88298
:10F97000CA5DD0408AE40F94B207882321F00E9428
:10F98000F9910C94088B86E50F941308882349F0AD
:10F990000F943406CC52DF4F79836883C45DD04026
:10F9A00006C0CC52DF4F19821882C45DD040CC52C1
:10F9B000DF4F28813981C45DD0402530310570F09A
:10F9C000EEEAF7E284918F010F5F1F4F882311F455
:10F9D0000C94088B0E944159F801F4CF84E40F94F1
:10F9E000B207882341F00E942F5BC152DF4F88830A
:10F9F000CF5DD04005C0C152DF4F1882CF5DD040EF
:10FA0000CC52DF4F48815981C45DD040433051050D
:10FA10006CF484E50F94B207882379F00E942F5B81
:10FA2000C352DF4F8883CD5DD0400CC051E0C3523C
:10FA3000DF4F5883CD5DD04005C0C352DF4F1882E1
:10FA4000CD5DD04088E50F941308882321F00F94F2
:10FA50003406162F01C012E089E50F94130888239D
:10FA600021F00F943406062F01C002E080E50F94C8
:10FA70001308811107C0CD52DF4F1883C35DD040FA
:10FA8000202E08C00F943406CD52DF4F6883C35D2B
:10FA9000D040262ECD52DF4F8881C35DD0408230CA
:10FAA00018F4E9E7F7E204C091E0921568F0F9CFA5
:10FAB00084918F010F5F1F4F882311F40C94088BE2
:10FAC0000E944159F801F4CF83E50F94130888236D
:10FAD00019F00F94440604C060E070E88BEB95E4E5
:10FAE00020E030E040E752E40F94F31E60935F02A1
:10FAF000709360028093610290936202C090470409
:10FB0000D0904804E0904904F0904A048CE40F94AB
:10FB10001308811109C020E030E040E151E4C70141
:10FB2000B6010F94161E02C00F9444060F945B1F7B
:10FB30006B017C01CA52DF4F79836883C65DD04078
:10FB40008090470490904804A0904904B0904A04E3
:10FB500082E50F941308811109C020E030E040E9EC
:10FB600053E4C501B4010F94171E02C00F9444065C
:10FB70000F945B1F4B015C01C553DF4F7983688392
:10FB8000CB5CD04040904B0450904C0460904D04AE
:10FB900070904E0486E40F941308811109C020E090
:10FBA00030E040E151E4C301B2010F94161E02C0DF
:10FBB0000F9444060F945B1FC954DF4F6883798309
:10FBC0008A839B83C75BD040C954DF4FA881B9812A
:10FBD000C75BD040C052DF4FB983A883C05ED0401E
:10FBE00040904B0450904C0460904D0470904E0433
:10FBF00082E40F941308811109C020E030E840E945
:10FC000053E4C301B2010F94171E02C00F944406BF
:10FC10000F945B1FC554DF4F688379838A839B836E
:10FC2000CB5BD040C554DF4FE881F981CB5BD0403E
:10FC3000C153DF4FF983E883CF5CD040B6018827FA
:10FC400077FD8095982F0F94EA19CA51DF4F68838A
:10FC500079838A839B83C65ED0404090470450904E
:10FC600048046090490470904A0420E030E040EA83
:10FC700051E4C301B2010F94161E9B01AC01CA519D
:10FC8000DF4F688179818A819B81C65ED0400F9465
:10FC9000E41987FD13C021E0C4010997CA52DF4F60
:10FCA00048815981C65DD040481759070CF420E0BF
:10FCB000C154DF4F2883CF5BD04006C051E0C15410
:10FCC000DF4F5883CF5BD040B401882777FD809504
:10FCD000982F0F94EA194B015C0120E030E041E9D4
:10FCE00053E4C301B2010F94171E9B01AC01C5017F
:10FCF000B4010F943D20181684F089E0C80ED11C81
:10FD000081E0C553DF4FE880F980CB5CD040CE1452
:10FD1000DF040CF480E0382E02C033243394C9543D
:10FD2000DF4F28813981C75BD040B901882777FD33
:10FD30008095982F0F94EA192B013C01C0904B0439
:10FD4000D0904C04E0904D04F0904E0420E030E060
:10FD500040EA51E4C701B6010F94161E9B01AC01A5
:10FD6000C301B2010F94E41901E087FD11C0C5542D
:10FD7000DF4F88819981CB5BD0400997C052DF4F1C
:10FD800048815981C05ED040481759070CF400E003
:10FD9000C554DF4FA881B981CB5BD040BD01882716
:10FDA00077FD8095982F0F94EA194B015C0120E0B4
:10FDB00030E847E953E4C701B6010F94171E9B01D1
:10FDC000AC01C501B4010F943D2018169CF0C95434
:10FDD000DF4F88819981C75BD040099611E0C153FC
:10FDE000DF4FC880D980CF5CD0408C159D051CF4B6
:10FDF00010E001C011E0C154DF4FD880CF5BD0408C
:10FE0000D1100CC0332029F08AE697E20E944859AD
:10FE10000BC0011109C011110DC016C082E797E295
:10FE20000E9448593110F0CF002321F082E697E27A
:10FE30000E944859112311F40C94088B8BE597E22A
:10FE40000E9448590C94088BCC52DF4FE880F9800F
:10FE5000C45DD040EF28F9F0E4E4F7E284918F012B
:10FE60000F5F1F4F882321F00E944159F801F6CF00
:10FE7000C152DF4FF880CF5DD040FF2061F0EBE250
:10FE8000F7E284918F010F5F1F4F882321F00E94BA
:10FE90004159F801F6CF0E947EFB10926B06C152C9
:10FEA000DF4FC880CF5DD040C1100AC00E942A57E2
:10FEB00087E097E00E945DA10F949B080F94A50333
:10FEC00081E00E940BEB882349F0C652DF4FD880B7
:10FED000CA5DD040D0926B060C94088B0F944B0AED
:10FEE00085E40F94B207882341F00E942F5BC45130
:10FEF000DF4F8883CC5ED04005C0C451DF4F1882ED
:10FF0000CC5ED040CD52DF4FF880C35DD040EF2CA7
:10FF1000F12CC251DF4FF982E882CE5ED040C22C74
:10FF2000D12CC051DF4FD982C882C05FD040CD52A2
:10FF3000DF4FF880C35DD040F29C70011124C552A0
:10FF4000DF4FF982E882CB5DD040C22CC0942C2DCB
:10FF50002170CD53DF4F2883C35CD040EE0CFF1CD3
:10FF6000C651DF4FF982E882CA5ED0402CEFA7016C
:10FF700024036001259FD00C1124CC50DF4FD9827F
:10FF8000C882C45FD040C552DF4FE880F980CB5DA6
:10FF9000D040EE0CFF1CEE0CFF1CCE50DF4FF98260
:10FFA000E882C25FD040C554DF4F19821882CB5B14
:10FFB000D0402FEF3FEFC954DF4F39832883C75B11
:10FFC000D040C553DF4FC880D980CB5CD040CA52E7
:10FFD000DF4FE880F980C65DD040CE18DF08C553FA
:10FFE000DF4FD982C882CB5CD040C153DF4FC8807D
:10FFF000D980CF5CD040C052DF4FE880F980C05E2E
:020000021000EC
:10000000D040CE18DF08C153DF4FD982C882CF5C01
:10001000D040C953DF4F288139814A815B81C75C59
:10002000D040CA01B9010F94C320811116C3CD532A
:10003000DF4FC880C35CD040CC2091F0CD52DF4F61
:10004000F880C35DD040CA52DF4FF882C65DD04011
:1000500021E0C052DF4F2883C05ED040312C12C057
:10006000CD52DF4F3880C35DD0403A943FEFC0524D
:10007000DF4F3883C05ED0404FEFCA52DF4F488316
:10008000C65DD04081E0CD53DF4FC880C35CD04017
:10009000C826CD53DF4FC882C35CD0409E01235C8D
:1000A0003F4FC954DF4F88819981C75BD04001968B
:1000B000C651DF4FC880D980CA5ED0408C0D9D1DCF
:1000C000880F991F880F991F280F391FC154DF4FC0
:1000D00039832883CF5BD040C251DF4F28813981DB
:1000E000CE5ED04021503109CA50DF4F398328837A
:1000F000C65FD040C051DF4F48815981C05FD040BA
:1001000041505109C850DF4F59834883C85FD040E0
:10011000C554DF4FC880D980CB5BD040EE24D7FCDC
:10012000E094FE2CC650DF4FC882D982EA82FB825F
:10013000CA5FD040CA52DF4FD880C65DD0403D1460
:1001400009F47AC2C553DF4F88819981CB5CD040D6
:10015000CA50DF4F68817981C65FD0400F94F32089
:10016000882777FD8095982F0F94EA196B017C0101
:10017000632D772767FD7095872F972F0F94EA19C6
:100180009B01AC01C701B6010F94491A9B01AC0158
:10019000CA51DF4F688179818A819B81C65ED040D8
:1001A0000F94171E4B015C01C153DF4F8881998169
:1001B000CF5CD040C850DF4F68817981C85FD040A4
:1001C0000F94F320882777FD8095982F0F94EA19D4
:1001D0006B017C01C650DF4F688179818A819B81E8
:1001E000CA5FD0400F94EA199B01AC01C701B60168
:1001F0000F94491A9B01AC01C301B2010F94171E61
:100200006B017C0120E030E0A901C501B4010F942D
:10021000E41987FF04C020E030E0A90104C020E019
:1002200030E040E05FE3C501B4010F94171E0F9466
:100230008C1FC355DF4F688379838A839B83CD5A94
:10024000D04020E030E0A901C701B6010F94E419C5
:1002500087FF04C020E030E0A90104C020E030E0C6
:1002600040E05FE3C701B6010F94171E0F948C1F87
:10027000C755DF4F688379838A839B83C95AD040EF
:10028000C954DF4F28813981C75BD0402F5F3F4F72
:10029000C954DF4F39832883C75BD040E32DEE0F6D
:1002A000FF0BC554DF4FC880D980CB5BD040EC0D2D
:1002B000FD1DEE0FFF1FA1EAEA2EF12CEC0EFD1E34
:1002C000EE0DFF1D31832083CC52DF4F2881C45DAA
:1002D000D040C451DF4F4881CC5ED040BE0167554D
:1002E0007F4FCE0183559F4F0E94B278C953DF4F95
:1002F000688379838A839B83C75CD0409B01AC0170
:100300000F94C320882341F0C652DF4FF880CA5DA6
:10031000D040F0926B0690C1C953DF4F28813981DC
:100320004A815B81C75CD040CE51DF4F68817981C3
:100330008A819B81C25ED0400F94171ECE51DF4F41
:10034000688379838A839B83C25ED040C954DF4F20
:10035000E881F981C75BD040EE0FFF1FEE0FFF1F52
:100360002DE630E02C0F3D1FE20FF31FC953DF4F86
:10037000C880D980EA80FB80C75CD040C082D1822F
:10038000E282F382C355DF4F88809980AA80BB80C8
:10039000CD5AD040C154DF4FE881F981CF5BD040C6
:1003A000CC50DF4FE880F980C45FD040EE0DFF1DD8
:1003B00080829182A282B382C755DF4FC880D980E4
:1003C000EA80FB80C95AD040CE50DF4F2881398166
:1003D000C25FD040E20FF31FC082D182E282F3827B
:1003E000C154DF4FE881F981CF5BD04080E090E0DD
:1003F000A0E8BFE381939193A193B193C154DF4FE0
:10040000F983E883CF5BD040A501940169817A81AB
:100410008B819C810F94171E69837A838B839C83C5
:10042000A70196016D817E818F8198850F94171E9B
:100430006D837E838F839887C953DF4F28813981ED
:100440004A815B81C75CD04069857A858B859C85B4
:100450000F94171E69877A878B879C87A501940163
:10046000C501B4010F94491A9B01AC016D857E85CD
:100470008F8598890F94171E6D877E878F87988B3D
:10048000A7019601C701B6010F94491A9B01AC015F
:1004900069897A898B899C890F94171E698B7A8B5D
:1004A0008B8B9C8BC953DF4F288139814A815B81BB
:1004B000C75CD040CA01B9010F94491A9B01AC0135
:1004C0006D897E898F89988D0F94171E6D8B7E8B19
:1004D0008F8B988FA7019601C501B4010F94491A1B
:1004E0009B01AC01698D7A8D8B8D9C8D0F94171EAD
:1004F000698F7A8F8B8F9C8FC953DF4F2881398109
:100500004A815B81C75CD040C501B4010F94491A90
:100510009B01AC016D8D7E8D8F8D98A10F94171E60
:100520006D8F7E8F8F8F98A3C953DF4F28813981BC
:100530004A815B81C75CD040C701B6010F94491A5C
:100540009B01AC0169A17AA18BA19CA10F94171EFC
:1005500069A37AA38BA39CA3E894B7F81DA10EA16D
:10056000FFA1C652DF4FF883CA5DD04028A5C35112
:10057000DF4F2883CD5ED040212F302F4F2FC35126
:10058000DF4F5881CD5ED040C501B4010F943D20AE
:1005900018162CF4182D092D3A2D2B2D0AC0C652F1
:1005A000DF4F3881CA5DD040C351DF4F2881CD5E17
:1005B000D040812F902FA32FB22F8DA39EA3AFA346
:1005C000B8A746015701E894B7F819A50AA5FBA4F6
:1005D000ECA4212F302F4F2D5E2DC501B4010F94B7
:1005E0003D20181624F4182D092DFA2CEB2C812F00
:1005F000902FAF2DBE2D89A79AA7ABA7BCA720E04F
:1006000030E040E85FE369AD7AAD8BAD9CAD0F940F
:10061000171E69AF7AAF8BAF9CAF80E00E9455F197
:10062000C052DF4FC880C05ED0403C0CC652DF4F86
:100630001882CA5DD0407ECDC554DF4F28813981F4
:10064000CB5BD0402F5F3F4FC554DF4F39832883AA
:10065000CB5BD040221508F4DCCC80E00E940BEB91
:10066000882341F0C652DF4FC880CA5DD040C09297
:100670006B06C5C7C953DF4F288139814A815B8129
:10068000C75CD040CA01B9010F94C3208111B7C71C
:1006900089AC9AACABACBCAC20E030E0A901C501A0
:1006A000B4010F94E419882309F408C2A501940148
:1006B00069817A818B819C810F94F31EC954DF4F2D
:1006C000688379838A839B83C75BD04069837A83FD
:1006D0008B839C83A50194016D817E818F81988598
:1006E0000F94F31EC554DF4F688379838A839B83FD
:1006F000CB5BD0406D837E838F839887A501940167
:1007000069857A858B859C850F94F31EC154DF4FD4
:10071000688379838A839B83CF5BD04069877A879C
:100720008B879C87A50194016D857E858F8598892F
:100730000F94F31E6B017C01C954DF4F288139816E
:100740004A815B81C75BD040CA01B9010F94491A45
:100750009B01AC01C701B6010F94161EC553DF4FB4
:10076000688379838A839B83CB5CD0406D877E8747
:100770008F87988BA501940169897A898B899C89D7
:100780000F94F31E6B017C01C554DF4F2881398122
:100790004A815B81CB5BD040CA01B9010F94491AF1
:1007A0009B01AC01C701B6010F94161EC153DF4F68
:1007B000688379838A839B83CF5CD040698B7A8BF3
:1007C0008B8B9C8BA50194016D897E898F89988D77
:1007D0000F94F31E6B017C01C154DF4F28813981D6
:1007E0004A815B81CF5BD040CA01B9010F94491A9D
:1007F0009B01AC01C701B6010F94161E6D8B7E8B59
:100800008F8B988FA5019401698D7A8D8B8D9C8D2E
:100810000F94F31E6B017C01C554DF4F2881398191
:100820004A815B81CB5BD040C954DF4F68817981BD
:100830008A819B81C75BD0400F94491A9B01AC0110
:10084000C701B6010F94161ECD53DF4F688379831D
:100850008A839B83C35CD040698F7A8F8B8F9C8FF8
:10086000A501940169A17AA18BA19CA10F94F31E0B
:100870006B017C01C154DF4F288139814A815B8142
:10088000CF5BD040C554DF4F688179818A819B81DD
:10089000CB5BD0400F94491A9B01AC01C701B60154
:1008A0000F94161E6B017C0169A37AA38BA39CA3F2
:1008B000A50194016D8D7E8D8F8D98A10F94F31EEF
:1008C0004B015C01C154DF4F288139814A815B8132
:1008D000CF5BD040C954DF4F688179818A819B8189
:1008E000C75BD0400F94491A9B01AC01C501B4010C
:1008F0000F94161E4B015C016D8F7E8F8F8F98A316
:10090000C153DF4F288139814A815B81CF5CD04060
:10091000C553DF4F688179818A819B81CB5CD04050
:100920000F94491A2B013C01CD53DF4F28813981A7
:100930004A815B81C35CD040CA01B9010F94491A56
:100940009B01AC01C301B2010F94161ECA52DF4FC6
:10095000688379838A839B83C65DD0402B013C01E9
:10096000E89477F829A53AA54BA55CA56DA17EA1D1
:100970008FA198A50F94171E2FEF36EE4BED5EE278
:100980000F94491A9B01AC01C301B2010F94E41901
:1009900018160CF093C0CD53DF4F288139814A815E
:1009A0005B81C35CD040C701B6010F94491A2B018B
:1009B0003C01C153DF4F288139814A815B81CF5C83
:1009C000D040C501B4010F94491A9B01AC01C30189
:1009D000B2010F94161ECA52DF4F288139814A8115
:1009E0005B81C65DD0400F94F31E2B013C016DA7C7
:1009F0007EA78FA798ABCD53DF4F288139814A81DD
:100A00005B81C35CD040C501B4010F94491A4B010E
:100A10005C01C553DF4F288139814A815B81CB5C02
:100A2000D040C701B6010F94491A9B01AC01C50122
:100A3000B4010F94161ECA52DF4F288139814A81B2
:100A40005B81C65DD0400F94F31E6B017C0169ABE6
:100A50007AAB8BAB9CABC954DF4F288139814A817B
:100A60005B81C75BD040C301B2010F94491A9B015F
:100A7000AC01C154DF4F688179818A819B81CF5B52
:100A8000D0400F94171E4B015C01C554DF4F2881E5
:100A900039814A815B81CB5BD040C701B6010F949D
:100AA000491A9B01AC01C501B4010F94171EDC016A
:100AB000CB01B0588DAB9EABAFABB8AFCDA4DEA42D
:100AC000EFA4F8A82601370177FA709477F87094AC
:100AD00089A89AA8ABA8BCA82DA93EA94FA958AD32
:100AE000C954DF4F288339834A835B83C75BD04077
:100AF000C552DF4F48815981CB5DD040BA0188276C
:100B000077FD8095982F0F94EA199B01AC01CE5187
:100B1000DF4F688179818A819B81C25ED0400F94CA
:100B2000F31EC153DF4F688379838A839B83CF5C35
:100B3000D040CC52DF4F88819981C45DD040892B51
:100B400009F460C0E5E1F7E284918F010F5F1F4F68
:100B5000882321F00E944159F801F6CF48E0C301F3
:100B6000B2010E941D4DE0E1F7E284918F010F5F19
:100B70001F4F882321F00E944159F801F6CF48E029
:100B8000C501B40190580E941D4DEBE0F7E284913D
:100B90008F010F5F1F4F882321F00E944159F801F8
:100BA000F6CFC954DF4F688179818A819B81C75B09
:100BB000D040905848E00E941D4D8AE00E94415963
:100BC000CC52DF4FA881B981C45DD0401397D4F0D7
:100BD000E2EFF6E284918F010F5F1F4F882321F02F
:100BE0000E944159F801F6CF48E0C153DF4F6881B8
:100BF00079818A819B81CF5CD0400E941D4D8AE023
:100C00000E944159C152DF4FB881CF5DD040B11130
:100C1000D1C1CB56DF4FC882D982EA82FB82C55947
:100C2000D040C756DF4F88829982AA82BB82C959B9
:100C3000D040C12CD12C50E8E52E5FE3F52EC356F1
:100C4000DF4FC882D982EA82FB82CD59D040CE01E3
:100C50008B569F4F0E94E39FC757DF4FC882D982B0
:100C6000EA82FB82C958D040C357DF4F18821982ED
:100C70001A821B82CD58D040CF56DF4F488259820E
:100C80006A827B82C159D040CE0187579F4F0E9414
:100C9000E39FCB56DF4FC880D980EA80FB80C559DF
:100CA000D040C954DF4FC882D982EA82FB82C75B39
:100CB000D040C756DF4F488059806A807B80C95931
:100CC000D040C356DF4F88809980AA80BB80CD5921
:100CD000D040C757DF4FC880D980EA80FB80C95811
:100CE000D040C554DF4FC882D982EA82FB82CB5BF9
:100CF000D040C357DF4FC880D980EA80FB80CD58F1
:100D0000D040C154DF4FC882D982EA82FB82CF5BD8
:100D1000D040CF56DF4FC880D980EA80FB80C159D0
:100D2000D040A7019601C301B2010F94491ACD53D7
:100D3000DF4F688379838A839B83C35CD040C1542F
:100D4000DF4F288139814A815B81CF5BD040C5016B
:100D5000B4010F94491A9B01AC01CD53DF4F688158
:100D600079818A819B81C35CD0400F94161EC35841
:100D7000DF4F688379838A839B83CD57D040C554E6
:100D8000DF4F288139814A815B81CB5BD040C5012F
:100D9000B4010F94491A4B015C01A7019601C95493
:100DA000DF4F688179818A819B81C75BD0400F9436
:100DB000491A9B01AC01C501B4010F94161ECF570F
:100DC000DF4F688379838A839B83C158D040C154A5
:100DD000DF4F288139814A815B81CF5BD040C95484
:100DE000DF4F688179818A819B81C75BD0400F94F6
:100DF000491A6B017C01C554DF4F288139814A8132
:100E00005B81CB5BD040C301B2010F94491A9B01B7
:100E1000AC01C701B6010F94161ECB57DF4F688394
:100E200079838A839B83C558D040CE0183589F4FD6
:100E30000E94E39FC757DF4F88809980AA80BB80BC
:100E4000C958D040C357DF4FC880D980EA80FB80A3
:100E5000CD58D040CF56DF4F488059806A807B8084
:100E6000C159D040C358DF4F288139814A815B8105
:100E7000CD57D040C954DF4F288339834A835B83E1
:100E8000C75BD040CF57DF4F88819981AA81BB8152
:100E9000C158D040C554DF4F88839983AA83BB8350
:100EA000CB5BD040CB57DF4F288139814A815B81B2
:100EB000C558D040C154DF4F288339834A835B83B0
:100EC000CF5BD040CB56DF4F088119812A813B810F
:100ED000C559D040C756DF4F488159816A817B810F
:100EE000C959D040C356DF4F88819981AA81BB81FF
:100EF000CD59D0408092E7119092E811A092E9116B
:100F0000B092EA11C092EB11D092EC11E092ED1187
:100F1000F092EE114092EF115092F0116092F111A7
:100F20007092F211C954DF4FC880D980EA80FB80EB
:100F3000C75BD040C092F311D092F411E092F5114A
:100F4000F092F611C554DF4FC880D980EA80FB804B
:100F5000CB5BD040C092F711D092F811E092F9111A
:100F6000F092FA11C154DF4FC880D980EA80FB802B
:100F7000CF5BD040C092FB11D092FC11E092FD11EA
:100F8000F092FE110093FF111093001220930112B2
:100F9000309302124093031250930412609305128F
:100FA000709306128093071290930812A09309126F
:100FB000B0930A12C352DF4FD880CD5DD040DD2000
:100FC00009F47EC2EFE2F6E284918F010F5F1F4FBA
:100FD000882321F00E944159F801F6CF44244A9415
:100FE000420C542CC554DF4F1882CB5BD04020EC10
:100FF000C154DF4F2883CF5BD04039E7CD53DF4F5B
:101000003883C35CD04044E4C553DF4F4883CB5C96
:10101000D040CE018B569F4FCF54DF4F99838883AA
:10102000C15BD040DE01A757BF4FCD54DF4FB9831E
:10103000A883C35BD040FE01E358FF4FCB54DF4F82
:10104000F983E883C55BD04057FC29C1652C660C49
:10105000770821EAE22EF12CEC0EFD1E6E0C7F1CAF
:10106000212C312CC954DF4F1882C75BD040F301CB
:10107000E20DF31DC080D180C352DF4FD982C882F8
:10108000CD5DD0408601000F111F000F111FEDE64E
:10109000F0E0EC0FFD1FE00FF11F80809180A28037
:1010A000B380C153DF4F288139814A815B81CF5C96
:1010B000D040C501B4010F94161E6B017C01E1E024
:1010C000F0E0EC0FFD1FE00FF11F84AD95ADA6AD74
:1010D000B7ADCB56DF4F88839983AA83BB83C559AD
:1010E000D040C352DF4FE881F981CD5DD040C55279
:1010F000DF4F28813981CB5DD040E20FF31FEE0F27
:10110000FF1FEE0FFF1F41E050E04C0F5D1FE40F8B
:10111000F51F84AD95ADA6ADB7ADC757DF4F88833A
:101120009983AA83BB83C958D040C358DF4F188224
:1011300019821A821B82CD57D040CA54DF4F588182
:10114000C65BD0405F93CB54DF4F8881C55BD040F6
:101150008F93CC54DF4F9881C45BD0409F93CD5484
:10116000DF4FA881C35BD040AF93CE54DF4FB8812F
:10117000C25BD040BF93CF54DF4FE881C15BD0400A
:10118000EF932DB73EB7245231090FB6F8943EBF06
:101190000FBE2DBFADB7BEB71196E7EEF1E184E209
:1011A00001900D928A95E1F70E9478A0C358DF4F15
:1011B000288139814A815B81CD57D040C501B40176
:1011C0000F94161E5B018C010FB6F894DEBF0FBEA4
:1011D000CDBF9B01AC01C554DF4F6881CB5BD040D4
:1011E000C154DF4F7881CF5BD040CD53DF4F888132
:1011F000C35CD040C553DF4F9881CB5CD0400F9487
:101200003D201816A4F4C554DF4FA882CB5BD04014
:10121000C154DF4FB882CF5BD040CD53DF4F08833E
:10122000C35CD040C553DF4F1883CB5CD04020E077
:1012300030E0A901C701B6010F943D2087FD0CC025
:10124000ECE2F6E284918F010F5F1F4F882339F0A3
:101250000E944159F801F6CF80E20E94415945E0D1
:10126000C701B6010E941D4DC954DF4F5881C75BAD
:10127000D0405F5FC954DF4F5883C75BD04084E0E4
:10128000280E311CCD52DF4FC880C35DD0405C15A5
:1012900008F4EDCE8AE00E9441595A94D5CE8AE0F6
:1012A0000E944159CC52DF4F28813981C45DD04022
:1012B0002430310509F004C1E3E0F6E284918F01A6
:1012C0000F5F1F4F811112C0AE014B565F4FCF54BD
:1012D000DF4F59834883C15BD0401E0159E8250E7A
:1012E000311C3E018DE7680E711C1AC00E944159E5
:1012F000F801E4CF80E20E94415945E0C501B40104
:101300000E941D4DD3940C5F1F4FCD52DF4FF881CB
:10131000C35DD040DF16A8F08AE00E9441594A948C
:1013200047FCCAC0E42CEE0CFF08A1EACA2ED12C5F
:10133000CC0EDD1EEC0CFD1C00E010E0D12CB4E264
:10134000CB2EF701E00FF11F0190F081E02D5F013E
:10135000AA0CBB1CAA0CBB1CA1E0B0E0AC0FBD1FCB
:10136000AA0DBB1DDC968D919D910D90BC91A02D79
:10137000CB56DF4F88839983AA83BB83C559D0405E
:10138000C552DF4FA881B981CB5DD040EA0FFB1F6A
:10139000EE0FFF1FEE0FFF1F21E030E02C0F3D1F6F
:1013A000E20FF31F84AD95ADA6ADB7ADF10180831B
:1013B0009183A283B383D3011D921D921D921C922F
:1013C00013977F926F923F922F92CE54DF4FB88146
:1013D000C25BD040BF93CF54DF4FE881C15BD040A8
:1013E000EF932DB73EB7245231090FB6F8943EBFA4
:1013F0000FBE2DBFADB7BEB71196E7EEF1E18C2D54
:1014000001900D928A95E1F70E9478A0EDE6F0E058
:10141000EC0FFD1FEA0DFB1DD3012D913D914D9168
:101420005C9160817181828193810F94161EC554F5
:10143000DF4F2881CB5BD040C154DF4F3881CF5B79
:10144000D040CD53DF4F4881C35CD040C553DF4F00
:101450005881CB5CD0400F94161E4B015C010FB637
:10146000F894DEBF0FBECDBF20E030E0A9010F949D
:101470003D2087FD3FCFE0E0F6E284919F012F5FA2
:101480003F4F882309F439CFC250DF4F2883CE5F06
:10149000D040C150DF4F3883CF5FD0400E944159C8
:1014A000C250DF4F2881CE5FD040C150DF4F38811E
:1014B000CF5FD040F901E1CF8AE00E94415908C0D6
:1014C000CC52DF4FE880F980C45DD040EF2821F096
:1014D00081EE95E20E9452C0C152DF4FF880CF5D8D
:1014E000D040F11085C08CE0ECE7F7E0DE01A358B6
:1014F000BF4F01900D928A95E1F781E080936B06D2
:10150000CE0183589F4F0E945DA1C355DF4F2881B4
:1015100039814A815B81CD5AD04060917C077091BE
:101520007D0780917E0790917F070F94161E6B01B7
:101530007C012DEB37E346E855EB0F943D2087FD0A
:101540004BC02DEB37E346E855E3C701B6010F94D6
:10155000E41918160CF440C0C755DF4F28813981B3
:101560004A815B81C95AD0406091800770918107A0
:1015700080918207909183070F94161E6B017C0166
:101580002DEB37E346E855EB0F943D2087FD24C053
:101590002DEB37E346E855E3C701B6010F94E41994
:1015A0001816D4F0C953DF4F288139814A815B81F5
:1015B000C75CD04060918407709185078091860751
:1015C000909187070F94161ECB57DF4F688379835E
:1015D0008A839B83C558D0408CE0FE01E358FF4FBF
:1015E000ACE7B7E001900D928A95E1F781E005C084
:1015F000C652DF4F8881CA5DD04080936B060F943E
:10160000320A0E9493BF80916B0681110F94A5034B
:10161000C150DF4F0FB6F894DEBF0FBECDBFDF91D4
:10162000CF911F910F91FF90EF90DF90CF90BF90DF
:10163000AF909F908F907F906F905F904F903F9072
:101640002F9008952F923F924F925F926F927F92C8
:101650008F929F92AF92BF92CF92DF92EF92FF92C2
:101660000F931F93CF93DF93CDB7DEB72B970FB6B2
:10167000F894DEBF0FBECDBF9E838D83DC015996EB
:101680002D903C905A97F101418452846384748474
:10169000FFEF4F1A5F0A6F0A7F0A1496CD90DD9014
:1016A000ED90FC901797C114D104E104F10439F0D6
:1016B0002FEFC21AD20AE20AF20A1B8607C0D10132
:1016C000CD90DD90ED90FC90B1E0BB8746015701D5
:1016D0001F82188619861A86F10181859285A38555
:1016E000B4852F81388549855A85281739074A07D7
:1016F0005B0708F08DC04C145D046E047F0450F449
:1017000082E0C82ED12CE12CF12C92E0892E912C74
:10171000A12CB12C9E012F5F3F4FB701A601C10143
:101720000E946472882309F473C089819A81AB8115
:10173000BC81892B8A2B8B2B41F0460157013FEF4F
:10174000831A930AA30AB30A05C0C814D904EA0489
:10175000FB0489F08F819885A985BA850196A11D22
:10176000B11D8F839887A987BA879FEFC91AD90AB5
:10177000E90AF90AB1CF0FEF1FEF2FEF3FE0B501F4
:10178000A401C1010E94AD75F82E882309F440C060
:10179000ED81FE8144815581668177814115510536
:1017A0006105710539F095018401C1010E94AD7593
:1017B000882371F1AD81BE8114968D929D92AD9278
:1017C000BC921797BB85BB2351F0D501C40101968C
:1017D000A11DB11DF10180839183A283B383ED81AB
:1017E000FE8185899689A789B08D892B8A2B8B2BC1
:1017F00081F4AD81BE8155968D929D92AD92BC9241
:10180000589711968C911197806811968C9301C00E
:10181000F12C8F2D2B960FB6F894DEBF0FBECDBFE7
:10182000DF91CF911F910F91FF90EF90DF90CF90BC
:10183000BF90AF909F908F907F906F905F904F90F0
:101840003F902F900895CF93DF93EC018B818823F5
:1018500091F1898187FF2BC06C857D858E859F8561
:1018600041E00E94D470882331F1E88980E2E89F4A
:10187000F0011124E95AFB4F3097E9F08081853E51
:10188000D1F08B81823040F449895A896B897C89F7
:10189000448F558F668F778F4D895E896F89788DDC
:1018A000538F428F758B648B89818F778983DF910A
:1018B000CF910C94967081E0888380E0DF91CF9186
:1018C0000895CF93DF93EC018B81813099F4898166
:1018D00081FF10C049895A896B897C89452B462B29
:1018E000472B59F140E050E0BA01CE010E945D74EF
:1018F000811102C080E022C04D895E896F89788D98
:10190000898D9A8D0E943C768823A1F31D8A1E8AB8
:101910001F8A188E198A1A8A1B8A1C8A89818068F4
:101920008983CE0190DF882329F340E050E0BA019B
:10193000CE01DF91CF910C945D7481E0DF91CF9166
:1019400008956F927F928F929F92AF92BF92CF92A3
:10195000DF92EF92FF920F931F93CF93DF931F922B
:10196000CDB7DEB78C015B014A01722EDB015996BF
:101970008D919C915A97F801928F818F40E050E0B1
:10198000BA01C5010E945D74E12CF5018085918545
:10199000A285B38541895289638974898417950723
:1019A000A607B70708F0CEC035E0B695A79597957E
:1019B00087953A95D1F7F82FFF70FF2ED501139632
:1019C0008C91823008F49BC141E050E0BE016F5F12
:1019D0007F4FC5010E94E372019719F4898190E05D
:1019E00002C08FEF9FEF019609F489C1F501808550
:1019F0009185A285B3854F96A11DB11D80879187E2
:101A0000A287B387F0E2FF9EB0011124695A7B4F91
:101A10006115710509F473C1DB018C91882311F004
:101A2000853EB9F4E1100EC080911607909117071A
:101A3000A0911807B0911907F80184879587A687A8
:101A4000B787F08ADB018C91EE24E39481119DCF5E
:101A500079C04BE050E0C4010F941821892B09F0A4
:101A600094CF77FC4CC120E2F29EF0011124E95A98
:101A7000FB4F8385817121F0872D827109F05EC053
:101A80004091160750911707609118077091190738
:101A9000D8011C964D935D936D937C931F97509640
:101AA000FC924489558960E070E0BA0155274427CB
:101AB000828D938DA0E0B0E0482B592B6A2B7B2BB5
:101AC000D80155964D935D936D937C93589783857C
:101AD000887159F4848D958DA68DB78DF801818B11
:101AE000928BA38BB48B81E010C0803139F59801C3
:101AF0002F5E3F4FD80159968D919C915A970E9425
:101B0000F6748823D9F084E0F8018383872D8F70E1
:101B1000D80111968C931197F801148215821682C0
:101B2000178218961D921D921D921C921B9774FE8F
:101B3000D9C0C801C6DE8111D5C0E2C0D801139654
:101B40001C92DDC0872D8274823409F0D8C0EE204B
:101B5000E1F0D8015096FC9050971C966D917D91C4
:101B60008D919C911F9741E00E94D470882309F4C5
:101B7000C6C0F8018089F0E28F9FC0011124895A04
:101B80009B4F009709F08EC0BAC0D50113968C9177
:101B90001397823009F4B3C051968D919D910D90A9
:101BA000BC91A02D803E9F4FAF41B10508F0A7C06A
:101BB000C50148DD882309F4A2C00E9496708823DD
:101BC00009F49DC0D5015996ED91FC915A97149650
:101BD000CD90DD90ED90FC901797B2E0CB1AD10834
:101BE000E108F108058404C0CC0CDD1CEE1CFF1CD0
:101BF0000A94D2F786859785A089B189C80ED91E27
:101C0000EA1EFB1E81E080931507C0921607D09252
